:100000000C94C74A0C94614B0C94614B0C94614B5B
:100010000C94614B0C94614B0C94614B0C94614BB0
:100020000C94614B0C94614B0C94614B0C94614BA0
:100030000C94614B0C94BF4C0C94614B0C94614B31
:100040000C94614B0C94614B0C94614B0C94614B80
:100050000C94614B0C94614B0C94614B0C94614B70
:100060000C94614B0C94614B0C94614B0C94614B60
:100070005A5501200101003808000000000000006E
:100080000000000000000000000000000000000070
:100090005E556C554756305A1A5A6F557E558D55D8
:1000A000015A9B55A95513021C1D001E1F2000213B
:1000B000222324252600002728292A002B2C2D2E38
:1000C0002F303132333435363738393A3B3C0E0530
:1000D0001800001800191919190018181818180014
:1000E000001800000019190018000000180000187E
:1000F0000000190000001818180018000018001956
:10010000000000001800000000181800001919195C
:100110001900181818180E051919190000181818C0
:100120001800190000191900001900180000180023
:1001300000191900191919000018000018000019F9
:100140001900190000190018000018001900001902
:1001500019191900001818181800190000190E05AF
:1001600019191919001800001800001919001900B0
:1001700000000018180018001900001900191900D3
:100180000018001818001919191900000019001892
:100190000018180019000019191919190018000081
:1001A0001800190000190E05180000180019191977
:1001B000190018181818180018000019000000007D
:1001C0001800000018180000001919190000001884
:1001D00018001800180000190000000000000018A6
:1001E00018000018001919191900181818180FEF1D
:1001F00008B919910FEF08B9159F0FEF08B9080E4C
:10020000191E0FEF08B9F9014A950FEF08B909F067
:10021000F0010FEF08B909940FEF08B919910FEF2A
:1002200008B9159F0FEF08B9080E191E0FEF08B98E
:10023000F9014A950FEF08B909F0F0010FEF08B97D
:1002400009940FEF08B919910FEF08B9159F0FEF37
:1002500008B9080E191E0FEF08B9F9014A950FEFFA
:1002600008B909F0F0010FEF08B909940FEF08B9C8
:1002700019910FEF08B9159F0FEF08B9080E191E55
:100280000FEF08B9F9014A950FEF08B909F0F0012D
:100290000FEF08B909940FEF08B919910FEF08B9DA
:1002A000159F0FEF08B9080E191E0FEF08B9F901D5
:1002B0004A950FEF08B909F0F0010FEF08B909945A
:1002C0000FEF08B919910FEF08B9159F0FEF08B993
:1002D000080E191E0FEF08B9F9014A950FEF08B97A
:1002E00009F0F0010FEF08B909940FEF08B919915F
:1002F0000FEF08B9159F0FEF08B9080E191E0FEF81
:1003000008B9F9014A950FEF08B909F0F0010FEFAC
:1003100008B909940FEF08B919910FEF08B9159FA3
:100320000FEF08B9080E191E0FEF08B9F9014A9529
:100330000FEF08B909F0F0010FEF08B9099406E3CF
:1003400008B9199106E308B9159F06E308B9080E24
:10035000191E06E308B9F9014A9506E308B909F040
:10036000F00106E308B9099406E308B9199106E318
:1003700008B9159F06E308B9080E191E06E308B967
:10038000F9014A9506E308B909F0F00106E308B956
:10039000099406E308B9199106E308B9159F06E325
:1003A00008B9080E191E06E308B9F9014A9506E3D3
:1003B00008B909F0F00106E308B9099406E308B9A1
:1003C000199106E308B9159F06E308B9080E191E2E
:1003D00006E308B9F9014A9506E308B909F0F00106
:1003E00006E308B9099406E308B9199106E308B9C8
:1003F000159F06E308B9080E191E06E308B9F901AE
:100400004A9506E308B909F0F00106E308B9099432
:1004100006E308B9199106E308B9159F06E308B980
:10042000080E191E06E308B9F9014A9506E308B952
:1004300009F0F00106E308B9099406E308B9199137
:1004400006E308B9159F06E308B9080E191E06E36E
:1004500008B9F9014A9506E308B909F0F00106E385
:1004600008B9099406E308B9199106E308B9159F7C
:1004700006E308B9080E191E06E308B9F9014A9502
:1004800006E308B909F0F00106E308B9099401E8A8
:1004900008B9199101E808B9159F01E808B9080ED3
:1004A000191E01E808B9F9014A950EE708B909F0E3
:1004B000F0010EE708B9099401E808B9199101E8BB
:1004C00008B9159F0EE708B9080E191E0EE708B9FE
:1004D000F9014A9501E808B909F0F00101E808B905
:1004E00009940EE708B919910EE708B9159F01E8BC
:1004F00008B9080E191E01E808B9F9014A9501E882
:1005000008B909F0F00101E808B9099401E808B94F
:10051000199101E808B9159F01E808B9080E191EDC
:1005200001E808B9F9014A9501E808B909F0F001B4
:1005300001E808B9099401E808B9199101E808B976
:10054000159F01E808B9080E191E01E808B9F9015C
:100550004A950EE708B909F0F0010EE708B90994C9
:1005600001E808B9199101E808B9159F0EE708B923
:10057000080E191E0EE708B9F9014A9501E808B9F5
:1005800009F0F00101E808B909940EE708B91991DA
:100590000EE708B9159F01E808B9080E191E01E811
:1005A00008B9F9014A9501E808B909F0F00101E834
:1005B00008B9099401E808B9199101E808B9159F2B
:1005C00001E808B9080E191E01E808B9F9014A95B1
:1005D00001E808B909F0F00101E808B9099406E357
:1005E00008B9199106E308B9159F09E208B9080E80
:1005F000191E09E208B9F9014A9506E308B909F09C
:10060000F00106E308B9099406E308B9199109E273
:1006100008B9159F09E208B9080E191E09E208B9C0
:10062000F9014A9509E208B909F0F00106E308B9B1
:10063000099406E308B9199109E208B9159F09E27E
:1006400008B9080E191E09E208B9F9014A9509E22C
:1006500008B909F0F00106E308B9099408E108B9FE
:10066000199108E108B9159F09E208B9080E191E89
:1006700009E208B9F9014A9509E208B909F0F0015F
:1006800009E208B9099409E208B919910FE008B91B
:10069000159F08E108B9080E191E09E208B9F90109
:1006A0004A950FE008B909F0F00109E208B9099488
:1006B00009E208B9199109E208B9159F09E208B9D8
:1006C000080E191E08E108B9F9014A9508E108B9B0
:1006D00009F0F00108E108B9099409E208B9199193
:1006E00009E208B9159F09E208B9080E191E09E2C6
:1006F00008B9F9014A9509E208B909F0F00109E2DF
:1007000008B9099409E208B9199109E208B9159FD5
:1007100009E208B9080E191E09E208B9F9014A955B
:1007200009E208B909F0F00109E208B9099409E2FF
:1007300008B9199109E208B9159F06E308B9080E2E
:10074000191E06E308B9F9014A9506E308B909F04C
:10075000F00106E308B9099409E208B9199109E220
:1007600008B9159F09E208B9080E191E06E308B971
:10077000F9014A9506E308B909F0F00106E308B962
:10078000099409E208B9199109E208B9159F0FE027
:1007900008B9080E191E08E108B9F9014A9509E2DD
:1007A00008B909F0F00106E308B9099409E208B9AB
:1007B000199109E208B9159F08E108B9080E191E38
:1007C00009E208B9F9014A9509E208B909F0F0010E
:1007D00009E208B9099409E208B9199108E108B9D0
:1007E000159F09E208B9080E191E09E208B9F901B6
:1007F0004A9509E208B909F0F00109E208B909943B
:1008000009E208B9199108E108B9159F0FE008B984
:10081000080E191E09E208B9F9014A9509E208B95A
:1008200009F0F00106E308B9099409E208B9199141
:1008300008E108B9159F09E208B9080E191E06E378
:1008400008B9F9014A9506E308B909F0F00106E391
:1008500008B9099408E108B9199109E208B9159F86
:1008600006E308B9080E191E06E308B9F9014A950E
:1008700006E308B909F0F00106E308B9099409E2B2
:1008800008B9199109E208B9159F09E208B9080EDB
:10089000191E09E208B9F9014A9509E208B909F0F7
:1008A000F00109E208B9099409E208B9199109E2CD
:1008B00008B9159F09E208B9080E191E09E208B91E
:1008C000F9014A9509E208B909F0F00109E208B90D
:1008D000099408E108B9199108E108B9159F08E1E0
:1008E00008B9080E191E09E208B9F9014A9509E28A
:1008F00008B909F0F00109E208B9099409E208B958
:1009000019910FE008B9159F09E208B9080E191EE0
:1009100008E108B9F9014A950FE008B909F0F001BA
:1009200009E208B9099409E208B9199109E208B97C
:10093000159F09E208B9080E191E09E208B9F90164
:100940004A9508E108B909F0F00108E108B90994ED
:1009500006E308B9199109E208B9159F09E208B937
:10096000080E191E09E208B9F9014A9509E208B909
:1009700009F0F00106E308B9099406E308B91991F2
:1009800009E208B9159F09E208B9080E191E09E223
:1009900008B9F9014A9509E208B909F0F00106E33E
:1009A00008B9099406E308B9199106E308B9159F37
:1009B00009E208B9080E191E09E208B9F9014A95B9
:1009C00006E308B909F0F00106E308B9099406E363
:1009D00008B9199106E308B9159F06E308B9080E8E
:1009E000191E06E308B9F9014A9509E208B909F0A8
:1009F000F00108E108B9099406E308B9199106E382
:100A000008B9159F06E308B9080E191E09E208B9CE
:100A1000F9014A9508E108B909F0F00109E208B9BD
:100A2000099406E308B9199109E208B9159F09E28A
:100A300008B9080E191E0FE008B9F9014A9508E136
:100A400008B909F0F00109E208B9099409E208B906
:100A5000199109E208B9159F09E208B9080E191E93
:100A600009E208B9F9014A9508E108B909F0F0016D
:100A700009E208B9099409E208B9199109E208B92B
:100A8000159F09E208B9080E191E08E108B9F90115
:100A90004A9509E208B909F0F00109E208B9099498
:100AA00006E308B9199109E208B9159F08E108B9E8
:100AB000080E191E0FE008B9F9014A9509E208B9B4
:100AC00009F0F00109E208B9099406E308B919919F
:100AD00006E308B9159F06E308B9080E191E09E2D6
:100AE00008B9F9014A9509E208B909F0F00109E2EB
:100AF00008B9099406E308B9199106E308B9159FE6
:100B000006E308B9080E191E06E308B9F9014A956B
:100B100009E208B909F0F00109E208B9099409E20B
:100B200008B9199108E108B9159F09E208B9080E3A
:100B3000191E08E108B9F9014A9509E208B909F056
:100B4000F00109E208B9099408E108B9199109E22C
:100B500008B9159F09E208B9080E191E09E208B97B
:100B6000F9014A9508E108B909F0F00109E208B96C
:100B7000099408E108B9199109E208B9159F09E239
:100B800008B9080E191E08E108B9F9014A9509E2E9
:100B900008B909F0F00108E108B9099409E208B9B7
:100BA000199109E208B9159F09E208B9080E191E42
:100BB00008E108B9F9014A9509E208B909F0F0011C
:100BC00009E208B9099409E208B9199109E208B9DA
:100BD000159F08E108B9080E191E09E208B9F901C4
:100BE0004A9508E108B909F0F00109E208B9099449
:100BF00009E208B9199108E108B9159F09E208B995
:100C0000080E191E09E208B9F9014A9508E108B968
:100C100009F0F00109E208B9099408E108B919914D
:100C200009E208B9159F09E208B9080E191E08E182
:100C300008B9F9014A9509E208B909F0F00109E299
:100C400008B9099409E208B9199108E108B9159F92
:100C500009E208B9080E191E08E108B9F9014A9518
:100C600009E208B909F0F00109E208B9099409E2BA
:100C700008B9199109E208B9159F09E208B9080EE7
:100C8000191E09E208B9F9014A9509E208B909F003
:100C9000F00109E208B9099409E208B9199109E2D9
:100CA00008B9159F09E208B9080E191E09E208B92A
:100CB000F9014A9509E208B909F0F00108E108B91B
:100CC000099409E208B9199109E208B9159F09E2E6
:100CD00008B9080E191E08E108B9F9014A9508E19A
:100CE00008B909F0F00109E208B9099408E108B966
:100CF000199108E108B9159F09E208B9080E191EF3
:100D000009E208B9F9014A9509E208B909F0F001C8
:100D100009E208B9099409E208B9199109E208B988
:100D2000159F08E108B9080E191E08E108B9F90174
:100D30004A9509E208B909F0F00109E208B90994F5
:100D400009E208B9199109E208B9159F09E208B941
:100D5000080E191E09E208B9F9014A9508E108B917
:100D600009F0F00109E208B9099406E308B91991FC
:100D700009E208B9159F09E208B9080E191E09E22F
:100D800008B9F9014A9509E208B909F0F00106E34A
:100D900008B9099406E308B9199106E308B9159F43
:100DA00009E208B9080E191E09E208B9F9014A95C5
:100DB00006E308B909F0F00106E308B9099406E36F
:100DC00008B9199106E308B9159F06E308B9080E9A
:100DD000191E09E208B9F9014A9508E108B909F0B4
:100DE000F00109E208B9099406E308B9199106E38C
:100DF00008B9159F09E208B9080E191E08E108B9DB
:100E0000F9014A9509E208B909F0F00109E208B9C7
:100E1000099406E308B9199109E208B9159F09E296
:100E200008B9080E191E08E108B9F9014A9509E246
:100E300008B909F0F00109E208B9099409E208B912
:100E4000199109E208B9159F08E108B9080E191EA1
:100E500009E208B9F9014A9509E208B909F0F00177
:100E600009E208B9099409E208B9199109E208B937
:100E7000159F08E108B9080E191E09E208B9F90121
:100E80004A9508E108B909F0F00109E208B90994A6
:100E900006E308B9199108E108B9159F09E208B9F4
:100EA000080E191E09E208B9F9014A9508E108B9C6
:100EB00009F0F00109E208B9099406E308B91991AB
:100EC00006E308B9159F09E208B9080E191E09E2E0
:100ED00008B9F9014A9509E208B909F0F00108E1F9
:100EE00008B9099406E308B9199106E308B9159FF2
:100EF00006E308B9080E191E09E208B9F9014A9576
:100F000009E208B909F0F00108E108B9099406E31B
:100F100008B9199106E308B9159F09E208B9080E46
:100F2000191E09E208B9F9014A9506E308B909F062
:100F3000F00106E308B9099406E308B9199109E23A
:100F400008B9159F09E208B9080E191E09E208B987
:100F5000F9014A9509E208B909F0F00106E308B978
:100F6000099409E208B9199108E108B9159F09E245
:100F700008B9080E191E09E208B9F9014A9509E2F3
:100F800008B909F0F00109E208B9099409E208B9C1
:100F9000199109E208B9159F08E108B9080E191E50
:100FA00008E108B9F9014A9509E208B909F0F00128
:100FB00009E208B9099409E208B9199109E208B9E6
:100FC000159F09E208B9080E191E09E208B9F901CE
:100FD0004A9508E108B909F0F00108E108B9099457
:100FE00009E208B9199108E108B9159F08E108B9A3
:100FF000080E191E09E208B9F9014A9509E208B973
:1010000009F0F00109E208B9099408E108B9199159
:1010100009E208B9159F09E208B9080E191E09E28C
:1010200008B9F9014A9509E208B909F0F00109E2A5
:1010300008B9099409E208B9199109E208B9159F9C
:1010400009E208B9080E191E09E208B9F9014A9522
:1010500009E208B909F0F00109E208B9099408E1C8
:1010600008B9199109E208B9159F09E208B9080EF3
:10107000191E06E308B9F9014A9506E308B909F013
:10108000F00106E308B9099408E108B9199109E2E9
:1010900008B9159F09E208B9080E191E09E208B936
:1010A000F9014A9506E308B909F0F00106E308B929
:1010B000099409E208B9199108E108B9159F09E2F4
:1010C00008B9080E191E09E208B9F9014A9508E1A4
:1010D00008B909F0F00106E308B9099409E208B972
:1010E000199108E108B9159F09E208B9080E191EFF
:1010F00008E108B9F9014A9509E208B909F0F001D7
:1011000009E208B9099409E208B9199109E208B994
:10111000159F09E208B9080E191E08E108B9F9017E
:101120004A9509E208B909F0F00109E208B9099401
:1011300009E208B9199109E208B9159F08E108B94F
:10114000080E191E09E208B9F9014A9509E208B921
:1011500009F0F00106E308B9099409E208B9199108
:1011600009E208B9159F08E108B9080E191E09E23D
:1011700008B9F9014A9506E308B909F0F00106E358
:1011800008B9099409E208B9199108E108B9159F4D
:1011900009E208B9080E191E06E308B9F9014A95D3
:1011A00006E308B909F0F00106E308B9099406E37B
:1011B00008B9199106E308B9159F0EE008B9080EA1
:1011C000191E0EE008B9F9014A9506E308B909F0BD
:1011D000F00106E308B9099406E308B919910EE095
:1011E00008B9159F0EE008B9080E191E0EE008B9DF
:1011F000F9014A950EE008B909F0F00106E308B9D3
:10120000099406E308B919910EE008B9159F0EE09C
:1012100008B9080E191E0EE008B9F9014A950EE04A
:1012200008B909F0F00106E308B9099403E008B928
:10123000199103E008B9159F0EE008B9080E191EB0
:101240000EE008B9F9014A950EE008B909F0F0017D
:101250000EE008B909940EE008B9199100EA08B93E
:10126000159F03E008B9080E191E0EE008B9F90130
:101270004A9500EA08B909F0F0010EE008B90994AE
:101280000EE008B919910EE008B9159F0EE008B9F3
:10129000080E191E03E008B9F9014A9503E008B9E0
:1012A00009F0F00103E008B909940EE008B91991BA
:1012B0000EE008B9159F0EE008B9080E191E0EE0E1
:1012C00008B9F9014A950EE008B909F0F0010EE0FD
:1012D00008B909940EE008B919910EE008B9159FF4
:1012E0000EE008B9080E191E0EE008B9F9014A957A
:1012F0000EE008B909F0F0010EE008B909940EE01B
:1013000008B919910EE008B9159F06E308B9080E4F
:10131000191E06E308B9F9014A9506E308B909F070
:10132000F00106E308B909940EE008B919910EE03E
:1013300008B9159F0EE008B9080E191E06E308B992
:10134000F9014A9506E308B909F0F00106E308B986
:1013500009940EE008B919910EE008B9159F00EA4A
:1013600008B9080E191E03E008B9F9014A950EE004
:1013700008B909F0F00106E308B909940EE008B9CC
:1013800019910EE008B9159F03E008B9080E191E5F
:101390000EE008B9F9014A950EE008B909F0F0012C
:1013A0000EE008B909940EE008B9199103E008B9F4
:1013B000159F0EE008B9080E191E0EE008B9F901D4
:1013C0004A950EE008B909F0F0010EE008B9099459
:1013D0000EE008B9199103E008B9159F00EA08B9B1
:1013E000080E191E0EE008B9F9014A950EE008B979
:1013F00009F0F00106E308B909940EE008B9199163
:1014000003E008B9159F0EE008B9080E191E06E39F
:1014100008B9F9014A9506E308B909F0F00106E3B5
:1014200008B9099403E008B919910EE008B9159FAD
:1014300006E308B9080E191E06E308B9F9014A9532
:1014400006E308B909F0F00106E308B909940EE0D3
:1014500008B919910EE008B9159F0EE008B9080EF9
:10146000191E0EE008B9F9014A950EE008B909F015
:10147000F0010EE008B909940EE008B919910EE0E8
:1014800008B9159F0EE008B9080E191E0EE008B93C
:10149000F9014A950EE008B909F0F0010EE008B92B
:1014A000099403E008B9199103E008B9159F03E016
:1014B00008B9080E191E0EE008B9F9014A950EE0A8
:1014C00008B909F0F0010EE008B909940EE008B976
:1014D000199100EA08B9159F0EE008B9080E191E07
:1014E00003E008B9F9014A9500EA08B909F0F001EA
:1014F0000EE008B909940EE008B919910EE008B998
:10150000159F0EE008B9080E191E0EE008B9F90182
:101510004A9503E008B909F0F00103E008B909941D
:1015200006E308B919910EE008B9159F0EE008B955
:10153000080E191E0EE008B9F9014A950EE008B927
:1015400009F0F00106E308B9099406E308B9199116
:101550000EE008B9159F0EE008B9080E191E0EE03E
:1015600008B9F9014A950EE008B909F0F00106E35F
:1015700008B9099406E308B9199106E308B9159F5B
:101580000EE008B9080E191E0EE008B9F9014A95D7
:1015900006E308B909F0F00106E308B9099406E387
:1015A00008B9199106E308B9159F06E308B9080EB2
:1015B000191E06E308B9F9014A950EE008B909F0C9
:1015C000F00103E008B9099406E308B9199106E3AC
:1015D00008B9159F06E308B9080E191E0EE008B9F0
:1015E000F9014A9503E008B909F0F0010EE008B9E5
:1015F000099406E308B919910EE008B9159F0EE0A9
:1016000008B9080E191E00EA08B9F9014A9503E065
:1016100008B909F0F0010EE008B909940EE008B924
:1016200019910EE008B9159F0EE008B9080E191EB1
:101630000EE008B9F9014A9503E008B909F0F00194
:101640000EE008B909940EE008B919910EE008B946
:10165000159F0EE008B9080E191E03E008B9F9013C
:101660004A950EE008B909F0F0010EE008B90994B6
:1016700006E308B919910EE008B9159F03E008B90F
:10168000080E191E00EA08B9F9014A950EE008B9DA
:1016900009F0F0010EE008B9099406E308B91991C0
:1016A00006E308B9159F06E308B9080E191E0EE0F7
:1016B00008B9F9014A950EE008B909F0F0010EE009
:1016C00008B9099406E308B9199106E308B9159F0A
:1016D00006E308B9080E191E06E308B9F9014A9590
:1016E0000EE008B909F0F0010EE008B909940EE027
:1016F00008B9199103E008B9159F0EE008B9080E62
:10170000191E03E008B9F9014A950EE008B909F07D
:10171000F0010EE008B9099403E008B919910EE050
:1017200008B9159F0EE008B9080E191E0EE008B999
:10173000F9014A9503E008B909F0F0010EE008B993
:10174000099403E008B919910EE008B9159F0EE05D
:1017500008B9080E191E03E008B9F9014A950EE010
:1017600008B909F0F00103E008B909940EE008B9DE
:1017700019910EE008B9159F0EE008B9080E191E60
:1017800003E008B9F9014A950EE008B909F0F00143
:101790000EE008B909940EE008B919910EE008B9F5
:1017A000159F03E008B9080E191E0EE008B9F901EB
:1017B0004A9503E008B909F0F0010EE008B9099470
:1017C0000EE008B9199103E008B9159F0EE008B9B9
:1017D000080E191E0EE008B9F9014A9503E008B990
:1017E00009F0F0010EE008B9099403E008B9199175
:1017F0000EE008B9159F0EE008B9080E191E03E0A7
:1018000008B9F9014A950EE008B909F0F0010EE0B7
:1018100008B909940EE008B9199103E008B9159FB9
:101820000EE008B9080E191E03E008B9F9014A953F
:101830000EE008B909F0F0010EE008B909940EE0D5
:1018400008B919910EE008B9159F0EE008B9080E05
:10185000191E0EE008B9F9014A950EE008B909F021
:10186000F0010EE008B909940EE008B919910EE0F4
:1018700008B9159F0EE008B9080E191E0EE008B948
:10188000F9014A950EE008B909F0F00103E008B942
:1018900009940EE008B919910EE008B9159F0EE001
:1018A00008B9080E191E03E008B9F9014A9503E0CA
:1018B00008B909F0F0010EE008B9099403E008B98D
:1018C000199103E008B9159F0EE008B9080E191E1A
:1018D0000EE008B9F9014A950EE008B909F0F001E7
:1018E0000EE008B909940EE008B919910EE008B9A4
:1018F000159F03E008B9080E191E03E008B9F901A5
:101900004A950EE008B909F0F0010EE008B9099413
:101910000EE008B919910EE008B9159F0EE008B95C
:10192000080E191E0EE008B9F9014A9503E008B93E
:1019300009F0F0010EE008B9099406E308B919911D
:101940000EE008B9159F0EE008B9080E191E0EE04A
:1019500008B9F9014A950EE008B909F0F00106E36B
:1019600008B9099406E308B9199106E308B9159F67
:101970000EE008B9080E191E0EE008B9F9014A95E3
:1019800006E308B909F0F00106E308B9099406E393
:1019900008B9199106E308B9159F06E308B9080EBE
:1019A000191E0EE008B9F9014A9503E008B909F0DB
:1019B000F0010EE008B9099406E308B9199106E3AD
:1019C00008B9159F0EE008B9080E191E03E008B902
:1019D000F9014A950EE008B909F0F0010EE008B9E6
:1019E000099406E308B919910EE008B9159F0EE0B5
:1019F00008B9080E191E03E008B9F9014A950EE06E
:101A000008B909F0F0010EE008B909940EE008B930
:101A100019910EE008B9159F03E008B9080E191EC8
:101A20000EE008B9F9014A950EE008B909F0F00195
:101A30000EE008B909940EE008B919910EE008B952
:101A4000159F03E008B9080E191E0EE008B9F90148
:101A50004A9503E008B909F0F0010EE008B90994CD
:101A600006E308B9199103E008B9159F0EE008B91B
:101A7000080E191E0EE008B9F9014A9503E008B9ED
:101A800009F0F0010EE008B9099406E308B91991CC
:101A900006E308B9159F0EE008B9080E191E0EE0FE
:101AA00008B9F9014A950EE008B909F0F00103E020
:101AB00008B9099406E308B9199106E308B9159F16
:101AC00006E308B9080E191E0EE008B9F9014A9597
:101AD0000EE008B909F0F00103E008B9099406E343
:101AE00008B9199106E308B9159F0EE008B9080E68
:101AF000191E0EE008B9F9014A9506E308B909F084
:101B0000F00106E308B9099406E308B919910EE05B
:101B100008B9159F0EE008B9080E191E0EE008B9A5
:101B2000F9014A950EE008B909F0F00106E308B999
:101B300009940EE008B9199103E008B9159F0EE069
:101B400008B9080E191E0EE008B9F9014A950EE011
:101B500008B909F0F0010EE008B909940EE008B9DF
:101B600019910EE008B9159F03E008B9080E191E77
:101B700003E008B9F9014A950EE008B909F0F0014F
:101B80000EE008B909940EE008B919910EE008B901
:101B9000159F0EE008B9080E191E0EE008B9F901EC
:101BA0004A9503E008B909F0F00103E008B9099487
:101BB0000EE008B9199103E008B9159F03E008B9D0
:101BC000080E191E0EE008B9F9014A950EE008B991
:101BD00009F0F0010EE008B9099403E008B9199181
:101BE0000EE008B9159F0EE008B9080E191E0EE0A8
:101BF00008B9F9014A950EE008B909F0F0010EE0C4
:101C000008B909940EE008B919910EE008B9159FBA
:101C10000EE008B9080E191E0EE008B9F9014A9540
:101C20000EE008B909F0F0010EE008B9099403E0EC
:101C300008B919910EE008B9159F0EE008B9080E11
:101C4000191E06E308B9F9014A9506E308B909F037
:101C5000F00106E308B9099403E008B919910EE010
:101C600008B9159F0EE008B9080E191E0EE008B954
:101C7000F9014A9506E308B909F0F00106E308B94D
:101C800009940EE008B9199103E008B9159F0EE018
:101C900008B9080E191E0EE008B9F9014A9503E0CB
:101CA00008B909F0F00106E308B909940EE008B993
:101CB000199103E008B9159F0EE008B9080E191E26
:101CC00003E008B9F9014A950EE008B909F0F001FE
:101CD0000EE008B909940EE008B919910EE008B9B0
:101CE000159F0EE008B9080E191E03E008B9F901A6
:101CF0004A950EE008B909F0F0010EE008B9099420
:101D00000EE008B919910EE008B9159F03E008B973
:101D1000080E191E0EE008B9F9014A950EE008B93F
:101D200009F0F00106E308B909940EE008B9199129
:101D30000EE008B9159F03E008B9080E191E0EE061
:101D400008B9F9014A9506E308B909F0F00106E37C
:101D500008B909940EE008B9199103E008B9159F74
:101D60000EE008B9080E191E06E308B9F9014A95F4
:101D700006E308B909F0F00106E308B9099406E39F
:101D800008B9199106E308B9159F0FEF08B9080EB5
:101D9000191E0FEF08B9F9014A9506E308B909F0D1
:101DA000F00106E308B9099406E308B919910FEFA9
:101DB00008B9159F04E008B9080E191E04E008B917
:101DC000F9014A950FEF08B909F0F00106E308B9E7
:101DD00009940FEF08B9199104E008B9159F04E0C0
:101DE00008B9080E191E04E008B9F9014A950FEF69
:101DF00008B909F0F00106E308B909940FEF08B932
:101E0000199104E008B9159F04E008B9080E191EDD
:101E100004E008B9F9014A9504E008B909F0F001B5
:101E20000FEF08B909940FEF08B9199104E008B948
:101E3000159F0FEF08B9080E191E04E008B9F90143
:101E40004A9504E008B909F0F0010FEF08B90994C8
:101E50000FEF08B9199104E008B9159F04E008B91B
:101E6000080E191E04E008B9F9014A950FEF08B9E8
:101E700009F0F00106E308B909940FEF08B91991C8
:101E800004E008B9159F04E008B9080E191E0FEF09
:101E900008B9F9014A9506E308B909F0F00106E32B
:101EA00008B9099406E308B919910FEF08B9159F0D
:101EB0000FEF08B9080E191E06E308B9F9014A9593
:101EC00006E308B909F0F00106E308B909940FE840
:101ED00008B919910FE808B9159F0FE808B9080E5D
:101EE000191E0FE808B9F9014A950FE808B909F079
:101EF000F00106E308B909940FE808B9199106E35F
:101F000008B9159F06E308B9080E191E06E308B9BB
:101F1000F9014A9506E308B909F0F0010FE808B99C
:101F200009940FE808B9199106E308B9159F06E36B
:101F300008B9080E191E06E308B9F9014A9506E327
:101F400008B909F0F0010FE808B909940FE808B9D9
:101F500019910FE808B9159F0FE808B9080E191E66
:101F60000FE808B9F9014A950FE808B909F0F0013E
:101F700006E308B909940FE808B9199106E308B90E
:101F8000159F0FE808B9080E191E06E308B9F901F4
:101F90004A9506E308B909F0F00106E308B9099487
:101FA0000FE808B9199106E308B9159F06E308B9C7
:101FB000080E191E0FE808B9F9014A9506E308B999
:101FC00009F0F00106E308B909940FE808B919917E
:101FD00006E308B9159F06E308B9080E191E06E3C3
:101FE00008B9F9014A950FE808B909F0F00106E3CC
:101FF00008B909940FE808B9199106E308B9159FC3
:1020000006E308B9080E191E06E308B9F9014A9556
:1020100006E308B909F0F0010FE808B9099408E1EE
:1020200008B919910DE108B9159F08E108B9080E22
:10203000191E0DE108B9F9014A9508E108B909F03E
:10204000F00108E108B9099408E108B919910DE116
:1020500008B9159F0DE108B9080E191E0DE108B960
:10206000F9014A950DE108B909F0F0010DE108B94F
:1020700009940DE108B919910DE108B9159F08E11E
:1020800008B9080E191E0DE108B9F9014A9508E1D1
:1020900008B909F0F00108E108B909940DE108B99F
:1020A00019910DE108B9159F08E108B9080E191E2C
:1020B0000DE108B9F9014A9508E108B909F0F00104
:1020C00008E108B9099408E108B919910DE108B9C6
:1020D000159F0DE108B9080E191E0DE108B9F901A7
:1020E0004A950DE108B909F0F00108E108B9099431
:1020F00008E108B919910DE108B9159F08E108B97F
:10210000080E191E0DE108B9F9014A9508E108B950
:1021100009F0F0010DE108B909940DE108B9199130
:102120000DE108B9159F0DE108B9080E191E0DE162
:1021300008B9F9014A950DE108B909F0F00108E183
:1021400008B9099408E108B919910DE108B9159F7A
:1021500008E108B9080E191E0DE108B9F9014A9500
:1021600008E108B909F0F00108E108B9099406E3AB
:1021700008B9199106E308B9159F06E308B9080ED6
:10218000191E06E308B9F9014A9506E308B909F0F2
:10219000F00106E308B9099406E308B9199106E3CA
:1021A00008B9159F00E508B9080E191E00E508B921
:1021B000F9014A9506E308B909F0F00106E308B908
:1021C000099406E308B9199100E508B9159F00E5DF
:1021D00008B9080E191E00E508B9F9014A9500E58D
:1021E00008B909F0F00106E308B9099400E508B957
:1021F000199100E508B9159F00E508B9080E191EE8
:1022000000E508B9F9014A9500E508B909F0F001BF
:1022100000E508B9099406E308B9199106E308B97D
:10222000159F00E508B9080E191E00E508B9F90167
:102230004A9506E308B909F0F00106E308B90994E4
:1022400006E308B9199106E308B9159F00E508B936
:10225000080E191E00E508B9F9014A9506E308B908
:1022600009F0F00106E308B9099406E308B91991E9
:1022700006E308B9159F00E508B9080E191E00E528
:1022800008B9F9014A9506E308B909F0F00106E337
:1022900008B9099406E308B9199106E308B9159F2E
:1022A00006E308B9080E191E06E308B9F9014A95B4
:1022B00006E308B909F0F00106E308B9099406E35A
:1022C00008B9199106E308B9159F06E308B9080E85
:1022D000191E06E308B9F9014A9506E308B909F0A1
:1022E000F00106E308B9099406E308B9199106E379
:1022F00008B9159F00E508B9080E191E00E508B9D0
:10230000F9014A9506E308B909F0F00106E308B9B6
:10231000099406E308B9199106E308B9159F00E589
:1023200008B9080E191E00E508B9F9014A9506E337
:1023300008B909F0F00106E308B9099406E308B901
:10234000199106E308B9159F00E508B9080E191E92
:1023500000E508B9F9014A9506E308B909F0F0016A
:1023600006E308B9099400E508B9199100E508B930
:10237000159F00E508B9080E191E00E508B9F90116
:102380004A9500E508B909F0F00100E508B909949B
:1023900006E308B9199100E508B9159F00E508B9E9
:1023A000080E191E00E508B9F9014A9500E508B9BB
:1023B00009F0F00106E308B9099406E308B9199198
:1023C00006E308B9159F00E508B9080E191E00E5D7
:1023D00008B9F9014A9506E308B909F0F00106E3E6
:1023E00008B9099406E308B9199106E308B9159FDD
:1023F00006E308B9080E191E06E308B9F9014A9563
:1024000006E308B909F0F00106E308B9099407E505
:1024100008B9199107E508B9159F07E508B9080E2D
:10242000191E07E508B9F9014A9507E508B909F049
:10243000F00107E508B9099407E508B9199107E51E
:1024400008B9159F07E508B9080E191E07E508B970
:10245000F9014A9507E508B909F0F00107E508B95F
:10246000099406E308B9199106E308B9159F07E531
:1024700008B9080E191E07E508B9F9014A9506E3DF
:1024800008B909F0F00106E308B9099406E308B9B0
:10249000199106E308B9159F07E508B9080E191E3A
:1024A00007E508B9F9014A9506E308B909F0F00112
:1024B00006E308B9099406E308B9199106E308B9D7
:1024C000159F07E508B9080E191E07E508B9F901B7
:1024D0004A9506E308B909F0F00106E308B9099442
:1024E00006E308B9199106E308B9159F07E508B98D
:1024F000080E191E07E508B9F9014A9506E308B95F
:1025000009F0F00106E308B9099407E508B9199143
:1025100007E508B9159F07E508B9080E191E07E574
:1025200008B9F9014A9507E508B909F0F00107E58E
:1025300008B9099407E508B9199107E508B9159F85
:1025400007E508B9080E191E07E508B9F9014A950B
:1025500007E508B909F0F00107E508B909940CEAA4
:1025600008B9199106E308B9159F06E308B9080EE2
:10257000191E06E308B9F9014A9506E308B909F0FE
:10258000F0010CEA08B9099406E308B919910CEABC
:1025900008B9159F06E308B9080E191E06E308B925
:1025A000F9014A9506E308B909F0F0010CEA08B907
:1025B000099406E308B919910CEA08B9159F06E3D6
:1025C00008B9080E191E06E308B9F9014A950CEA84
:1025D00008B909F0F00106E308B9099406E308B95F
:1025E000199106E308B9159F0CEA08B9080E191EDF
:1025F0000CEA08B9F9014A9506E308B909F0F001B7
:1026000006E308B9099406E308B9199106E308B985
:10261000159F0CEA08B9080E191E0CEA08B9F90151
:102620004A9506E308B909F0F00106E308B90994F0
:1026300006E308B9199106E408B9159F06E308B93D
:10264000080E191E06E308B9F9014A9506E408B90F
:1026500009F0F00106E308B9099406E408B91991F4
:1026600006E308B9159F06E408B9080E191E06E42A
:1026700008B9F9014A9506E308B909F0F00106E442
:1026800008B9099406E308B9199106E408B9159F39
:1026900006E308B9080E191E06E308B9F9014A95C0
:1026A00006E408B909F0F00106E308B909940FEF50
:1026B00008B919910FEF08B9159F0FEF08B9080E67
:1026C000191E00E008B9F9014A9500E008B909F0BF
:1026D000F0010FEF08B909940FEF08B919910FEF46
:1026E00008B9159F00E008B9080E191E01E208B9E3
:1026F000F9014A9501E208B909F0F00100E008B9D2
:1027000009940FEF08B919910FEF08B9159F00E070
:1027100008B9080E191E01E208B9F9014A9501E24B
:1027200008B909F0F00109E308B909940FEF08B9F5
:1027300019910FEF08B9159F00E008B9080E191E8E
:1027400001E208B9F9014A9509E308B909F0F00175
:1027500009E308B909940FEF08B919910FEF08B907
:10276000159F00E008B9080E191E09E308B9F90120
:102770004A9509E308B909F0F00109E308B9099499
:102780000FEF08B919910FEF08B9159F0FEF08B9AE
:10279000080E191E00E008B9F9014A9509E308B9C5
:1027A00009F0F00109E308B909940FEF08B919918C
:1027B0000FEF08B9159F0FEF08B9080E191E0FEF9C
:1027C00008B9F9014A9500E008B909F0F00100E004
:1027D00008B909940FEF08B919910FEF08B9159FBF
:1027E0000FEF08B9080E191E0FEF08B9F9014A9545
:1027F0000FEF08B909F0F0010FEF08B909940FEFD6
:1028000008B919910FEF08B9159F0FEF08B9080E15
:10281000191E0FEF08B9F9014A950FEF08B909F031
:10282000F0010FEF08B909940FEF08B919910FEFF4
:1028300008B9159F0FEF08B9080E191E0FEF08B958
:10284000F9014A950FEF08B909F0F0010FEF08B947
:10285000099400E008B919910FEF08B9159F0FEF1F
:1028600008B9080E191E0FEF08B9F9014A950FEFC4
:1028700008B909F0F0010FEF08B9099409E308B9A4
:10288000199100E008B9159F0FEF08B9080E191E3D
:102890000FEF08B9F9014A950FEF08B909F0F001F7
:1028A0000FEF08B9099409E308B9199109E308B9C8
:1028B000159F00E008B9080E191E00E008B9F901DB
:1028C0004A950FEF08B909F0F0010FEF08B9099424
:1028D00009E308B9199109E308B9159F01E208B99C
:1028E000080E191E01E208B9F9014A9500E008B97D
:1028F00009F0F0010FEF08B9099409E308B919913B
:1029000001E208B9159F01E208B9080E191E01E29B
:1029100008B9F9014A9501E208B909F0F00100E0AF
:1029200008B9099400E008B9199100E008B9159FA9
:1029300001E208B9080E191E01E208B9F9014A9529
:1029400001E208B909F0F00100E008B909940FEFBD
:1029500008B919910FEF08B9159F0FEF08B9080EC4
:10296000191E0FEF08B9F9014A950FEF08B909F0E0
:10297000F0010FEF08B909940FEF08B919910FEFA3
:1029800008B9159F0FEF08B9080E191E0FEF08B907
:10299000F9014A9500E008B909F0F00100E008B932
:1029A00009940FEF08B919910FEF08B9159F0FEFB0
:1029B00008B9080E191E00E008B9F9014A9501E2AC
:1029C00008B909F0F00101E208B909940FEF08B95C
:1029D00019910FEF08B9159F00E008B9080E191EEC
:1029E00001E208B9F9014A9501E208B909F0F001DC
:1029F00001E208B909940FEF08B9199100E008B98C
:102A0000159F01E208B9080E191E01E208B9F90183
:102A10004A9501E208B909F0F00101E208B9099408
:102A20000FEF08B9199100E008B9159F01E208B944
:102A3000080E191E01E208B9F9014A9501E208B928
:102A400009F0F00101E208B9099400E008B9199110
:102A500009E308B9159F01E208B9080E191E01E241
:102A600008B9F9014A9501E208B909F0F00101E25B
:102A700008B9099400E008B9199101E208B9159F55
:102A800001E208B9080E191E01E208B9F9014A95D8
:102A900001E208B909F0F00101E208B9099400E087
:102AA00008B9199100E008B9159F0FEF08B9080E91
:102AB000191E0FEF08B9F9014A950FEF08B909F08F
:102AC000F0010FEF08B9099409E308B9199109E376
:102AD00008B9159F00E008B9080E191E00E008B9F2
:102AE000F9014A950FEF08B909F0F0010FEF08B9A5
:102AF000099409E308B9199109E308B9159F09E395
:102B000008B9080E191E09E308B9F9014A9500E051
:102B100008B909F0F0010FEF08B9099409E308B901
:102B2000199109E308B9159F09E308B9080E191EA0
:102B300009E308B9F9014A9509E308B909F0F00178
:102B400000E008B9099409E308B9199109E308B943
:102B5000159F09E308B9080E191E09E308B9F90120
:102B60004A9509E308B909F0F00101E208B90994AE
:102B700009E308B9199109E308B9159F09E308B9F0
:102B8000080E191E09E308B9F9014A9501E208B9CE
:102B900009F0F00101E208B9099409E308B91991B3
:102BA00009E308B9159F09E308B9080E191E01E2E7
:102BB00008B9F9014A9501E208B909F0F00101E20A
:102BC00008B9099409E308B9199109E308B9159FEF
:102BD00001E208B9080E191E01E208B9F9014A9587
:102BE00001E208B909F0F00101E208B909940FEF18
:102BF00008B919910FEF08B9159F0FEF08B9080E22
:102C0000191E0FEF08B9F9014A950FEF08B909F03D
:102C1000F0010FEF08B909940FEF08B919910FEF00
:102C200008B9159F0FEF08B9080E191E0FEF08B964
:102C3000F9014A950FEF08B909F0F0010FEF08B953
:102C400009940FEF08B919910FEF08B9159F0FEF0D
:102C500008B9080E191E0FEF08B9F9014A950FEFD0
:102C600008B909F0F0010FEF08B909940FEF08B99E
:102C700019910FEF08B9159F0FEF08B9080E191E2B
:102C80000FEF08B9F9014A950FEF08B909F0F00103
:102C90000FEF08B9099400E008B919910FEF08B9CE
:102CA000159F0FEF08B9080E191E0FEF08B9F901AB
:102CB0004A950FEF08B909F0F0010FEF08B9099430
:102CC00001E208B9199100E008B9159F0FEF08B9A2
:102CD000080E191E0FEF08B9F9014A950FEF08B950
:102CE00009F0F0010FEF08B9099401E208B9199150
:102CF00001E208B9159F00E008B9080E191E00E0AE
:102D000008B9F9014A950FEF08B909F0F0010FEF82
:102D100008B9099401E208B9199101E208B9159FAF
:102D200001E208B9080E191E09E308B9F9014A952C
:102D300000E008B909F0F00100E008B909940FEFCC
:102D400008B919910FEF08B9159F0FEF08B9080ED0
:102D5000191E0FEF08B9F9014A950FEF08B909F0EC
:102D6000F0010FEF08B909940FEF08B919910FEFAF
:102D700008B9159F0FEF08B9080E191E0FEF08B913
:102D8000F9014A950FEF08B909F0F0010FEF08B902
:102D900009940FEF08B919910FEF08B9159F0FEFBC
:102DA00008B9080E191E0FEF08B9F9014A950FEF7F
:102DB00008B909F0F0010FEF08B909940FEF08B94D
:102DC00019910FEF08B9159F0FEF08B9080E191EDA
:102DD0000FEF08B9F9014A950FEF08B909F0F001B2
:102DE0000FEF08B909940FEF08B919910FEF08B95F
:102DF000159F0FEF08B9080E191E0FEF08B9F9015A
:102E00004A950FEF08B909F0F0010FEF08B90994DE
:102E10000FEF08B919910FEF08B9159F0FEF08B917
:102E2000080E191E0FEF08B9F9014A9500E008B91C
:102E300009F0F00100E008B909940FEF08B9199101
:102E40000FEF08B9159F00E008B9080E191E00E041
:102E500008B9F9014A9509E308B909F0F00109E355
:102E600008B9099400E008B9199100E008B9159F64
:102E700009E308B9080E191E09E308B9F9014A95D2
:102E800009E308B909F0F00101E208B909940FEF6C
:102E900008B919910FEF08B9159F0FEF08B9080E7F
:102EA000191E0FEF08B9F9014A9500E008B909F0B9
:102EB000F00100E008B909940FEF08B919910FEF7C
:102EC00008B9159F0FEF08B9080E191E00E008B9E0
:102ED000F9014A9509E308B909F0F00109E308B9D5
:102EE00009940FEF08B919910FEF08B9159F00E089
:102EF00008B9080E191E01E208B9F9014A9509E35B
:102F000008B909F0F00109E308B909940FEF08B90D
:102F1000199100E008B9159F01E208B9080E191EC1
:102F200001E208B9F9014A9509E308B909F0F0018D
:102F300009E308B9099400E008B9199101E208B958
:102F4000159F01E208B9080E191E01E208B9F9013E
:102F50004A9509E308B909F0F00109E308B90994B1
:102F600001E208B9199101E208B9159F01E208B917
:102F7000080E191E01E208B9F9014A9509E308B9DA
:102F800009F0F00109E308B9099401E208B91991BF
:102F900001E208B9159F01E208B9080E191E01E205
:102FA00008B9F9014A9509E308B909F0F00109E304
:102FB00008B9099401E208B9199101E208B9159F0D
:102FC00001E208B9080E191E09E308B9F9014A958A
:102FD00009E308B909F0F00109E308B9099400E030
:102FE00008B919910FEF08B9159F0FEF08B9080E2E
:102FF000191E0FEF08B9F9014A950FEF08B909F04A
:10300000F0010FEF08B9099409E308B9199100E03C
:1030100008B9159F0FEF08B9080E191E0FEF08B970
:10302000F9014A950FEF08B909F0F0010FEF08B95F
:10303000099409E308B9199109E308B9159F00E05B
:1030400008B9080E191E0FEF08B9F9014A950FEFDC
:1030500008B909F0F0010FEF08B9099409E308B9BC
:10306000199109E308B9159F09E308B9080E191E5B
:1030700000E008B9F9014A950FEF08B909F0F0012D
:1030800000E008B9099409E308B9199109E308B9FE
:10309000159F09E308B9080E191E09E308B9F901DB
:1030A0004A9500E008B909F0F00101E208B9099475
:1030B00009E308B9199109E308B9159F09E308B9AB
:1030C000080E191E09E308B9F9014A9509E308B980
:1030D00009F0F00101E208B9099409E308B919916E
:1030E00009E308B9159F09E308B9080E191E09E399
:1030F00008B9F9014A9501E208B909F0F00101E2C5
:1031000008B9099409E308B9199109E308B9159FA9
:1031100009E308B9080E191E01E208B9F9014A9538
:1031200001E208B909F0F00101E208B909940FEFD2
:1031300008B919910FEF08B9159F0FEF08B9080EDC
:10314000191E0FEF08B9F9014A950FEF08B909F0F8
:10315000F0010FEF08B909940FEF08B919910FEFBB
:1031600008B9159F0FEF08B9080E191E0FEF08B91F
:10317000F9014A950FEF08B909F0F0010FEF08B90E
:1031800009940FEF08B919910FEF08B9159F00E0E6
:1031900008B9080E191E00E008B9F9014A9500E0C7
:1031A00008B909F0F00100E008B9099400E008B995
:1031B000199100E008B9159F01E208B9080E191E1F
:1031C00001E208B9F9014A9501E208B909F0F001F4
:1031D00009E308B9099401E208B9199101E208B9B3
:1031E000159F01E208B9080E191E01E208B9F9019C
:1031F0004A9501E208B909F0F00109E308B9099418
:1032000001E208B9199101E208B9159F01E208B974
:10321000080E191E01E208B9F9014A9509E308B937
:1032200009F0F00109E308B9099401E208B919911C
:1032300001E208B9159F01E208B9080E191E01E262
:1032400008B9F9014A9509E308B909F0F00109E361
:1032500008B9099401E208B9199101E208B9159F6A
:1032600001E208B9080E191E09E308B9F9014A95E7
:1032700009E308B909F0F00109E308B909940FEF6F
:1032800008B919910FEF08B9159F0FEF08B9080E8B
:10329000191E0FEF08B9F9014A950FEF08B909F0A7
:1032A000F0010FEF08B909940FEF08B919910FEF6A
:1032B00008B9159F0FEF08B9080E191E0FEF08B9CE
:1032C000F9014A950FEF08B909F0F0010FEF08B9BD
:1032D000099400E008B9199100E008B9159F00E0D1
:1032E00008B9080E191E00E008B9F9014A9500E076
:1032F00008B909F0F00100E008B9099409E308B938
:10330000199109E308B9159F09E308B9080E191EB8
:1033100009E308B9F9014A9509E308B909F0F00190
:1033200009E308B9099409E308B9199109E308B94F
:10333000159F09E308B9080E191E09E308B9F90138
:103340004A9509E308B909F0F00109E308B90994BD
:1033500009E308B9199109E308B9159F09E308B908
:10336000080E191E09E308B9F9014A9509E308B9DD
:1033700009F0F00109E308B9099409E308B91991C2
:1033800009E308B9159F09E308B9080E191E09E3F6
:1033900008B9F9014A9509E308B909F0F00109E310
:1033A00008B9099409E308B9199109E308B9159F07
:1033B00009E308B9080E191E09E308B9F9014A958D
:1033C00009E308B909F0F00109E308B909940FEF1E
:1033D00008B919910FEF08B9159F0FEF08B9080E3A
:1033E000191E0FEF08B9F9014A950FEF08B909F056
:1033F000F0010FEF08B909940FEF08B919910FEF19
:1034000008B9159F0FEF08B9080E191E0FEF08B97C
:10341000F9014A950FEF08B909F0F0010FEF08B96B
:1034200009940FEF08B919910FEF08B9159F0FEF25
:1034300008B9080E191E0FEF08B9F9014A950FEFE8
:1034400008B909F0F0010FEF08B9099400E008B9D4
:1034500019910FEF08B9159F0FEF08B9080E191E43
:103460000FEF08B9F9014A950FEF08B909F0F0011B
:103470000FEF08B9099409E308B9199100E008B9F8
:10348000159F0FEF08B9080E191E0FEF08B9F901C3
:103490004A950FEF08B909F0F0010FEF08B9099448
:1034A00009E308B9199109E308B9159F00E008B9C3
:1034B000080E191E0FEF08B9F9014A950FEF08B968
:1034C00009F0F0010FEF08B9099409E308B919915F
:1034D00009E308B9159F09E308B9080E191E00E0B1
:1034E00008B9F9014A950FEF08B909F0F0010FEF9B
:1034F00008B9099401E208B9199101E208B9159FC8
:1035000001E208B9080E191E01E208B9F9014A954D
:1035100000E008B909F0F0010FEF08B909940FEFC6
:1035200008B919910FEF08B9159F00E008B9080E06
:10353000191E00E008B9F9014A9500E008B909F040
:10354000F00100E008B909940FEF08B9199100E003
:1035500008B9159F01E208B9080E191E01E208B961
:10356000F9014A9501E208B909F0F00101E208B950
:10357000099400E008B9199101E208B9159F01E228
:1035800008B9080E191E01E208B9F9014A9501E2CD
:1035900008B909F0F00101E208B9099400E008B99E
:1035A000199101E208B9159F01E208B9080E191E28
:1035B00001E208B9F9014A9501E208B909F0F00100
:1035C00001E208B9099400E008B9199101E208B9CB
:1035D000159F01E208B9080E191E01E208B9F901A8
:1035E0004A9501E208B909F0F00101E208B909942D
:1035F00000E008B9199101E208B9159F01E208B984
:10360000080E191E01E208B9F9014A9501E208B94C
:1036100009F0F00109E308B9099400E008B919912B
:1036200001E208B9159F01E208B9080E191E01E26E
:1036300008B9F9014A9501E208B909F0F00109E376
:1036400008B9099400E008B9199101E208B9159F79
:1036500001E208B9080E191E01E208B9F9014A95FC
:1036600009E308B909F0F00109E308B9099400E099
:1036700008B9199100E008B9159F00E008B9080ED3
:10368000191E00E008B9F9014A9500E008B909F0EF
:10369000F00100E008B9099401E208B9199109E3C1
:1036A00008B9159F09E308B9080E191E09E308B9FE
:1036B000F9014A9509E308B909F0F00109E308B9ED
:1036C000099401E208B9199109E308B9159F09E3C2
:1036D00008B9080E191E09E308B9F9014A9509E36A
:1036E00008B909F0F00109E308B9099409E308B938
:1036F000199109E308B9159F09E308B9080E191EC5
:1037000009E308B9F9014A9509E308B909F0F0019C
:1037100009E308B9099409E308B9199109E308B95B
:10372000159F09E308B9080E191E09E308B9F90144
:103730004A9509E308B909F0F00100E008B90994D5
:1037400009E308B9199109E308B9159F09E308B914
:10375000080E191E09E308B9F9014A9509E308B9E9
:1037600009F0F00100E008B9099409E308B91991DA
:1037700009E308B9159F09E308B9080E191E09E302
:1037800008B9F9014A9509E308B909F0F00109E31C
:1037900008B9099409E308B9199109E308B9159F13
:1037A00009E308B9080E191E09E308B9F9014A9599
:1037B00009E308B909F0F00109E308B9099400E048
:1037C00008B9199100E008B9159F0FEF08B9080E64
:1037D000191E0FEF08B9F9014A950FEF08B909F062
:1037E000F0010FEF08B9099409E308B9199109E349
:1037F00008B9159F00E008B9080E191E0FEF08B9A7
:10380000F9014A950FEF08B909F0F0010FEF08B977
:10381000099409E308B9199109E308B9159F09E367
:1038200008B9080E191E00E008B9F9014A950FEF12
:1038300008B909F0F0010FEF08B9099400E008B9E0
:10384000199100E008B9159F09E308B9080E191E7F
:1038500009E308B9F9014A9500E008B909F0F00157
:103860000FEF08B909940FEF08B9199105E008B9ED
:10387000159F00E008B9080E191E09E308B9F901FF
:103880004A9509E308B909F0F00100E008B9099484
:103890000FEF08B9199105E008B9159F00E008B9C4
:1038A000080E191E09E308B9F9014A9509E308B998
:1038B00009F0F00100E008B9099400E008B9199195
:1038C00000E008B9159F09E308B9080E191E09E3BD
:1038D00008B9F9014A9509E308B909F0F00109E3CB
:1038E00008B9099409E308B9199109E308B9159FC2
:1038F00000E008B9080E191E09E308B9F9014A9554
:1039000009E308B909F0F00109E308B909940FEFD8
:1039100008B919910FEF08B9159F0FEF08B9080EF4
:10392000191E0FEF08B9F9014A950FEF08B909F010
:10393000F0010FEF08B909940FEF08B919910FEFD3
:1039400008B9159F0FEF08B9080E191E0FEF08B937
:10395000F9014A950FEF08B909F0F0010FEF08B926
:1039600009940FEF08B919910FEF08B9159F0FEFE0
:1039700008B9080E191E0FEF08B9F9014A950FEFA3
:1039800008B909F0F0010FEF08B909940FEF08B971
:1039900019910FEF08B9159F0FEF08B9080E191EFE
:1039A0000FEF08B9F9014A950FEF08B909F0F001D6
:1039B0000FEF08B909940FEF08B919910FEF08B983
:1039C000159F0FEF08B9080E191E0FEF08B9F9017E
:1039D0004A950FEF08B909F0F0010FEF08B9099403
:1039E0000FEF08B919910FEF08B9159F0FEF08B93C
:1039F000080E191E0FEF08B9F9014A950FEF08B923
:103A000009F0F0010FEF08B9099400E008B9199125
:103A10000FEF08B9159F0FEF08B9080E191E0FEF29
:103A200008B9F9014A950FEF08B909F0F0010FEF55
:103A300008B9099409E308B9199100E008B9159F7C
:103A40000FEF08B9080E191E0FEF08B9F9014A95D2
:103A50000FEF08B909F0F0010FEF08B909940FEF63
:103A600008B919910FEF08B9159F00E008B9080EC1
:103A7000191E01E208B9F9014A9501E208B909F0F5
:103A8000F00101E208B909940FEF08B919910FEF9D
:103A900008B9159F0FEF08B9080E191E00E008B904
:103AA000F9014A9501E208B909F0F00101E208B90B
:103AB00009940FEF08B919910FEF08B9159F0FEF8F
:103AC00008B9080E191E0FEF08B9F9014A9500E070
:103AD00008B909F0F00101E208B909940FEF08B93B
:103AE00019910FEF08B9159F0FEF08B9080E191EAD
:103AF0000FEF08B9F9014A9500E008B909F0F001A3
:103B000009E308B909940FEF08B919910FEF08B943
:103B1000159F0FEF08B9080E191E0FEF08B9F9012C
:103B20004A950FEF08B909F0F00100E008B90994CF
:103B30000FEF08B919910FEF08B9159F0FEF08B9EA
:103B4000080E191E0FEF08B9F9014A950FEF08B9D1
:103B500009F0F0010FEF08B909940FEF08B91991B6
:103B60000FEF08B9159F0FEF08B9080E191E0FEFD8
:103B700008B9F9014A950FEF08B909F0F0010FEF04
:103B800008B909940FEF08B919910FEF08B9159FFB
:103B90000FEF08B9080E191E0FEF08B9F9014A9581
:103BA0000FEF08B909F0F0010FEF08B9099400E030
:103BB00008B9199100E008B9159F00E008B9080E8E
:103BC000191E00E008B9F9014A9500E008B909F0AA
:103BD000F00100E008B9099401E208B9199109E37C
:103BE00008B9159F09E308B9080E191E09E308B9B9
:103BF000F9014A9509E308B909F0F00101E208B9B1
:103C0000099409E308B9199109E308B9159F09E373
:103C100008B9080E191E09E308B9F9014A9501E22D
:103C200008B909F0F00101E208B9099409E308B9FB
:103C3000199109E308B9159F09E308B9080E191E7F
:103C400001E208B9F9014A9501E208B909F0F00169
:103C500001E208B9099400E008B9199100E008B937
:103C6000159F00E008B9080E191E00E008B9F90117
:103C70004A9500E008B909F0F00101E208B9099499
:103C80000FEF08B919910FEF08B9159F0FEF08B999
:103C9000080E191E0FEF08B9F9014A950FEF08B980
:103CA00009F0F00100E008B909940FEF08B9199183
:103CB0000FEF08B9159F0FEF08B9080E191E0FEF87
:103CC00008B9F9014A950FEF08B909F0F0010FEFB3
:103CD00008B909940FEF08B919910FEF08B9159FAA
:103CE0000FEF08B9080E191E0FEF08B9F9014A9530
:103CF0000FEF08B909F0F0010FEF08B9099401E2DC
:103D000008B9199101E208B9159F01E208B9080E36
:103D1000191E01E208B9F9014A9501E208B909F052
:103D2000F00109E308B9099401E208B9199101E227
:103D300008B9159F01E208B9080E191E01E208B979
:103D4000F9014A9509E308B909F0F00109E308B956
:103D5000099401E208B9199101E208B9159F01E23D
:103D600008B9080E191E09E308B9F9014A9509E3D3
:103D700008B909F0F00100E008B9099401E208B9B6
:103D8000199101E208B9159F01E208B9080E191E40
:103D900009E308B9F9014A9500E008B909F0F00112
:103DA0000FEF08B9099401E208B9199101E208B9C5
:103DB000159F00E008B9080E191E00E008B9F901C6
:103DC0004A950FEF08B909F0F0010FEF08B909940F
:103DD00000E008B9199100E008B9159F0FEF08B984
:103DE000080E191E0FEF08B9F9014A950FEF08B92F
:103DF00009F0F0010FEF08B909940FEF08B9199114
:103E00000FEF08B9159F0FEF08B9080E191E0FEF35
:103E100008B9F9014A950FEF08B909F0F0010FEF61
:103E200008B909940FEF08B919910FEF08B9159F58
:103E30000FEF08B9080E191E0FEF08B9F9014A95DE
:103E40000FEF08B909F0F0010FEF08B9099409E381
:103E500008B9199101E208B9159F01E208B9080EE5
:103E6000191E01E208B9F9014A9501E208B909F001
:103E7000F00101E208B9099400E008B9199100E0E5
:103E800008B9159F01E208B9080E191E01E208B928
:103E9000F9014A9501E208B909F0F00101E208B917
:103EA00009940FEF08B919910FEF08B9159F00E0B9
:103EB00008B9080E191E00E008B9F9014A9501E297
:103EC00008B909F0F00101E208B909940FEF08B947
:103ED00019910FEF08B9159F0FEF08B9080E191EB9
:103EE0000FEF08B9F9014A9500E008B909F0F001AF
:103EF00000E008B909940FEF08B919910FEF08B95C
:103F0000159F0FEF08B9080E191E0FEF08B9F90138
:103F10004A950FEF08B909F0F0010FEF08B90994BD
:103F20000FEF08B919910FEF08B9159F0FEF08B9F6
:103F3000080E191E0FEF08B9F9014A950FEF08B9DD
:103F400009F0F0010FEF08B909940FEF08B91991C2
:103F50000FEF08B9159F0FEF08B9080E191E0FEFE4
:103F600008B9F9014A950FEF08B909F0F0010FEF10
:103F700008B909940FEF08B919910FEF08B9159F07
:103F80000FEF08B9080E191E0FEF08B9F9014A958D
:103F90000FEF08B909F0F0010FEF08B9099401E239
:103FA00008B9199101E208B9159F01E208B9080E94
:103FB000191E09E308B9F9014A9509E308B909F09E
:103FC000F00109E308B9099401E208B9199109E37C
:103FD00008B9159F09E308B9080E191E09E308B9C5
:103FE000F9014A9509E308B909F0F00109E308B9B4
:103FF000099409E308B9199109E308B9159F09E380
:1040000008B9080E191E09E308B9F9014A9501E239
:1040100008B909F0F00101E208B9099409E308B907
:10402000199109E308B9159F09E308B9080E191E8B
:1040300001E208B9F9014A9501E208B909F0F00175
:1040400001E208B9099400E008B9199100E008B943
:10405000159F01E208B9080E191E01E208B9F9011D
:104060004A9501E208B909F0F00101E208B90994A2
:104070000FEF08B919910FEF08B9159F00E008B9C3
:10408000080E191E00E008B9F9014A9500E008B9C8
:1040900009F0F00100E008B909940FEF08B919918F
:1040A0000FEF08B9159F0FEF08B9080E191E0FEF93
:1040B00008B9F9014A950FEF08B909F0F0010FEFBF
:1040C00008B909940FEF08B919910FEF08B9159FB6
:1040D0000FEF08B9080E191E0FEF08B9F9014A953C
:1040E0000FEF08B909F0F0010FEF08B9099400E0EB
:1040F00008B9199100E008B9159F00E008B9080E49
:10410000191E00E008B9F9014A9500E008B909F064
:10411000F00100E008B9099401E208B9199101E23F
:1041200008B9159F01E208B9080E191E01E208B985
:10413000F9014A9501E208B909F0F00101E208B974
:10414000099401E208B9199101E208B9159F01E249
:1041500008B9080E191E01E208B9F9014A9501E2F1
:1041600008B909F0F00109E308B9099401E208B9B6
:10417000199101E208B9159F01E208B9080E191E4C
:1041800001E208B9F9014A9509E308B909F0F0011B
:1041900009E308B9099401E208B9199101E208B9E3
:1041A000159F01E208B9080E191E09E308B9F901C3
:1041B0004A9509E308B909F0F00109E308B909943F
:1041C00000E008B9199100E008B9159F00E008B9AE
:1041D000080E191E00E008B9F9014A9500E008B977
:1041E00009F0F00100E008B909940FEF08B919913E
:1041F0000FEF08B9159F0FEF08B9080E191E0FEF42
:1042000008B9F9014A950FEF08B909F0F0010FEF6D
:1042100008B909940FEF08B919910FEF08B9159F64
:104220000FEF08B9080E191E0FEF08B9F9014A95EA
:104230000FEF08B909F0F0010FEF08B9099409E38D
:1042400008B9199109E308B9159F09E308B9080EDF
:10425000191E09E308B9F9014A9501E208B909F004
:10426000F00101E208B9099409E308B9199109E3D9
:1042700008B9159F09E308B9080E191E09E308B922
:10428000F9014A9501E208B909F0F00101E208B923
:10429000099409E308B9199109E308B9159F09E3DD
:1042A00008B9080E191E01E208B9F9014A9501E2A0
:1042B00008B909F0F00101E208B9099409E308B965
:1042C000199109E308B9159F09E308B9080E191EE9
:1042D00001E208B9F9014A9501E208B909F0F001D3
:1042E00001E208B9099409E308B9199109E308B989
:1042F000159F09E308B9080E191E00E008B9F90175
:104300004A9500E008B909F0F00100E008B9099405
:1043100000E008B9199100E008B9159F00E008B95C
:10432000080E191E0FEF08B9F9014A950FEF08B9E9
:1043300009F0F0010FEF08B909940FEF08B91991CE
:104340000FEF08B9159F0FEF08B9080E191E0FEFF0
:1043500008B9F9014A950FEF08B909F0F0010FEF1C
:1043600008B909940FEF08B919910FEF08B9159F13
:104370000FEF08B9080E191E0FEF08B9F9014A9599
:104380000FEF08B909F0F0010FEF08B9099401E245
:1043900008B9199101E208B9159F01E208B9080EA0
:1043A000191E09E308B9F9014A9500E008B909F0B6
:1043B000F00100E008B9099401E208B9199101E29D
:1043C00008B9159F01E208B9080E191E00E008B9E6
:1043D000F9014A950FEF08B909F0F0010FEF08B99C
:1043E000099401E208B9199100E008B9159F00E0AD
:1043F00008B9080E191E0FEF08B9F9014A950FEF19
:1044000008B909F0F0010FEF08B9099400E008B904
:1044100019910FEF08B9159F0FEF08B9080E191E73
:104420000FEF08B9F9014A950FEF08B909F0F0014B
:104430000FEF08B909940FEF08B919910FEF08B9F8
:10444000159F0FEF08B9080E191E0FEF08B9F901F3
:104450004A950FEF08B909F0F0010FEF08B9099478
:104460000FEF08B919910FEF08B9159F0FEF08B9B1
:10447000080E191E0FEF08B9F9014A950FEF08B998
:1044800009F0F0010FEF08B909940FEF08B919917D
:104490000FEF08B9159F0FEF08B9080E191E0FEF9F
:1044A00008B9F9014A950FEF08B909F0F0010FEFCB
:1044B00008B909940FEF08B919910FEF08B9159FC2
:1044C0000FEF08B9080E191E0FEF08B9F9014A9548
:1044D0000FEF08B909F0F0010FEF08B9099400E0F7
:1044E00008B9199109E308B9159F01E208B9080E46
:1044F000191E01E208B9F9014A9501E208B909F06B
:10450000F00101E208B909940FEF08B9199100E030
:1045100008B9159F01E208B9080E191E01E208B991
:10452000F9014A9501E208B909F0F00101E208B980
:1045300009940FEF08B9199100E008B9159F01E23D
:1045400008B9080E191E01E208B9F9014A9501E2FD
:1045500008B909F0F00101E208B909940FEF08B9B0
:1045600019910FEF08B9159F00E008B9080E191E40
:1045700001E208B9F9014A9501E208B909F0F00130
:1045800001E208B909940FEF08B919910FEF08B9C2
:10459000159F0FEF08B9080E191E00E008B9F901C0
:1045A0004A9500E008B909F0F00100E008B9099463
:1045B0000FEF08B919910FEF08B9159F0FEF08B960
:1045C000080E191E0FEF08B9F9014A950FEF08B947
:1045D00009F0F0010FEF08B909940FEF08B919912C
:1045E0000FEF08B9159F0FEF08B9080E191E0FEF4E
:1045F00008B9F9014A950FEF08B909F0F0010FEF7A
:1046000008B909940FEF08B919910FEF08B9159F70
:104610000FEF08B9080E191E0FEF08B9F9014A95F6
:104620000FEF08B909F0F0010FEF08B9099401E2A2
:1046300008B9199101E208B9159F01E208B9080EFD
:10464000191E09E308B9F9014A9509E308B909F007
:10465000F00109E308B9099401E208B9199101E2EE
:1046600008B9159F09E308B9080E191E09E308B92E
:10467000F9014A9509E308B909F0F00109E308B91D
:10468000099401E208B9199101E208B9159F09E3FB
:1046900008B9080E191E09E308B9F9014A9509E39A
:1046A00008B909F0F00109E308B9099400E008B974
:1046B000199100E008B9159F00E008B9080E191E0D
:1046C00000E008B9F9014A9500E008B909F0F001E5
:1046D00000E008B909940FEF08B919910FEF08B974
:1046E000159F0FEF08B9080E191E0FEF08B9F90151
:1046F0004A950FEF08B909F0F0010FEF08B90994D6
:104700000FEF08B919910FEF08B9159F0FEF08B90E
:10471000080E191E0FEF08B9F9014A950FEF08B9F5
:1047200009F0F0010FEF08B909940FEF08B91991DA
:104730000FEF08B9159F0FEF08B9080E191E0FEFFC
:1047400008B9F9014A950FEF08B909F0F0010FEF28
:1047500008B909940FEF08B919910FEF08B9159F1F
:104760000FEF08B9080E191E0FEF08B9F9014A95A5
:104770000FEF08B909F0F0010FEF08B9099409E348
:1047800008B9199109E308B9159F09E308B9080E9A
:10479000191E01E208B9F9014A9501E208B909F0C8
:1047A000F00101E208B9099409E308B9199101E29D
:1047B00008B9159F01E208B9080E191E01E208B9EF
:1047C000F9014A9501E208B909F0F00101E208B9DE
:1047D000099401E208B9199101E208B9159F01E2B3
:1047E00008B9080E191E01E208B9F9014A9501E25B
:1047F00008B909F0F00101E208B9099400E008B92C
:10480000199100E008B9159F00E008B9080E191EBB
:1048100001E208B9F9014A9501E208B909F0F0018D
:1048200001E208B909940FEF08B919910FEF08B91F
:10483000159F0FEF08B9080E191E00E008B9F9011D
:104840004A9501E208B909F0F00101E208B90994BA
:104850000FEF08B919910FEF08B9159F0FEF08B9BD
:10486000080E191E0FEF08B9F9014A9500E008B9C2
:1048700009F0F00101E208B909940FEF08B91991A4
:104880000FEF08B9159F0FEF08B9080E191E0FEFAB
:1048900008B9F9014A950FEF08B909F0F00100E0F5
:1048A00008B909940FEF08B919910FEF08B9159FCE
:1048B0000FEF08B9080E191E0FEF08B9F9014A9554
:1048C0000FEF08B909F0F0010FEF08B9099401E200
:1048D00008B9199101E208B9159F01E208B9080E5B
:1048E000191E01E208B9F9014A9501E208B909F077
:1048F000F00100E008B9099401E208B9199101E258
:1049000008B9159F01E208B9080E191E01E208B99D
:10491000F9014A9501E208B909F0F00101E208B98C
:10492000099401E208B9199101E208B9159F01E261
:1049300008B9080E191E01E208B9F9014A9509E300
:1049400008B909F0F00109E308B9099401E208B9CE
:10495000199101E208B9159F01E208B9080E191E64
:1049600009E308B9F9014A9509E308B909F0F0012A
:1049700009E308B9099401E208B9199101E208B9FB
:10498000159F09E308B9080E191E09E308B9F901D2
:104990004A9509E308B909F0F00109E308B9099457
:1049A00009E308B9199109E308B9159F09E308B9A2
:1049B000080E191E09E308B9F9014A9509E308B977
:1049C00009F0F00109E308B9099409E308B919915C
:1049D00009E308B9159F09E308B9080E191E09E390
:1049E00008B9F9014A9509E308B909F0F00109E3AA
:1049F00008B9099400E008B9199100E008B9159FB9
:104A000000E008B9080E191E00E008B9F9014A953E
:104A100000E008B909F0F00100E008B909940FEFCF
:104A200008B919910FEF08B9159F0FEF08B9080ED3
:104A3000191E0FEF08B9F9014A950FEF08B909F0EF
:104A4000F0010FEF08B9099400E008B9199100E0EE
:104A500008B9159F00E008B9080E191E00E008B952
:104A6000F9014A9500E008B909F0F00100E008B941
:104A7000099409E308B9199109E308B9159F09E3F5
:104A800008B9080E191E09E308B9F9014A9509E3A6
:104A900008B909F0F00109E308B9099409E308B974
:104AA000199109E308B9159F09E308B9080E191E01
:104AB00009E308B9F9014A9509E308B909F0F001D9
:104AC00009E308B9099409E308B9199109E308B998
:104AD000159F09E308B9080E191E09E308B9F90181
:104AE0004A9509E308B909F0F00109E308B9099406
:104AF00009E308B9199109E308B9159F09E308B951
:104B0000080E191E09E308B9F9014A9509E308B925
:104B100009F0F00101E208B9099409E308B9199113
:104B200009E308B9159F09E308B9080E191E09E33E
:104B300008B9F9014A9509E308B909F0F00101E261
:104B400008B9099400E008B9199100E008B9159F67
:104B500000E008B9080E191E00E008B9F9014A95ED
:104B600000E008B909F0F00100E008B909940FEF7E
:104B700008B9199100E008B9159F00E008B9080EBE
:104B8000191E00E008B9F9014A9500E008B909F0DA
:104B9000F00100E008B9099400E008B9199109E3AF
:104BA00008B9159F01E208B9080E191E01E208B9FB
:104BB000F9014A9501E208B909F0F00101E208B9EA
:104BC000099409E308B9199101E208B9159F01E2B6
:104BD00008B9080E191E01E208B9F9014A9501E267
:104BE00008B909F0F00101E208B9099409E308B92C
:104BF000199101E208B9159F01E208B9080E191EC2
:104C000001E208B9F9014A9501E208B909F0F00199
:104C100001E208B9099401E208B9199101E208B961
:104C2000159F01E208B9080E191E01E208B9F90141
:104C30004A9501E208B909F0F00101E208B90994C6
:104C400001E208B9199101E208B9159F01E208B91A
:104C5000080E191E01E208B9F9014A9501E208B9E6
:104C600009F0F00109E308B9099401E208B91991C2
:104C700001E208B9159F01E208B9080E191E01E208
:104C800008B9F9014A9509E308B909F0F00100E013
:104C900008B9099400E008B9199100E008B9159F16
:104CA00000E008B9080E191E00E008B9F9014A959C
:104CB00000E008B909F0F0010FEF08B9099401E22A
:104CC00008B9199101E208B9159F01E208B9080E67
:104CD000191E01E208B9F9014A9509E308B909F07A
:104CE000F00109E308B9099401E208B9199101E258
:104CF00008B9159F01E208B9080E191E09E308B9A1
:104D0000F9014A9509E308B909F0F00100E008B992
:104D1000099401E208B9199101E208B9159F09E364
:104D200008B9080E191E00E008B9F9014A9500E01B
:104D300008B909F0F0010FEF08B9099401E208B9C8
:104D4000199109E308B9159F00E008B9080E191E6A
:104D50000FEF08B9F9014A950FEF08B909F0F00112
:104D60000FEF08B9099409E308B9199100E008B9EF
:104D7000159F0FEF08B9080E191E0FEF08B9F901BA
:104D80004A950FEF08B909F0F0010FEF08B909943F
:104D900000E008B919910FEF08B9159F0FEF08B996
:104DA000080E191E0FEF08B9F9014A950FEF08B95F
:104DB00009F0F0010FEF08B909940FEF08B9199144
:104DC0000FEF08B9159F0FEF08B9080E191E0FEF66
:104DD00008B9F9014A950FEF08B909F0F0010FEF92
:104DE00008B909940FEF08B919910FEF08B9159F89
:104DF0000FEF08B9080E191E0FEF08B9F9014A950F
:104E00000FEF08B909F0F0010FEF08B9099409E3B1
:104E100008B9199109E308B9159F09E308B9080E03
:104E2000191E09E308B9F9014A9509E308B909F01F
:104E3000F00109E308B9099400E008B9199100E00C
:104E400008B9159F00E008B9080E191E00E008B95E
:104E5000F9014A9509E308B909F0F00109E308B935
:104E600009940FEF08B919910FEF08B9159F0FEFCB
:104E700008B9080E191E00E008B9F9014A9509E3BE
:104E800008B909F0F00109E308B909940FEF08B96E
:104E900019910FEF08B9159F0FEF08B9080E191EE9
:104EA0000FEF08B9F9014A9500E008B909F0F001DF
:104EB00009E308B909940FEF08B919910FEF08B980
:104EC000159F0FEF08B9080E191E0FEF08B9F90169
:104ED0004A950FEF08B909F0F00100E008B909940C
:104EE0000FEF08B919910FEF08B9159F0FEF08B927
:104EF000080E191E0FEF08B9F9014A950FEF08B90E
:104F000009F0F0010FEF08B909940FEF08B91991F2
:104F10000FEF08B9159F0FEF08B9080E191E0FEF14
:104F200008B9F9014A950FEF08B909F0F0010FEF40
:104F300008B909940FEF08B919910FEF08B9159F37
:104F40000FEF08B9080E191E0FEF08B9F9014A95BD
:104F50000FEF08B909F0F0010FEF08B9099409E360
:104F600008B9199100E008B9159F0FEF08B9080EAC
:104F7000191E00E008B9F9014A9509E308B909F0DA
:104F8000F00109E308B9099400E008B9199105E0B6
:104F900008B9159F05E008B9080E191E0FEF08B9EA
:104FA000F9014A9500E008B909F0F00100E008B9FC
:104FB000099409E308B9199100E008B9159F00E0C8
:104FC00008B9080E191E05E008B9F9014A950FEF56
:104FD00008B909F0F0010FEF08B9099409E308B91D
:104FE000199109E308B9159F09E308B9080E191EBC
:104FF00000E008B9F9014A9505E008B909F0F001A7
:1050000005E008B9099409E308B9199109E308B959
:10501000159F09E308B9080E191E00E008B9F90147
:105020004A950FEF08B909F0F00105E008B90994B5
:1050300000E008B9199100E008B9159F00E008B92F
:10504000080E191E0FEF08B9F9014A950FEF08B9BC
:1050500009F0F0010FEF08B909940FEF08B91991A1
:105060000FEF08B9159F0FEF08B9080E191E0FEFC3
:1050700008B9F9014A950FEF08B909F0F0010FEFEF
:1050800008B909940FEF08B919910FEF08B9159FE6
:105090000FEF08B9080E191E0FEF08B9F9014A956C
:1050A0000FEF08B909F0F0010FEF08B9099409E30F
:1050B00008B9199109E308B9159F00E008B9080E6D
:1050C000191E0FEF08B9F9014A950FEF08B909F059
:1050D000F0010FEF08B9099400E008B9199100E058
:1050E00008B9159F0FEF08B9080E191E0FEF08B980
:1050F000F9014A950FEF08B909F0F0010FEF08B96F
:1051000009940FEF08B9199105E008B9159F0FEF41
:1051100008B9080E191E0FEF08B9F9014A950FEFEB
:1051200008B909F0F0010FEF08B9099405E008B9D2
:1051300019910FEF08B9159F0FEF08B9080E191E46
:105140000FEF08B9F9014A950FEF08B909F0F0011E
:105150000FEF08B909940FEF08B919910FEF08B9CB
:10516000159F0FEF08B9080E191E0FEF08B9F901C6
:105170004A950FEF08B909F0F0010FEF08B909944B
:1051800005E008B919910FEF08B9159F0FEF08B99D
:10519000080E191E0FEF08B9F9014A950FEF08B96B
:1051A00009F0F0010FEF08B909940FEF08B9199150
:1051B00005E008B9159F0FEF08B9080E191E0FEF8B
:1051C00008B9F9014A950FEF08B909F0F0010FEF9E
:1051D00008B909940FEF08B919910FEF08B9159F95
:1051E0000FEF08B9080E191E0FEF08B9F9014A951B
:1051F0000FEF08B909F0F0010FEF08B909940FEFAC
:1052000008B919910FEF08B9159F0FEF08B9080EEB
:10521000191E0FEF08B9F9014A950FEF08B909F007
:10522000F0010FEF08B909940FEF08B9199108E5DB
:1052300008B9159F08E508B9080E191E08E508B950
:10524000F9014A950FEF08B909F0F0010FEF08B91D
:10525000099408E508B919910FEF08B9159F0FEFE8
:1052600008B9080E191E0FEF08B9F9014A9508E5AB
:1052700008B909F0F0010FEF08B9099408E508B979
:1052800019910FEF08B9159F0FEF08B9080E191EF5
:1052900008E508B9F9014A9508E508B909F0F001EF
:1052A0000FEF08B9099408E508B919910FEF08B98B
:1052B000159F08E508B9080E191E0FEF08B9F90186
:1052C0004A9508E508B909F0F0010FEF08B909940B
:1052D00008E508B9199108E508B9159F0FEF08B955
:1052E000080E191E0FEF08B9F9014A9508E508B92B
:1052F00009F0F0010FEF08B9099408E508B9199110
:105300000FEF08B9159F0FEF08B9080E191E0FEF20
:1053100008B9F9014A9508E508B909F0F0010FEF5D
:1053200008B909940FEF08B9199108E508B9159F54
:1053300008E508B9080E191E08E508B9F9014A95EB
:105340000FEF08B909F0F0010FEF08B909940FEF5A
:1053500008B919910FEF08B9159F0FEF08B9080E9A
:10536000191E0FEF08B9F9014A950FEF08B909F0B6
:10537000F0010FEF08B909940FEF08B919910FEF79
:1053800008B9159F08E508B9080E191E0FEF08B9EE
:10539000F9014A950FEF08B909F0F0010FEF08B9CC
:1053A00009940FEF08B9199108E508B9159F08E5A8
:1053B00008B9080E191E0FEF08B9F9014A950FEF49
:1053C00008B909F0F0010FEF08B909940FEF08B917
:1053D00019910FEF08B9159F08E508B9080E191EB5
:1053E0000FEF08B9F9014A950FEF08B909F0F0017C
:1053F0000FEF08B909940FEF08B919910FEF08B929
:10540000159F08E508B9080E191E0FEF08B9F90134
:105410004A950FEF08B909F0F0010FEF08B90994A8
:105420000FEF08B919910FEF08B9159F08E508B9F2
:10543000080E191E0FEF08B9F9014A950FEF08B9C8
:1054400009F0F0010FEF08B909940FEF08B91991AD
:105450000FEF08B9159F08E508B9080E191E0FEFE0
:1054600008B9F9014A950FEF08B909F0F0010FEFFB
:1054700008B909940FEF08B9199108E508B9159F03
:1054800008E508B9080E191E08E508B9F9014A959A
:105490000FEF08B909F0F0010FEF08B909940FEF09
:1054A00008B919910FEF08B9159F0FEF08B9080E49
:1054B000191E0FEF08B9F9014A950FEF08B909F065
:1054C000F0010FEF08B909940FEF08B9199108E539
:1054D00008B9159F08E508B9080E191E08E508B9AE
:1054E000F9014A950FEF08B909F0F0010FEF08B97B
:1054F000099408E508B919910FEF08B9159F0FEF46
:1055000008B9080E191E0FEF08B9F9014A9508E508
:1055100008B909F0F0010FEF08B909940FEF08B9C5
:1055200019910FEF08B9159F0FEF08B9080E191E52
:105530000FEF08B9F9014A9508E508B909F0F0013B
:105540000FEF08B909940FEF08B919910FEF08B9D7
:10555000159F08E508B9080E191E08E508B9F901F4
:105560004A950FEF08B909F0F0010FEF08B9099457
:105570000FEF08B9199108E508B9159F0FEF08B9A1
:10558000080E191E0FEF08B9F9014A950FEF08B977
:1055900009F0F0010FEF08B9099408E508B919916D
:1055A0000FEF08B9159F0FEF08B9080E191E0FEF7E
:1055B00008B9F9014A950FEF08B909F0F0010FEFAA
:1055C00008B9099408E508B9199108E508B9159FC3
:1055D00008E508B9080E191E08E508B9F9014A9549
:1055E00008E508B909F0F0010FEF08B909940FEFC9
:1055F00008B919910FEF08B9159F0FEF08B9080EF8
:10560000191E0FEF08B9F9014A950FEF08B909F013
:10561000F0010FEF08B909940FEF08B9199108E5E7
:1056200008B9159F08E508B9080E191E08E508B95C
:10563000F9014A950FEF08B909F0F0010FEF08B929
:10564000099408E508B919910FEF08B9159F0FEFF4
:1056500008B9080E191E0FEF08B9F9014A9508E5B7
:1056600008B909F0F0010FEF08B909940FEF08B974
:1056700019910FEF08B9159F0FEF08B9080E191E01
:105680000FEF08B9F9014A9508E508B909F0F001EA
:105690000FEF08B909940FEF08B9199108E508B997
:1056A000159F08E508B9080E191E08E508B9F901A3
:1056B0004A950FEF08B909F0F0010FEF08B9099406
:1056C0000FEF08B919910FEF08B9159F0FEF08B93F
:1056D000080E191E0FEF08B9F9014A9508E508B937
:1056E00009F0F0010FEF08B9099408E508B919911C
:1056F0000FEF08B9159F0FEF08B9080E191E0FEF2D
:1057000008B9F9014A9508E508B909F0F0010FEF69
:1057100008B909940FEF08B9199108E508B9159F60
:1057200008E508B9080E191E08E508B9F9014A95F7
:105730000FEF08B909F0F0010FEF08B909940FEF66
:1057400008B919910FEF08B9159F0FEF08B9080EA6
:10575000191E0FEF08B9F9014A950FEF08B909F0C2
:10576000F0010FEF08B909940FEF08B919910FEF85
:1057700008B9159F0FEF08B9080E191E08E508B9FA
:10578000F9014A950FEF08B909F0F0010FEF08B9D8
:1057900009940FEF08B919910FEF08B9159F08E5A3
:1057A00008B9080E191E08E508B9F9014A950FEF66
:1057B00008B909F0F0010FEF08B909940FEF08B923
:1057C000199108E508B9159F0FEF08B9080E191EC1
:1057D00008E508B9F9014A950FEF08B909F0F00199
:1057E0000FEF08B9099408E508B919910FEF08B946
:1057F000159F0FEF08B9080E191E08E508B9F90141
:105800004A950FEF08B909F0F0010FEF08B90994B4
:1058100008E508B9199108E508B9159F08E508B920
:10582000080E191E08E508B9F9014A9508E508B9F6
:1058300009F0F0010FEF08B909940FEF08B91991B9
:105840000FEF08B9159F0FEF08B9080E191E08E5EC
:1058500008B9F9014A950FEF08B909F0F0010FEF07
:1058600008B909940FEF08B919910FEF08B9159FFE
:105870000FEF08B9080E191E08E508B9F9014A9595
:105880000FEF08B909F0F0010FEF08B909940FEF15
:1058900008B919910FEF08B9159F0FEF08B9080E55
:1058A000191E0FEF08B9F9014A950FEF08B909F071
:1058B000F0010FEF08B9099408E508B9199108E556
:1058C00008B9159F08E508B9080E191E08E508B9BA
:1058D000F9014A9508E508B909F0F0010FEF08B998
:1058E000099408E508B919910FEF08B9159F0FEF52
:1058F00008B9080E191E0FEF08B9F9014A950FEF04
:1059000008B909F0F0010FEF08B9099408E508B9E2
:1059100019910FEF08B9159F0FEF08B9080E191E5E
:105920000FEF08B9F9014A950FEF08B909F0F00136
:105930000FEF08B9099408E508B9199108E508B905
:10594000159F08E508B9080E191E08E508B9F90100
:105950004A950FEF08B909F0F0010FEF08B9099463
:105960000FEF08B919910FEF08B9159F0FEF08B99C
:10597000080E191E0FEF08B9F9014A9508E508B994
:1059800009F0F0010FEF08B9099408E508B9199179
:105990000FEF08B9159F0FEF08B9080E191E0FEF8A
:1059A00008B9F9014A9508E508B909F0F0010FEFC7
:1059B00008B909940FEF08B9199108E508B9159FBE
:1059C00008E508B9080E191E08E508B9F9014A9555
:1059D0000FEF08B909F0F0010FEF08B909940FEFC4
:1059E00008B919910FEF08B9159F0FEF08B9080E04
:1059F000191E0FEF08B9F9014A950FEF08B909F020
:105A0000F0010FEF08B909940FEF08B919910FEFE2
:105A100008B9159F08E508B9080E191E08E508B968
:105A2000F9014A950FEF08B909F0F0010FEF08B935
:105A300009940FEF08B9199108E508B9159F0FEF00
:105A400008B9080E191E0FEF08B9F9014A950FEFB2
:105A500008B909F0F0010FEF08B9099408E508B991
:105A600019910FEF08B9159F0FEF08B9080E191E0D
:105A70000FEF08B9F9014A950FEF08B909F0F001E5
:105A80000FEF08B9099408E508B9199108E508B9B4
:105A9000159F08E508B9080E191E08E508B9F901AF
:105AA0004A950FEF08B909F0F0010FEF08B9099412
:105AB00008E508B919910FEF08B9159F0FEF08B95C
:105AC000080E191E0FEF08B9F9014A9508E508B943
:105AD00009F0F0010FEF08B9099408E508B9199128
:105AE0000FEF08B9159F0FEF08B9080E191E0FEF39
:105AF00008B9F9014A9508E508B909F0F0010FEF76
:105B000008B909940FEF08B9199108E508B9159F6C
:105B100008E508B9080E191E08E508B9F9014A9503
:105B20000FEF08B909F0F0010FEF08B909940FEF72
:105B300008B919910FEF08B9159F0FEF08B9080EB2
:105B4000191E0FEF08B9F9014A950FEF08B909F0CE
:105B5000F0010FEF08B9099408E508B9199108E5B3
:105B600008B9159F08E508B9080E191E08E508B917
:105B7000F9014A9508E508B909F0F0010FEF08B9F5
:105B800009940FEF08B919910FEF08B9159F0FEF9E
:105B900008B9080E191E0FEF08B9F9014A9508E572
:105BA00008B909F0F0010FEF08B909940FEF08B92F
:105BB00019910FEF08B9159F0FEF08B9080E191EBC
:105BC00008E508B9F9014A950FEF08B909F0F001A5
:105BD0000FEF08B909940FEF08B919910FEF08B941
:105BE000159F08E508B9080E191E0FEF08B9F9014D
:105BF0004A950FEF08B909F0F0010FEF08B90994C1
:105C00000FEF08B9199108E508B9159F0FEF08B90A
:105C1000080E191E0FEF08B9F9014A950FEF08B9E0
:105C200009F0F0010FEF08B909940FEF08B91991C5
:105C300008E508B9159F0FEF08B9080E191E0FEFF8
:105C400008B9F9014A950FEF08B909F0F0010FEF13
:105C500008B909940FEF08B9199108E508B9159F1B
:105C60000FEF08B9080E191E0FEF08B9F9014A9590
:105C70000FEF08B909F0F0010FEF08B909940FEF21
:105C800008B919910FEF08B9159F0FEF08B9080E61
:105C9000191E0FEF08B9F9014A950FEF08B909F07D
:105CA000F0010FEF08B909940FEF08B9199108E551
:105CB00008B9159F08E508B9080E191E08E508B9C6
:105CC000F9014A950FEF08B909F0F0010FEF08B993
:105CD000099408E508B919910FEF08B9159F0FEF5E
:105CE00008B9080E191E0FEF08B9F9014A9508E521
:105CF00008B909F0F0010FEF08B9099408E508B9EF
:105D000019910FEF08B9159F0FEF08B9080E191E6A
:105D10000FEF08B9F9014A9508E508B909F0F00153
:105D20000FEF08B909940FEF08B9199108E508B900
:105D3000159F08E508B9080E191E08E508B9F9010C
:105D40004A950FEF08B909F0F0010FEF08B909946F
:105D500008E508B919910FEF08B9159F0FEF08B9B9
:105D6000080E191E0FEF08B9F9014A9508E508B9A0
:105D700009F0F0010FEF08B9099408E508B9199185
:105D80000FEF08B9159F0FEF08B9080E191E0FEF96
:105D900008B9F9014A9508E508B909F0F0010FEFD3
:105DA00008B909940FEF08B9199108E508B9159FCA
:105DB00008E508B9080E191E08E508B9F9014A9561
:105DC0000FEF08B909F0F0010FEF08B909940FEFD0
:105DD00008B919910FEF08B9159F0FEF08B9080E10
:105DE000191E0FEF08B9F9014A950FEF08B909F02C
:105DF000F0010FEF08B909940FEF08B9199108E500
:105E000008B9159F08E508B9080E191E08E508B974
:105E1000F9014A950FEF08B909F0F0010FEF08B941
:105E2000099408E508B919910FEF08B9159F0FEF0C
:105E300008B9080E191E0FEF08B9F9014A9508E5CF
:105E400008B909F0F0010FEF08B9099408E508B99D
:105E500019910FEF08B9159F0FEF08B9080E191E19
:105E60000FEF08B9F9014A9508E508B909F0F00102
:105E70000FEF08B909940FEF08B9199108E508B9AF
:105E8000159F08E508B9080E191E08E508B9F901BB
:105E90004A9508E508B909F0F0010FEF08B909942F
:105EA0000FEF08B919910FEF08B9159F0FEF08B957
:105EB000080E191E0FEF08B9F9014A9508E508B94F
:105EC00009F0F0010FEF08B909940FEF08B9199123
:105ED0000FEF08B9159F0FEF08B9080E191E08E556
:105EE00008B9F9014A950FEF08B909F0F0010FEF71
:105EF00008B909940FEF08B9199108E508B9159F79
:105F000008E508B9080E191E0FEF08B9F9014A95FE
:105F10000FEF08B909F0F0010FEF08B909940FEF7E
:105F200008B919910FEF08B9159F0FEF08B9080EBE
:105F3000191E0FEF08B9F9014A950FEF08B909F0DA
:105F4000F0010FEF08B909940FEF08B919910FEF9D
:105F500008B9159F0FEF08B9080E191E0FEF08B901
:105F6000F9014A950FEF08B909F0F0010FEF08B9F0
:105F700009940FEF08B919910FEF08B9159F0FEFAA
:105F800008B9080E191E0FEF08B9F9014A950FEF6D
:105F900008B909F0F0010FEF08B909940FEF08B93B
:105FA000199108E908B9159F08E908B9080E191EE2
:105FB0000FEF08B9F9014A950FEF08B909F0F001A0
:105FC0000FEF08B909940FEF08B9199108E908B95A
:105FD000159F08E908B9080E191E0FEF08B9F90155
:105FE0004A950FEF08B909F0F0010FEF08B90994CD
:105FF0000FEF08B919910FEF08B9159F0FEF08B906
:10600000080E191E0FEF08B9F9014A950FEF08B9EC
:1060100009F0F0010FEF08B909940FEF08B91991D1
:1060200008E908B9159F08E908B9080E191E0FEF0D
:1060300008B9F9014A950FEF08B909F0F0010FEF1F
:1060400008B909940FEF08B9199108E908B9159F23
:1060500008E908B9080E191E0FEF08B9F9014A95A9
:106060000FEF08B909F0F0010FEF08B909940FEF2D
:1060700008B919910FEF08B9159F0FEF08B9080E6D
:10608000191E0FEF08B9F9014A9508E908B909F096
:10609000F0010FEF08B909940FEF08B919910FEF4C
:1060A00008B9159F0FEF08B9080E191E08E908B9BD
:1060B000F9014A950FEF08B909F0F0010FEF08B99F
:1060C00009940FEF08B9199108E908B9159F08E973
:1060D00008B9080E191E08E908B9F9014A950FEF29
:1060E00008B909F0F0010FEF08B9099408E908B9F7
:1060F00019910FEF08B9159F0FEF08B9080E191E77
:106100000FEF08B9F9014A9508E908B909F0F0015B
:106110000FEF08B9099408E908B919910FEF08B908
:10612000159F0FEF08B9080E191E0FEF08B9F901F6
:106130004A9508E908B909F0F0010FEF08B9099488
:1061400008E908B9199108E908B9159F08E908B9DB
:10615000080E191E08E908B9F9014A9508E908B9B5
:1061600009F0F0010FEF08B9099408E908B919918D
:106170000FEF08B9159F0FEF08B9080E191E0FEFA2
:1061800008B9F9014A9508E908B909F0F0010FEFDB
:1061900008B9099408E908B919910FEF08B9159FD2
:1061A0000FEF08B9080E191E0FEF08B9F9014A954B
:1061B00008E908B909F0F0010FEF08B909940FEFE9
:1061C00008B919910FEF08B9159F0FEF08B9080E1C
:1061D000191E0FEF08B9F9014A950FEF08B909F038
:1061E000F0010FEF08B909940FEF08B919910FEFFB
:1061F00008B9159F08E908B9080E191E08E908B979
:10620000F9014A950FEF08B909F0F0010FEF08B94D
:1062100009940FEF08B9199108E908B9159F0FEF14
:1062200008B9080E191E0FEF08B9F9014A9508E9D7
:1062300008B909F0F0010FEF08B9099408E908B9A5
:1062400019910FEF08B9159F08E908B9080E191E32
:1062500008E908B9F9014A950FEF08B909F0F0010A
:1062600008E908B9099408E908B919910FEF08B9C4
:10627000159F08E908B9080E191E0FEF08B9F901B2
:106280004A950FEF08B909F0F00108E908B9099437
:1062900008E908B919910FEF08B9159F08E908B97D
:1062A000080E191E08E908B9F9014A950FEF08B957
:1062B00009F0F00108E908B909940FEF08B919913C
:1062C00008E908B9159F0FEF08B9080E191E0FEF5E
:1062D00008B9F9014A9508E908B909F0F0010FEF8A
:1062E00008B909940FEF08B919910FEF08B9159F74
:1062F00008E908B9080E191E08E908B9F9014A9514
:106300000FEF08B909F0F0010FEF08B909940FEF8A
:1063100008B919910FEF08B9159F0FEF08B9080ECA
:10632000191E0FEF08B9F9014A950FEF08B909F0E6
:10633000F0010FEF08B909940FEF08B9199108E9B6
:1063400008B9159F08E908B9080E191E08E908B927
:10635000F9014A950FEF08B909F0F0010FEF08B9FC
:10636000099408E908B919910FEF08B9159F0FEFC3
:1063700008B9080E191E0FEF08B9F9014A9508E986
:1063800008B909F0F0010FEF08B9099408E908B954
:1063900019910FEF08B9159F0FEF08B9080E191ED4
:1063A0000FEF08B9F9014A9508E908B909F0F001B9
:1063B0000FEF08B9099408E908B919910FEF08B966
:1063C000159F0FEF08B9080E191E0FEF08B9F90154
:1063D0004A9508E908B909F0F0010FEF08B90994E6
:1063E00008E908B9199108E908B9159F08E908B939
:1063F000080E191E08E908B9F9014A9508E908B913
:1064000009F0F0010FEF08B9099408E908B91991EA
:106410000FEF08B9159F0FEF08B9080E191E0FEFFF
:1064200008B9F9014A9508E908B909F0F0010FEF38
:1064300008B9099408E908B919910FEF08B9159F2F
:106440000FEF08B9080E191E0FEF08B9F9014A95A8
:1064500008E908B909F0F0010FEF08B909940FEF46
:1064600008B919910FEF08B9159F0FEF08B9080E79
:10647000191E0FEF08B9F9014A950FEF08B909F095
:10648000F0010FEF08B9099408E908B9199108E972
:1064900008B9159F08E908B9080E191E08E908B9D6
:1064A000F9014A950FEF08B909F0F0010FEF08B9AB
:1064B000099408E908B919910FEF08B9159F0FEF72
:1064C00008B9080E191E0FEF08B9F9014A9508E935
:1064D00008B909F0F0010FEF08B9099408E908B903
:1064E00019910FEF08B9159F0FEF08B9080E191E83
:1064F0000FEF08B9F9014A9508E908B909F0F00168
:106500000FEF08B9099408E908B9199108E908B921
:10651000159F08E908B9080E191E08E908B9F9011C
:106520004A950FEF08B909F0F0010FEF08B9099487
:1065300008E908B919910FEF08B9159F0FEF08B9CD
:10654000080E191E0FEF08B9F9014A9508E908B9B4
:1065500009F0F0010FEF08B9099408E908B9199199
:106560000FEF08B9159F0FEF08B9080E191E0FEFAE
:1065700008B9F9014A9508E908B909F0F0010FEFE7
:1065800008B9099408E908B9199108E908B9159FEB
:1065900008E908B9080E191E08E908B9F9014A9571
:1065A0000FEF08B909F0F0010FEF08B909940FEFE8
:1065B00008B919910FEF08B9159F0FEF08B9080E28
:1065C000191E0FEF08B9F9014A950FEF08B909F044
:1065D000F0010FEF08B909940FEF08B9199108E914
:1065E00008B9159F08E908B9080E191E08E908B985
:1065F000F9014A950FEF08B909F0F0010FEF08B95A
:10660000099408E908B919910FEF08B9159F0FEF20
:1066100008B9080E191E0FEF08B9F9014A9508E9E3
:1066200008B909F0F0010FEF08B9099408E908B9B1
:1066300019910FEF08B9159F0FEF08B9080E191E31
:106640000FEF08B9F9014A950FEF08B909F0F00109
:106650000FEF08B9099408E908B919910FEF08B9C3
:10666000159F0FEF08B9080E191E0FEF08B9F901B1
:106670004A950FEF08B909F0F0010FEF08B9099436
:1066800008E908B919910FEF08B9159F0FEF08B97C
:10669000080E191E0FEF08B9F9014A950FEF08B956
:1066A00009F0F0010FEF08B9099408E908B9199148
:1066B0000FEF08B9159F0FEF08B9080E191E0FEF5D
:1066C00008B9F9014A9508E908B909F0F0010FEF96
:1066D00008B909940FEF08B9199108E908B9159F8D
:1066E00008E908B9080E191E08E908B9F9014A9520
:1066F0000FEF08B909F0F0010FEF08B909940FEF97
:1067000008B919910FEF08B9159F0FEF08B9080ED6
:10671000191E0FEF08B9F9014A950FEF08B909F0F2
:10672000F0010FEF08B9099408E908B9199108E9CF
:1067300008B9159F08E908B9080E191E08E908B933
:10674000F9014A950FEF08B909F0F0010FEF08B908
:10675000099408E908B919910FEF08B9159F0FEFCF
:1067600008B9080E191E0FEF08B9F9014A9508E992
:1067700008B909F0F0010FEF08B9099408E908B960
:1067800019910FEF08B9159F0FEF08B9080E191EE0
:106790000FEF08B9F9014A9508E908B909F0F001C5
:1067A0000FEF08B9099408E908B919910FEF08B972
:1067B000159F0FEF08B9080E191E0FEF08B9F90160
:1067C0004A9508E908B909F0F0010FEF08B90994F2
:1067D00008E908B919910FEF08B9159F0FEF08B92B
:1067E000080E191E0FEF08B9F9014A9508E908B912
:1067F00009F0F0010FEF08B9099408E908B91991F7
:106800000FEF08B9159F0FEF08B9080E191E0FEF0B
:1068100008B9F9014A9508E908B909F0F0010FEF44
:1068200008B9099408E908B9199108E908B9159F48
:1068300008E908B9080E191E08E908B9F9014A95CE
:106840000FEF08B909F0F0010FEF08B909940FEF45
:1068500008B919910FEF08B9159F0FEF08B9080E85
:10686000191E0FEF08B9F9014A950FEF08B909F0A1
:10687000F0010FEF08B9099408E908B9199108E97E
:1068800008B9159F08E908B9080E191E08E908B9E2
:10689000F9014A9508E908B909F0F0010FEF08B9C4
:1068A000099408E908B919910FEF08B9159F0FEF7E
:1068B00008B9080E191E0FEF08B9F9014A950FEF34
:1068C00008B909F0F0010FEF08B9099408E908B90F
:1068D00019910FEF08B9159F0FEF08B9080E191E8F
:1068E0000FEF08B9F9014A950FEF08B909F0F00167
:1068F0000FEF08B9099408E908B9199108E908B92E
:10690000159F08E908B9080E191E08E908B9F90128
:106910004A950FEF08B909F0F0010FEF08B9099493
:1069200008E908B919910FEF08B9159F0FEF08B9D9
:10693000080E191E0FEF08B9F9014A950FEF08B9B3
:1069400009F0F0010FEF08B9099408E908B91991A5
:106950000FEF08B9159F0FEF08B9080E191E0FEFBA
:1069600008B9F9014A950FEF08B909F0F0010FEFE6
:1069700008B9099408E908B9199108E908B9159FF7
:1069800008E908B9080E191E08E908B9F9014A957D
:1069900008E908B909F0F0010FEF08B909940FEF01
:1069A00008B919910FEF08B9159F0FEF08B9080E34
:1069B000191E0FEF08B9F9014A950FEF08B909F050
:1069C000F0010FEF08B9099408E908B9199108E92D
:1069D00008B9159F08E908B9080E191E08E908B991
:1069E000F9014A9508E908B909F0F0010FEF08B973
:1069F000099408E908B919910FEF08B9159F0FEF2D
:106A000008B9080E191E0FEF08B9F9014A950FEFE2
:106A100008B909F0F0010FEF08B9099408E908B9BD
:106A200019910FEF08B9159F0FEF08B9080E191E3D
:106A30000FEF08B9F9014A950FEF08B909F0F00115
:106A40000FEF08B9099408E908B9199108E908B9DC
:106A5000159F08E908B9080E191E08E908B9F901D7
:106A60004A950FEF08B909F0F0010FEF08B9099442
:106A700008E908B919910FEF08B9159F0FEF08B988
:106A8000080E191E0FEF08B9F9014A950FEF08B962
:106A900009F0F0010FEF08B9099408E908B9199154
:106AA0000FEF08B9159F0FEF08B9080E191E0FEF69
:106AB00008B9F9014A950FEF08B909F0F0010FEF95
:106AC00008B9099408E908B919910FEF08B9159F99
:106AD0000FEF08B9080E191E0FEF08B9F9014A9512
:106AE0000FEF08B909F0F0010FEF08B909940FEFA3
:106AF00008B919910FEF08B9159F0FEF08B9080EE3
:106B0000191E0FEF08B9F9014A950FEF08B909F0FE
:106B1000F0010FEF08B909940FEF08B9199108E9CE
:106B200008B9159F08E908B9080E191E08E908B93F
:106B3000F9014A950FEF08B909F0F0010FEF08B914
:106B4000099408E908B919910FEF08B9159F0FEFDB
:106B500008B9080E191E0FEF08B9F9014A9508E99E
:106B600008B909F0F0010FEF08B9099408E908B96C
:106B700019910FEF08B9159F0FEF08B9080E191EEC
:106B80000FEF08B9F9014A950FEF08B909F0F001C4
:106B90000FEF08B9099408E908B919910FEF08B97E
:106BA000159F08E908B9080E191E08E908B9F90186
:106BB0004A9508E908B909F0F0010FEF08B90994FE
:106BC00008E908B919910FEF08B9159F0FEF08B937
:106BD000080E191E0FEF08B9F9014A9508E908B91E
:106BE00009F0F0010FEF08B9099408E908B9199103
:106BF0000FEF08B9159F0FEF08B9080E191E0FEF18
:106C000008B9F9014A9508E908B909F0F0010FEF50
:106C100008B909940FEF08B9199108E908B9159F47
:106C200008E908B9080E191E08E908B9F9014A95DA
:106C300008E908B909F0F0010FEF08B909940FEF5E
:106C400008B919910FEF08B9159F0FEF08B9080E91
:106C5000191E0FEF08B9F9014A950FEF08B909F0AD
:106C6000F0010FEF08B9099408E908B919910FEF7D
:106C700008B9159F0FEF08B9080E191E0FEF08B9D4
:106C8000F9014A9508E908B909F0F0010FEF08B9D0
:106C9000099408E908B919910FEF08B9159F0FEF8A
:106CA00008B9080E191E0FEF08B9F9014A9508E94D
:106CB00008B909F0F0010FEF08B9099408E908B91B
:106CC00019910FEF08B9159F0FEF08B9080E191E9B
:106CD0000FEF08B9F9014A9508E908B909F0F00180
:106CE0000FEF08B9099408E908B9199108E908B93A
:106CF000159F08E908B9080E191E08E908B9F90135
:106D00004A9508E908B909F0F0010FEF08B90994AC
:106D100008E908B919910FEF08B9159F0FEF08B9E5
:106D2000080E191E0FEF08B9F9014A9508E908B9CC
:106D300009F0F0010FEF08B9099408E908B91991B1
:106D40000FEF08B9159F0FEF08B9080E191E0FEFC6
:106D500008B9F9014A9508E908B909F0F0010FEFFF
:106D600008B9099408E908B919910FEF08B9159FF6
:106D70000FEF08B9080E191E0FEF08B9F9014A956F
:106D800008E908B909F0F0010FEF08B909940FEF0D
:106D900008B919910FEF08B9159F0FEF08B9080E40
:106DA000191E0FEF08B9F9014A950FEF08B909F05C
:106DB000F0010FEF08B909940FEF08B9199108E92C
:106DC00008B9159F08E908B9080E191E08E908B99D
:106DD000F9014A950FEF08B909F0F0010FEF08B972
:106DE00009940FEF08B919910FEF08B9159F08E939
:106DF00008B9080E191E0FEF08B9F9014A950FEFEF
:106E000008B909F0F0010FEF08B909940FEF08B9BC
:106E100019910FEF08B9159F08E908B9080E191E56
:106E20000FEF08B9F9014A950FEF08B909F0F00121
:106E30000FEF08B909940FEF08B919910FEF08B9CE
:106E4000159F08E908B9080E191E0FEF08B9F901D6
:106E50004A950FEF08B909F0F0010FEF08B909944E
:106E60000FEF08B919910FEF08B9159F08E908B994
:106E7000080E191E0FEF08B9F9014A950FEF08B96E
:106E800009F0F0010FEF08B909940FEF08B9199153
:106E90000FEF08B9159F08E908B9080E191E0FEF82
:106EA00008B9F9014A950FEF08B909F0F0010FEFA1
:106EB00008B909940FEF08B9199108E908B9159FA5
:106EC00008E908B9080E191E08E908B9F9014A9538
:106ED0000FEF08B909F0F0010FEF08B909940FEFAF
:106EE00008B919910FEF08B9159F0FEF08B9080EEF
:106EF000191E0FEF08B9F9014A950FEF08B909F00B
:106F0000F0010FEF08B909940FEF08B919910FEFCD
:106F100008B9159F0FEF08B9080E191E0FEF08B931
:106F2000F9014A9508E908B909F0F0010FEF08B92D
:106F300009940FEF08B919910FEF08B9159F0FEFDA
:106F400008B9080E191E0FEF08B9F9014A9508E9AA
:106F500008B909F0F0010FEF08B909940FEF08B96B
:106F600019910FEF08B9159F0FEF08B9080E191EF8
:106F70000FEF08B9F9014A9508E908B909F0F001DD
:106F80000FEF08B909940FEF08B919910FEF08B97D
:106F9000159F0FEF08B9080E191E0FEF08B9F90178
:106FA0004A9508E908B909F0F0010FEF08B909940A
:106FB00008E908B919910FEF08B9159F0FEF08B943
:106FC000080E191E0FEF08B9F9014A9508E908B92A
:106FD00009F0F0010FEF08B9099408E908B919910F
:106FE0000FEF08B9159F0FEF08B9080E191E0FEF24
:106FF00008B9F9014A9508E908B909F0F0010FEF5D
:1070000008B909940FEF08B9199108E908B9159F53
:1070100008E908B9080E191E08E908B9F9014A95E6
:107020000FEF08B909F0F0010FEF08B909940FEF5D
:1070300008B919910FEF08B9159F0FEF08B9080E9D
:10704000191E0FEF08B9F9014A950FEF08B909F0B9
:10705000F0010FEF08B9099408E908B919910FEF89
:1070600008B9159F0FEF08B9080E191E0FEF08B9E0
:10707000F9014A9508E908B909F0F0010FEF08B9DC
:10708000099408E908B919910FEF08B9159F0FEF96
:1070900008B9080E191E08E908B9F9014A950FEF59
:1070A00008B909F0F0010FEF08B9099408E908B927
:1070B00019910FEF08B9159F08E908B9080E191EB4
:1070C0000FEF08B9F9014A950FEF08B909F0F0017F
:1070D0000FEF08B9099408E908B9199108E908B946
:1070E000159F0FEF08B9080E191E0FEF08B9F90127
:1070F0004A950FEF08B909F0F0010FEF08B90994AC
:1071000008E908B919910FEF08B9159F08E908B9FE
:10711000080E191E0FEF08B9F9014A950FEF08B9CB
:1071200009F0F0010FEF08B9099408E908B91991BD
:107130000FEF08B9159F0FEF08B9080E191E08E9DF
:1071400008B9F9014A950FEF08B909F0F0010FEFFE
:1071500008B9099408E908B919910FEF08B9159F02
:107160000FEF08B9080E191E0FEF08B9F9014A957B
:1071700008E908B909F0F0010FEF08B909940FEF19
:1071800008B919910FEF08B9159F0FEF08B9080E4C
:10719000191E0FEF08B9F9014A950FEF08B909F068
:1071A000F0010FEF08B9099408E908B919910FEF38
:1071B00008B9159F0FEF08B9080E191E0FEF08B98F
:1071C000F9014A950FEF08B909F0F0010FEF08B97E
:1071D000099408E908B919910FEF08B9159F0FEF45
:1071E00008B9080E191E0FEF08B9F9014A950FEFFB
:1071F00008B909F0F0010FEF08B9099408E908B9D6
:1072000019910FEF08B9159F0FEF08B9080E191E55
:107210000FEF08B9F9014A950FEF08B909F0F0012D
:107220000FEF08B9099408E908B919910FEF08B9E7
:10723000159F0FEF08B9080E191E0FEF08B9F901D5
:107240004A950FEF08B909F0F0010FEF08B909945A
:1072500008E908B919910FEF08B9159F0FEF08B9A0
:10726000080E191E0FEF08B9F9014A950FEF08B97A
:1072700009F0F0010FEF08B9099408E908B919916C
:107280000FEF08B9159F0FEF08B9080E191E0FEF81
:1072900008B9F9014A950FEF08B909F0F0010FEFAD
:1072A00008B9099408E908B9199108E908B9159FBE
:1072B00008E908B9080E191E08E908B9F9014A9544
:1072C00008E908B909F0F0010FEF08B909940FEFC8
:1072D00008B919910FEF08B9159F0FEF08B9080EFB
:1072E000191E0FEF08B9F9014A950FEF08B909F017
:1072F000F0010FEF08B9099408E908B919910FEFE7
:1073000008B9159F0FEF08B9080E191E0FEF08B93D
:10731000F9014A9508E908B909F0F0010FEF08B939
:10732000099408E908B9199108E908B9159F0FEF00
:1073300008B9080E191E08E908B9F9014A9508E9C3
:1073400008B909F0F0010FEF08B9099408E908B984
:1073500019910FEF08B9159F08E908B9080E191E11
:107360000FEF08B9F9014A9508E908B909F0F001E9
:107370000FEF08B9099408E908B919910FEF08B996
:10738000159F0FEF08B9080E191E0FEF08B9F90184
:107390004A9508E908B909F0F0010FEF08B9099416
:1073A00008E908B919910FEF08B9159F0FEF08B94F
:1073B000080E191E0FEF08B9F9014A9508E908B936
:1073C00009F0F0010FEF08B9099408E908B919911B
:1073D0000FEF08B9159F0FEF08B9080E191E0FEF30
:1073E00008B9F9014A9508E908B909F0F0010FEF69
:1073F00008B9099408E908B919910FEF08B9159F60
:107400000FEF08B9080E191E0FEF08B9F9014A95D8
:1074100008E908B909F0F0010FEF08B909940FEF76
:1074200008B919910FEF08B9159F0FEF08B9080EA9
:10743000191E0FEF08B9F9014A950FEF08B909F0C5
:10744000F0010FEF08B9099408E908B919910FEF95
:1074500008B9159F0FEF08B9080E191E0FEF08B9EC
:10746000F9014A9508E908B909F0F0010FEF08B9E8
:10747000099408E908B9199108E908B9159F0FEFAF
:1074800008B9080E191E0FEF08B9F9014A9508E965
:1074900008B909F0F0010FEF08B9099408E908B933
:1074A00019910FEF08B9159F08E908B9080E191EC0
:1074B0000FEF08B9F9014A9508E908B909F0F00198
:1074C0000FEF08B9099408E908B919910FEF08B945
:1074D000159F0FEF08B9080E191E08E908B9F90140
:1074E0004A9508E908B909F0F0010FEF08B90994C5
:1074F00008E908B919910FEF08B9159F0FEF08B9FE
:10750000080E191E0FEF08B9F9014A9508E908B9E4
:1075100009F0F0010FEF08B9099408E908B91991C9
:107520000FEF08B9159F0FEF08B9080E191E0FEFDE
:1075300008B9F9014A9508E908B909F0F0010FEF17
:1075400008B9099408E908B919910FEF08B9159F0E
:107550000FEF08B9080E191E0FEF08B9F9014A9587
:1075600008E908B909F0F0010FEF08B909940FEF25
:1075700008B919910FEF08B9159F0FEF08B9080E58
:10758000191E0FEF08B9F9014A950FEF08B909F074
:10759000F0010FEF08B909940FEF08B9199108E944
:1075A00008B9159F08E908B9080E191E08E908B9B5
:1075B000F9014A950FEF08B909F0F0010FEF08B98A
:1075C000099408E908B919910FEF08B9159F0FEF51
:1075D00008B9080E191E0FEF08B9F9014A9508E914
:1075E00008B909F0F0010FEF08B9099408E908B9E2
:1075F00019910FEF08B9159F0FEF08B9080E191E62
:107600000FEF08B9F9014A9508E908B909F0F00146
:107610000FEF08B9099408E908B919910FEF08B9F3
:10762000159F0FEF08B9080E191E0FEF08B9F901E1
:107630004A9508E908B909F0F0010FEF08B9099473
:1076400008E908B919910FEF08B9159F0FEF08B9AC
:10765000080E191E0FEF08B9F9014A9508E908B993
:1076600009F0F0010FEF08B9099408E908B9199178
:107670000FEF08B9159F0FEF08B9080E191E0FEF8D
:1076800008B9F9014A9508E908B909F0F0010FEFC6
:1076900008B909940FEF08B9199108E908B9159FBD
:1076A00008E908B9080E191E08E908B9F9014A9550
:1076B0000FEF08B909F0F0010FEF08B909940FEFC7
:1076C00008B919910FEF08B9159F0FEF08B9080E07
:1076D000191E0FEF08B9F9014A950FEF08B909F023
:1076E000F0010FEF08B9099408E908B9199108E900
:1076F00008B9159F08E908B9080E191E08E908B964
:10770000F9014A950FEF08B909F0F0010FEF08B938
:10771000099408E908B919910FEF08B9159F0FEFFF
:1077200008B9080E191E0FEF08B9F9014A9508E9C2
:1077300008B909F0F0010FEF08B9099408E908B990
:1077400019910FEF08B9159F0FEF08B9080E191E10
:107750000FEF08B9F9014A9508E908B909F0F001F5
:107760000FEF08B9099408E908B9199108E908B9AF
:10777000159F08E908B9080E191E08E908B9F901AA
:107780004A950FEF08B909F0F0010FEF08B9099415
:1077900008E908B919910FEF08B9159F0FEF08B95B
:1077A000080E191E0FEF08B9F9014A950FEF08B935
:1077B00009F0F0010FEF08B9099408E908B9199127
:1077C0000FEF08B9159F0FEF08B9080E191E0FEF3C
:1077D00008B9F9014A950FEF08B909F0F0010FEF68
:1077E00008B9099408E908B919910FEF08B9159F6C
:1077F0000FEF08B9080E191E0FEF08B9F9014A95E5
:107800000FEF08B909F0F0010FEF08B909940FEF75
:1078100008B919910FEF08B9159F0FEF08B9080EB5
:10782000191E0FEF08B9F9014A950FEF08B909F0D1
:10783000F0010FEF08B909940FEF08B9199108E9A1
:1078400008B9159F08E908B9080E191E08E908B912
:10785000F9014A950FEF08B909F0F0010FEF08B9E7
:10786000099408E908B919910FEF08B9159F0FEFAE
:1078700008B9080E191E0FEF08B9F9014A9508E971
:1078800008B909F0F0010FEF08B9099408E908B93F
:1078900019910FEF08B9159F0FEF08B9080E191EBF
:1078A0000FEF08B9F9014A9508E908B909F0F001A4
:1078B0000FEF08B9099408E908B919910FEF08B951
:1078C000159F0FEF08B9080E191E0FEF08B9F9013F
:1078D0004A9508E908B909F0F0010FEF08B90994D1
:1078E00008E908B919910FEF08B9159F08E908B917
:1078F000080E191E0FEF08B9F9014A9508E908B9F1
:1079000009F0F0010FEF08B9099408E908B91991D5
:107910000FEF08B9159F0FEF08B9080E191E08E9F7
:1079200008B9F9014A950FEF08B909F0F0010FEF16
:1079300008B909940FEF08B9199108E908B9159F1A
:1079400008E908B9080E191E0FEF08B9F9014A95A0
:1079500008E908B909F0F0010FEF08B909940FEF31
:1079600008B919910FEF08B9159F0FEF08B9080E64
:10797000191E0FEF08B9F9014A950FEF08B909F080
:10798000F0010FEF08B9099408E908B9199108E95D
:1079900008B9159F08E908B9080E191E08E908B9C1
:1079A000F9014A950FEF08B909F0F0010FEF08B996
:1079B000099408E908B919910FEF08B9159F0FEF5D
:1079C00008B9080E191E0FEF08B9F9014A9508E920
:1079D00008B909F0F0010FEF08B9099408E908B9EE
:1079E00019910FEF08B9159F0FEF08B9080E191E6E
:1079F0000FEF08B9F9014A9508E908B909F0F00153
:107A00000FEF08B9099408E908B9199108E908B90C
:107A1000159F08E908B9080E191E08E908B9F90107
:107A20004A950FEF08B909F0F0010FEF08B9099472
:107A300008E908B919910FEF08B9159F0FEF08B9B8
:107A4000080E191E08E908B9F9014A950FEF08B99F
:107A500009F0F0010FEF08B9099408E908B9199184
:107A60000FEF08B9159F0FEF08B9080E191E0FEF99
:107A700008B9F9014A9508E908B909F0F0010FEFD2
:107A800008B9099408E908B919910FEF08B9159FC9
:107A90000FEF08B9080E191E0FEF08B9F9014A9542
:107AA00008E908B909F0F0010FEF08B909940FEFE0
:107AB00008B919910FEF08B9159F0FEF08B9080E13
:107AC000191E0FEF08B9F9014A950FEF08B909F02F
:107AD000F0010FEF08B909940FEF08B9199108E9FF
:107AE00008B9159F08E908B9080E191E08E908B970
:107AF000F9014A950FEF08B909F0F0010FEF08B945
:107B0000099408E908B919910FEF08B9159F0FEF0B
:107B100008B9080E191E0FEF08B9F9014A9508E9CE
:107B200008B909F0F0010FEF08B9099408E908B99C
:107B300019910FEF08B9159F0FEF08B9080E191E1C
:107B40000FEF08B9F9014A950FEF08B909F0F001F4
:107B50000FEF08B909940FEF08B9199108E908B9AE
:107B6000159F08E908B9080E191E08E908B9F901B6
:107B70004A950FEF08B909F0F0010FEF08B9099421
:107B80000FEF08B919910FEF08B9159F0FEF08B95A
:107B9000080E191E0FEF08B9F9014A9508E908B94E
:107BA00009F0F0010FEF08B9099408E908B9199133
:107BB0000FEF08B9159F0FEF08B9080E191E0FEF48
:107BC00008B9F9014A9508E908B909F0F0010FEF81
:107BD00008B909940FEF08B9199108E908B9159F78
:107BE00008E908B9080E191E08E908B9F9014A950B
:107BF0000FEF08B909F0F0010FEF08B909940FEF82
:107C000008B919910FEF08B9159F0FEF08B9080EC1
:107C1000191E0FEF08B9F9014A950FEF08B909F0DD
:107C2000F0010FEF08B9099408E908B9199108E9BA
:107C300008B9159F08E908B9080E191E08E908B91E
:107C4000F9014A9508E908B909F0F0010FEF08B900
:107C500009940FEF08B919910FEF08B9159F08E9BA
:107C600008B9080E191E0FEF08B9F9014A950FEF70
:107C700008B909F0F0010FEF08B909940FEF08B93E
:107C800019910FEF08B9159F08E908B9080E191ED8
:107C90000FEF08B9F9014A950FEF08B909F0F001A3
:107CA0000FEF08B909940FEF08B919910FEF08B950
:107CB000159F08E908B9080E191E0FEF08B9F90158
:107CC0004A950FEF08B909F0F0010FEF08B90994D0
:107CD0000FEF08B919910FEF08B9159F08E908B916
:107CE000080E191E0FEF08B9F9014A950FEF08B9F0
:107CF00009F0F0010FEF08B909940FEF08B91991D5
:107D00000FEF08B9159F08E908B9080E191E0FEF03
:107D100008B9F9014A950FEF08B909F0F0010FEF22
:107D200008B909940FEF08B919910FEF08B9159F19
:107D300008E908B9080E191E0FEF08B9F9014A95AC
:107D40000FEF08B909F0F0010FEF08B909940FEF30
:107D500008B919910FEF08B9159F0FEF08B9080E70
:107D6000191E0FEF08B9F9014A950FEF08B909F08C
:107D7000F0010FEF08B9099408E908B919910FEF5C
:107D800008B9159F0FEF08B9080E191E0FEF08B9B3
:107D9000F9014A9508E908B909F0F0010FEF08B9AF
:107DA000099408E908B919910FEF08B9159F0FEF69
:107DB00008B9080E191E0FEF08B9F9014A9508E92C
:107DC00008B909F0F0010FEF08B9099408E908B9FA
:107DD00019910FEF08B9159F0FEF08B9080E191E7A
:107DE0000FEF08B9F9014A9508E908B909F0F0015F
:107DF0000FEF08B9099408E908B919910FEF08B90C
:107E0000159F0FEF08B9080E191E0FEF08B9F901F9
:107E10004A9508E908B909F0F0010FEF08B909948B
:107E200008E908B919910FEF08B9159F0FEF08B9C4
:107E3000080E191E0FEF08B9F9014A9508E908B9AB
:107E400009F0F0010FEF08B9099408E908B9199190
:107E50000FEF08B9159F0FEF08B9080E191E0FEFA5
:107E600008B9F9014A9508E908B909F0F0010FEFDE
:107E700008B909940FEF08B9199108E908B9159FD5
:107E800008E908B9080E191E08E908B9F9014A9568
:107E90000FEF08B909F0F0010FEF08B909940FEFDF
:107EA00008B919910FEF08B9159F0FEF08B9080E1F
:107EB000191E0FEF08B9F9014A950FEF08B909F03B
:107EC000F0010FEF08B9099408E908B919910FEF0B
:107ED00008B9159F0FEF08B9080E191E0FEF08B962
:107EE000F9014A9508E908B909F0F0010FEF08B95E
:107EF000099408E908B919910FEF08B9159F0FEF18
:107F000008B9080E191E0FEF08B9F9014A9508E9DA
:107F100008B909F0F0010FEF08B9099408E908B9A8
:107F200019910FEF08B9159F0FEF08B9080E191E28
:107F30000FEF08B9F9014A9508E908B909F0F0010D
:107F40000FEF08B9099408E908B919910FEF08B9BA
:107F5000159F0FEF08B9080E191E0FEF08B9F901A8
:107F60004A9508E908B909F0F0010FEF08B909943A
:107F700008E908B919910FEF08B9159F0FEF08B973
:107F8000080E191E0FEF08B9F9014A9508E908B95A
:107F900009F0F0010FEF08B909940FEF08B9199132
:107FA00008E908B9159F0FEF08B9080E191E08E96E
:107FB00008B9F9014A950FEF08B909F0F0010FEF80
:107FC00008B909940FEF08B919910FEF08B9159F77
:107FD00008E908B9080E191E0FEF08B9F9014A950A
:107FE0000FEF08B909F0F0010FEF08B909940FEF8E
:107FF00008B919910FEF08B9159F0FEF08B9080ECE
:10800000191E0FEF08B9F9014A950FEF08B909F0E9
:10801000F0010FEF08B9099408E908B919910FEFB9
:1080200008B9159F0FEF08B9080E191E0FEF08B910
:10803000F9014A9508E908B909F0F0010FEF08B90C
:10804000099408E908B919910FEF08B9159F0FEFC6
:1080500008B9080E191E0FEF08B9F9014A9508E989
:1080600008B909F0F0010FEF08B9099408E908B957
:1080700019910FEF08B9159F08E908B9080E191EE4
:108080000FEF08B9F9014A9508E908B909F0F001BC
:108090000FEF08B9099408E908B919910FEF08B969
:1080A000159F08E908B9080E191E0FEF08B9F90164
:1080B0004A9508E908B909F0F0010FEF08B90994E9
:1080C00008E908B919910FEF08B9159F08E908B92F
:1080D000080E191E0FEF08B9F9014A9508E908B909
:1080E00009F0F0010FEF08B9099408E908B91991EE
:1080F0000FEF08B9159F08E908B9080E191E0FEF10
:1081000008B9F9014A9508E908B909F0F0010FEF3B
:1081100008B909940FEF08B9199108E908B9159F32
:108120000FEF08B9080E191E08E908B9F9014A95B8
:108130000FEF08B909F0F0010FEF08B909940FEF3C
:1081400008B919910FEF08B9159F0FEF08B9080E7C
:10815000191E0FEF08B9F9014A950FEF08B909F098
:10816000F0010FEF08B9099408E908B919910FEF68
:1081700008B9159F0FEF08B9080E191E0FEF08B9BF
:10818000F9014A9508E908B909F0F0010FEF08B9BB
:10819000099408E908B919910FEF08B9159F0FEF75
:1081A00008B9080E191E0FEF08B9F9014A9508E938
:1081B00008B909F0F0010FEF08B909940FEF08B9F9
:1081C000199108E908B9159F0FEF08B9080E191E93
:1081D00008E908B9F9014A950FEF08B909F0F0016B
:1081E0000FEF08B909940FEF08B919910FEF08B90B
:1081F000159F08E908B9080E191E0FEF08B9F90113
:108200004A950FEF08B909F0F0010FEF08B909948A
:108210000FEF08B9199108E908B9159F0FEF08B9D0
:10822000080E191E08E908B9F9014A950FEF08B9B7
:1082300009F0F0010FEF08B9099408E908B919919C
:108240000FEF08B9159F0FEF08B9080E191E0FEFB1
:1082500008B9F9014A9508E908B909F0F0010FEFEA
:1082600008B9099408E908B919910FEF08B9159FE1
:108270000FEF08B9080E191E0FEF08B9F9014A955A
:1082800008E908B909F0F0010FEF08B909940FEFF8
:1082900008B919910FEF08B9159F0FEF08B9080E2B
:1082A000191E0FEF08B9F9014A950FEF08B909F047
:1082B000F0010FEF08B9099408E908B919910FEF17
:1082C00008B9159F0FEF08B9080E191E0FEF08B96E
:1082D000F9014A9508E908B909F0F0010FEF08B96A
:1082E000099408E908B919910FEF08B9159F0FEF24
:1082F00008B9080E191E0FEF08B9F9014A9508E9E7
:1083000008B909F0F0010FEF08B9099408E908B9B4
:1083100019910FEF08B9159F0FEF08B9080E191E34
:108320000FEF08B9F9014A9508E908B909F0F00119
:108330000FEF08B909940FEF08B9199108E908B9C6
:10834000159F0FEF08B9080E191E08E908B9F901C1
:108350004A950FEF08B909F0F0010FEF08B9099439
:108360000FEF08B919910FEF08B9159F08E908B97F
:10837000080E191E0FEF08B9F9014A950FEF08B959
:1083800009F0F0010FEF08B909940FEF08B919913E
:108390000FEF08B9159F08E908B9080E191E0FEF6D
:1083A00008B9F9014A950FEF08B909F0F0010FEF8C
:1083B00008B909940FEF08B919910FEF08B9159F83
:1083C00008E908B9080E191E0FEF08B9F9014A9516
:1083D0000FEF08B909F0F0010FEF08B909940FEF9A
:1083E00008B919910FEF08B9159F0FEF08B9080EDA
:1083F000191E0FEF08B9F9014A950FEF08B909F0F6
:10840000F0010FEF08B9099408E908B9199108E9D2
:1084100008B9159F08E908B9080E191E08E908B936
:10842000F9014A950FEF08B909F0F0010FEF08B90B
:1084300009940FEF08B919910FEF08B9159F0FEFC5
:1084400008B9080E191E08E908B9F9014A950FEF95
:1084500008B909F0F0010FEF08B909940FEF08B956
:1084600019910FEF08B9159F08E908B9080E191EF0
:108470000FEF08B9F9014A950FEF08B909F0F001BB
:108480000FEF08B909940FEF08B9199108E908B975
:10849000159F0FEF08B9080E191E0FEF08B9F90163
:1084A0004A950FEF08B909F0F0010FEF08B90994E8
:1084B00008E908B919910FEF08B9159F0FEF08B92E
:1084C000080E191E0FEF08B9F9014A950FEF08B908
:1084D00009F0F0010FEF08B9099408E908B91991FA
:1084E0000FEF08B9159F0FEF08B9080E191E0FEF0F
:1084F00008B9F9014A950FEF08B909F0F0010FEF3B
:1085000008B9099408E908B9199108E908B9159F4B
:1085100008E908B9080E191E08E908B9F9014A95D1
:108520000FEF08B909F0F0010FEF08B90994000244
:10853000060000FB00FF0002090000F100FF00013F
:10854000280000FBFA010102050000FF0001050000
:1085500000E219010302050000FF0001000000E233
:108560000F010302050000FF0001000000FB96015F
:108570000302050000FF00020800085504085A0025
:1085800000F8000990000A1E32050000FF000000FC
:108590002E8500000000000000368500000000016C
:1085A00000003E85000000000100004C8500000036
:1085B000000100005A8500000000010000688500ED
:1085C00000000000000076850000000000B0077F7A
:1085D000005C00000B7F00902B5F00FF0601530042
:1085E000C00000B1077F005C00000B7F00C10000ED
:1085F000912B5F00B2077F005C00000B7F00C20080
:108600000092365F0D90375F0091325F0092375FC6
:108610000E90305F0091305F0092395F0E903C5FAA
:108620000091375F00923B5F0E902B5F00912B5FB4
:108630000E90375F0091325F0092375F0E90305F8F
:108640000091305F0092395F0E903C5F0091375F80
:108650000092375F0E902B5F00912B5F0E90375F7B
:108660000091325F0E90305F0091305F0D903C5F63
:108670000091375F0E902B5F00912B5F0E90375F5C
:108680000091325F0E90305F0091305F0E903C5F42
:108690000091375F0E902B5F00912B5F0092365F49
:1086A0000E90375F0091325F0092375F0E90305F1F
:1086B0000091305F0092395F0E903C5F0091375F10
:1086C00000923B5F0E902B5F00912B5F0D90375F08
:1086D0000091325F0092375F0E90305F0091305F03
:1086E0000092395F0E903C5F0091375F0092375FD8
:1086F0000E902B5F00912B5F0E90375F0091325FE1
:108700000E90305F0091305F0E903C5F0091375FBC
:108710000E902B5F00912B5F0E90375F0091325FC0
:108720000E90305F0091305F0D903C5F0091375F9D
:108730000E902B5F00912B5F0092365F0E90375F9B
:108740000091325F0092375F0E90305F0091305F92
:108750000092395F0E903C5F0091375F00923B5F63
:108760000E902B5F00912B5F0E90375F0091325F70
:108770000092375F0E90305F0091305F0092395F5A
:108780000E903C5F0091375F0092375F0E902B5F39
:1087900000912B5F0E90375F0091325F0D90305F3C
:1087A0000091305F0E903C5F0091375F0E902B5F21
:1087B00000912B5F0E90375F0091325F0E90305F1B
:1087C0000091305F0E903C5F0091375F0E902B5F01
:1087D00000912B5F0092365F0E90375F0091325F01
:1087E0000092375F0E90305F0091305F0092395FEA
:1087F0000E903C5F0091375F00923B5F0D902B5FC6
:1088000000912B5F0E90375F0091325F0092375FCF
:108810000E90305F0091305F0092395F0E903C5FA8
:108820000091375F0092375F0E902B5F00912B5FB6
:108830000E90375F0091325F0E90305F0091305F95
:108840000E903C5F0091375F0E902B5F00912B5F85
:108850000E90375F0091325F0D90305F0091305F76
:108860000E903C5F0091375F0E90325F0091325F57
:1088700000923E5F0E903E5F0091395F00923E5F36
:108880000E90305F0091305F00923E5F0E903C5F33
:108890000091375F00923C5F0E902B5F00912B5F41
:1088A00000923B5F0E90375F0091325F0092375F1E
:1088B0000E902B5F00912B5F00923B5F0E90375F15
:1088C0000091325F0092375F0E90325F0091325F0D
:1088D0000092365F0D903E5F0091395F0092375FE6
:1088E0000E90305F0091305F0092375F0E903C5FDA
:1088F0000091375F0092425F0E902B5F00912B5FDB
:108900000092375F0E90375F0091325F0E902B5FC1
:1089100000912B5F0E90375F0091325F0E90325FB7
:108920000091325F00923E5F0E903E5F0091395F92
:1089300000923E5F0E90305F0091305F00923E5F8C
:108940000D903C5F0091375F00923C5F0E902B5F73
:1089500000912B5F00923B5F0E90375F0091325F7A
:108960000092375F0E902B5F00912B5F00923B5F70
:108970000E90375F0091325F0092375F0E90325F4A
:108980000091325F0092365F0E903E5F0091395F3A
:108990000092375F0E90305F0091305F0092375F3A
:1089A0000E903C5F0091375F0092425F0E902B5F0C
:1089B00000912B5F0092375F0D90375F0091325F1F
:1089C0000E902B5F00912B5F0E90375F0091325F0E
:1089D0000E90325F0091325F00923E5F0E903E5FDC
:1089E0000091395F00923E5F0E90305F0091305FE2
:1089F00000923E5F0E903C5F0091375F00923C5FBB
:108A00000E902B5F00912B5F00923B5F0E90375FC3
:108A10000091325F0092375F0E902B5F00912B5FC9
:108A200000923B5F0D90375F0091325F0092375F9D
:108A30000E90325F0091325F0092365F0E903E5F83
:108A40000091395F0092375F0E90305F0091305F88
:108A50000092375F0E903C5F0091375F0092425F5B
:108A60000E902B5F00912B5F0092375F0E90375F67
:108A70000091325F0E902B5F00912B5F0E90375F5D
:108A80000091325F0E90325F0091325F00923E5F44
:108A90000E903E5F0091395F00923E5F0D90305F17
:108AA0000091305F00923E5F0E903C5F0091375F17
:108AB00000923C5F0E902B5F00912B5F00923B5F1A
:108AC0000E90375F0091325F0092375F0E902B5F00
:108AD00000912B5F00923B5F0E90375F0091325FF9
:108AE0000092375F0E90325F0091325F0092365FE6
:108AF0000E903E5F0091395F0092375F0E90305FBD
:108B00000091305F0092375F0E903C5F0091375FBD
:108B10000092425F0D902B5F00912B5F0092375FB8
:108B20000E90375F0091325F0E902B5F00912B5FAC
:108B30000E90375F0091325F0E902B5F00912B5F9C
:108B40000092365F0E90375F0091325F0092375F80
:108B50000E90305F0091305F0092395F0E903C5F65
:108B60000091375F00923B5F0E902B5F00912B5F6F
:108B70000E90375F0091325F0092375F0D90305F4B
:108B80000091305F0092395F0E903C5F0091375F3B
:108B90000092375F0E902B5F00912B5F0E90375F36
:108BA0000091325F0E90305F0091305F0E903C5F1D
:108BB0000091375F0E902B5F00912B5F0E90375F17
:108BC0000091325F0E90305F0091305F0E903C5FFD
:108BD0000091375F0E902B5F00912B5F0092365F04
:108BE0000D90375F0091325F0092375F0E90305FDB
:108BF0000091305F0092395F0E903C5F0091375FCB
:108C000000923B5F0E902B5F00912B5F0E90375FC1
:108C10000091325F0092375F0E90305F0091305FBD
:108C20000092395F0E903C5F0091375F0092375F92
:108C30000E902B5F00912B5F0E90375F0091325F9B
:108C40000E90305F0091305F0D903C5F0091375F78
:108C50000E902B5F00912B5F0E90375F0091325F7B
:108C60000E90305F0091305F0E903C5F0091375F57
:108C70000E902B5F00912B5F0092365F0E90375F56
:108C80000091325F0092375F0E90305F0091305F4D
:108C90000092395F0E903C5F0091375F00923B5F1E
:108CA0000E902B5F00912B5F0D90375F0091325F2C
:108CB0000092375F0E90305F0091305F0092395F15
:108CC0000E903C5F0091375F0092375F0E902B5FF4
:108CD00000912B5F0E90375F0091325F0E90305FF6
:108CE0000091305F0E903C5F0091375F0E902B5FDC
:108CF00000912B5F0E90375F0091325F0E90305FD6
:108D00000091305F0D903C5F0091375F0E902B5FBC
:108D100000912B5F0092365F0E90375F0091325FBB
:108D20000092375F0E90305F0091305F0092395FA4
:108D30000E903C5F0091375F00923B5F0E902B5F7F
:108D400000912B5F0E90375F0091325F0092375F8A
:108D50000E90305F0091305F0092395F0E903C5F63
:108D60000091375F0092375F0E902B5F00912B5F71
:108D70000E90375F0091325F0D90305F0091305F51
:108D80000E903C5F0091375F0E902B5F00912B5F40
:108D90000E90375F0091325F0E90305F0091305F30
:108DA0000E903C5F0091375F0E90325F0091325F12
:108DB00000923E5F0E903E5F0091395F00923E5FF1
:108DC0000E90305F0091305F00923E5F0E903C5FEE
:108DD0000091375F00923C5F0D902B5F00912B5FFD
:108DE00000923B5F0E90375F0091325F0092375FD9
:108DF0000E902B5F00912B5F00923B5F0E90375FD0
:108E00000091325F0092375F0E90325F0091325FC7
:108E10000092365F0E903E5F0091395F0092375F9F
:108E20000E90305F0091305F0092375F0E903C5F94
:108E30000091375F0092425F0E902B5F00912B5F95
:108E40000092375F0E90375F0091325F0D902B5F7D
:108E500000912B5F0E90375F0091325F0E90325F72
:108E60000091325F00923E5F0E903E5F0091395F4D
:108E700000923E5F0E90305F0091305F00923E5F47
:108E80000E903C5F0091375F00923C5F0E902B5F2D
:108E900000912B5F00923B5F0E90375F0091325F35
:108EA0000092375F0E902B5F00912B5F00923B5F2B
:108EB0000E90375F0091325F0092375F0E90325F05
:108EC0000091325F0092365F0D903E5F0091395FF6
:108ED0000092375F0E90305F0091305F0092375FF5
:108EE0000E903C5F0091375F0092425F0E902B5FC7
:108EF00000912B5F0092375F0E90375F0091325FD9
:108F00000E902B5F00912B5F0E90375F0091325FC8
:108F10000E90325F0091325F00923E5F0E903E5F96
:108F20000091395F00923E5F0E90305F0091305F9C
:108F300000923E5F0D903C5F0091375F00923C5F76
:108F40000E902B5F00912B5F00923B5F0E90375F7E
:108F50000091325F0092375F0E902B5F00912B5F84
:108F600000923B5F0E90375F0091325F0092375F57
:108F70000E90325F0091325F0092365F0E903E5F3E
:108F80000091395F0092375F0E90305F0091305F43
:108F90000092375F0E903C5F0091375F0092425F16
:108FA0000E902B5F00912B5F0092375F0D90375F23
:108FB0000091325F0E902B5F00912B5F0E90375F18
:108FC0000091325F0E90325F0091325F00923E5FFF
:108FD0000E903E5F0091395F00923E5F0E90305FD1
:108FE0000091305F00923E5F0E903C5F0091375FD2
:108FF00000923C5F0E902B5F00912B5F00923B5FD5
:109000000E90375F0091325F0092375F0E902B5FBA
:1090100000912B5F00923B5F0E90375F0091325FB3
:109020000092375F0D90325F0091325F0092365FA1
:109030000E903E5F0091395F0092375F0E90305F77
:109040000091305F0092375F0E903C5F0091375F78
:109050000092425F0E902B5F00912B5F0092375F72
:109060000E90375F0091325F0E902B5F00912B5F67
:109070000E90375F0091325F0EFF06014500FF2F13
:109080000000FF06015300B00747005C00000B7FA3
:1090900000C00100902B5F00B10747005C00000B8F
:1090A0007F00C10000912B5F00B20757005C0000F9
:1090B0000B7F00C2000092475F0F90325F00912B40
:1090C0005F0F902F5F0091325F00924A5F0F9032E6
:1090D0005F0091325F00924A5F10902B5F00912BEE
:1090E0005F0092475F0F90325F00912B5F0F902FD0
:1090F0005F0091325F0092455F1090325F009132C5
:109100005F0092455F0F902B5F00912B5F009243B1
:109110005F0F90325F00912B5F0F902F5F009132B5
:109120005F1090325F0091325F0F902B5F00912BA8
:109130005F00924F5F0F90325F00912B5F00924F64
:109140005F10902F5F0091325F00924F5F0F90325F
:109150005F0091325F00924F5F0F90305F0091305F
:109160005F00924C5F0F90375F0091305F1090343A
:109170005F0091375F00924A5F0F90375F00913731
:109180005F00924A5F0F90305F0091305F0092471E
:109190005F1090375F0091305F0F90345F00913720
:1091A0005F0092455F0F90375F0091375F009245F7
:1091B0005F1090305F0091305F0092435F0F9037F7
:1091C0005F0091305F0F90345F0091375F0F9037F1
:1091D0005F0091375F1090305F0091305F00924CDC
:1091E0005F0F90375F0091305F00924C5F0F9034BB
:1091F0005F0091375F00924C5F1090375F009137AE
:109200005F00924C5F0F902B5F00912B5F009247A5
:109210005F0F90325F00912B5F0F902F5F009132B4
:109220005F00924A5F1090325F0091325F00924A75
:109230005F0F902B5F00912B5F0092475F0F903282
:109240005F00912B5F10902F5F0091325F0092457D
:109250005F0F90325F0091325F0092455F0F902B5D
:109260005F00912B5F0092435F1090325F00912B63
:109270005F0F902F5F0091325F0F90325F0091324D
:109280005F0F902B5F00912B5F1090325F00912B4E
:109290005F0F902F5F0091325F0F90325F0091322D
:1092A0005F1090325F0091325F00924C5F0F9039F7
:1092B0005F0091325F00924A5F0F90365F009139F4
:1092C0005F00924C5F0F90395F0091395F00924AC6
:1092D0005F1090325F0091325F00924A5F0F9039C9
:1092E0005F0091325F0092475F0F90365F009139C7
:1092F0005F00924A5F1090395F0091395F0092479A
:109300005F0F90305F0091305F0092455F0F9037A4
:109310005F0091305F0092475F1090345F0091379B
:109320005F0092455F0F90375F0091375F00924773
:109330005F0F90305F0091305F0092435F0F903776
:109340005F0091305F1090345F0091375F00924072
:109350005F0F90375F0091375F0F902B5F00912B6D
:109360005F00923E5F1090325F00912B5F0F902F55
:109370005F0091325F0F90325F0091325F0F902B50
:109380005F00912B5F00923B5F1090325F00912B4A
:109390005F0F902F5F0091325F0F90325F0091322C
:1093A0005F1090325F0091325F00923E5F0F903904
:1093B0005F0091325F0F90365F0091395F0F9039F7
:1093C0005F0091395F1090325F0091325F0F9039EA
:1093D0005F0091325F0F90365F0091395F109039D6
:1093E0005F0091395F0FFF06014500FF2F0040200D
:1093F000464C3F56494F205A4156414E203230315B
:1094000030004C4943454E53454420554E44455247
:1094100020474E552047504C205633004D45444977
:109420004120554E4445522043432041534120336F
:1094300020554E504F52544544004D5553494320FA
:1094400042592049444552414C444F204C55495AB9
:109450002044412053494C56410057575720444F10
:1094600054204E45424F534F534F20444F542043B6
:109470004F4D003120504C415945520000003220E0
:10948000504C41594552533A0044454C41593A00D9
:10949000000000004D415A453A0000000000005312
:1094A0004F554E443A00000000004E4F4E4500001C
:1094B0000000424F524445525300524F4F4D53000B
:1094C000000048414C4C574159004E4F524D414CC1
:1094D0000000535045454455500047524F5754489B
:1094E000000054494D45440000004E4F20534F5555
:1094F0004E440000000000004D55534943204F4E9C
:109500004C5900000000534658204F4E4C59000063
:10951000000000004D5553494320414E442053461E
:1095200058004D494E555445533A0053495A453A0F
:1095300000504C4159455220313A00504C41594558
:109540005220323A0047414D45204F564552005077
:109550004C41594552203120574F4E00504C4159F3
:109560004552203220574F4E004452415700544933
:109570004D453A2020202020203A005041555345A7
:109580004400524553554D4500515549540011244E
:109590001FBECFEFD0E1DEBFCDBF14BE88E10FB656
:1095A000F89480936000109260000FBE11E0A0E07C
:1095B000B1E0E2E4FFEC02C005900D92A831B107E2
:1095C000D9F71CE0A8E1B1E001C01D92AB3FB107A3
:1095D000E1F70E942555882311F40E943C55F89428
:1095E000E0ECF7E080E8819399E0EC3CF907D9F7EB
:1095F00080EC97E09093CD098093CC091092CE092E
:109600001092D1091092DB091092E5091092EF092E
:1096100081E08093F1098093F2098093F009109220
:10962000810015BC9FEF97B994B998E99AB95C9AF3
:109630009CE091B99BEF92B91092A80796E09093A5
:10964000A907109285001092840093E090938900FE
:109650009DE89093880099E09093810092E0909328
:109660006F0092E494BD17BC85BD93E89093B00061
:109670001092B3008093B10081E185B91092BD07CB
:109680001092AC071092AD071092B8071092B7076E
:109690001092BC071092BB071092BE070E94D754CD
:1096A00080E00E94B85480FF03C084E00E94B5545B
:1096B0000E94455A78940E94475A0E9402660C9470
:1096C0009F670C940000EFEC00C000C0EA95E1F742
:1096D00000C000C00000C8E1D1E000EEA02E662767
:1096E00072D139E23A95F1F70E949E4B30E13A95FA
:1096F000F1F70000AA9489F0C8956395683029F0C5
:10970000C895C895C8950000EBCF662700243CE3B8
:10971000C30FD01DC8950000E3CF35E03A95F1F7AF
:1097200000C051D111E00091AB0701270093AB07B6
:109730001093AA07E2E0E09336000895CF93DF93F9
:1097400024EB3BE458EA75E18091B2079091B307AE
:1097500096958795679F800D911D4991459F080EAD
:10976000191EF0014CE30994002708B9DF91CF914D
:10977000089501E008B9199102E008B9159F03E0C6
:1097800008B9080E191E04E008B9F9014A9505E068
:1097900008B909F0F00106E008B9099401E008B938
:1097A000199102E008B9159F03E008B9080E191EC7
:1097B00004E008B9F9014A9505E008B911F0F00193
:1097C00006E008B9099401E008B9199102E008B966
:1097D000159F03E008B9080E191E04E008B9F90145
:1097E0004A9505E008B911F0F00106E008B90994BE
:1097F00001E008B9199102E008B9159F03E008B922
:10980000080E191E04E008B9F9014A9505E008B9E7
:1098100011F0F00106E008B9099401E008B91991C6
:1098200002E008B9159F03E008B9080E191E04E00C
:1098300008B9F9014A9505E008B911F0F00106E010
:1098400008B9099401E008B9199102E008B9159F17
:1098500003E008B9080E191E04E008B9F9014A9599
:1098600005E008B911F0F00106E008B9099401E03B
:1098700008B9199102E008B9159F03E008B9080E6C
:10988000191E04E008B9F9014A9505E008B911F07C
:10989000F00106E008B9099401E008B9199102E065
:1098A00008B9159F03E008B9080E191E04E008B9AD
:1098B000F9014A9505E008B911F0F00106E008B990
:1098C0000994F14C004D0E4D654C28980E949A4E1B
:1098D000EBE0EA95F1F700C0E7E0E0938900EBE107
:1098E000E0938800E0E0F6E0BED0289AE0FF30D0B8
:1098F000E0FF2DC02F933F934F935F936F937F9320
:109900008F939F93AF93BF9378941124E091AE0708
:10991000F091AF07E115F10509F009950E94465A4B
:109920000E9414550E94C74D1124E091B007F09198
:10993000B107E115F10509F00995BF91AF919F912C
:109940008F917F916F915F914F913F912F910895EA
:10995000EF93E091A907E93E80F4E93070F0EDE182
:10996000FF2700800F92EA95E1F70E94634BE1E048
:10997000FF270F900192EE31E0F3EF910895FF93EE
:10998000EF93EFB7EF93E0918400EE50F1E0EF1723
:1099900000F0F395FA30D8F305D0EF91EFBFEF91D7
:1099A000FF9118950F921F92E2ECF8E90090A8073A
:1099B000000C1124E00DF11D05901490F0010995A3
:1099C0001F900F90089528980E949A4EE5E1EA951D
:1099D000F1F7E091A907EA95E093A907289A00C05A
:1099E000089528980E94BC4E289A0000E1E0F6E015
:1099F0003AD0E3E0E0938900EDE8E0938800089531
:109A000028980E94BC4EE9EA0000EA95E9F700C0F8
:109A10000000F6E0E2E027D0289A089528980E94F6
:109A2000BC4E289A0000E3E0FDEF1DD0E091A907AD
:109A3000E53091F4E091AB07E1300000F091BD0713
:109A400019F4F091BD07F195E3E0E0938900EDE8AA
:109A5000EF0FE09388000895E3E0E0938900EDE8DC
:109A6000E093880008950090A9070A9410905F0081
:109A700011FC0F2E0092A9070090A80711FC0E2ED2
:109A80000092A807E0E011FCE1E00895000000006A
:109A900000000000000000000000000000000000C6
:109AA00000000000000000000000000000000000B6
:109AB00000000000000000000000000000000000A6
:109AC0000000000000000000000000000000000096
:109AD0000000000000000000000000000000000086
:109AE0000000000000000000000000000000000076
:109AF0000000000000000000000000000000000066
:109B000099277727833008F00895ECE8FDE9660F80
:109B1000771FE60FF71FA591B491E1EDF9E02AE078
:109B2000289FE00DF11DA183B28311240895909127
:109B3000F0099170880F892B8093F0090895992777
:109B40007727E1EDF9E02AE0289FE00DF11D6E3F57
:109B500031F46091F0096E7F6093F0090BC06F3FA4
:109B600031F46091F0096E6F6093F00903C07FE9F2
:109B7000760F75831124089599277727E1EDF9E091
:109B80002AE0289FE00DF11D6083112408950E94B2
:109B9000F7560090CE09002019F4A0ECB7E002C0FF
:109BA000A6ECB8E021E002260092CE0922E0209344
:109BB000CF092F923F924F925F926F927F928F9236
:109BC0009F92AF92BF92CF92DF92EF92FF920F934C
:109BD0001F93CF93DF935091EF096091F10970913A
:109BE000F2098091F3092090D2093090D309409076
:109BF000D5095090D6096090D4091091D109709080
:109C0000DC098090DD099090DE09A090DF09B0901A
:109C1000E0092091DB09C090E609D090E709E090C7
:109C2000E909F090EA090091E8093091E5099FEF10
:109C3000620C431CF2014491410300240008C12D31
:109C4000D02D970CA81CF501449142030024000874
:109C5000C10DD01D0C0DED1CF701449143030024F0
:109C60000008C10DD01D8A956AF44091F009842F37
:109C70008695062E0694062600FA7695679576F95F
:109C800040FF66F940E860FD4FE745030024000807
:109C9000C10DD01D0024C038D0050CF0CFE70A94C8
:109CA000C038D0050CF4C0E8C058CD939A9509F09F
:109CB000BFCF4091CF094A954093CF0997E009F073
:109CC000B7CF6092D4094092D5099092DE09A09254
:109CD000DF090093E809E092E9096093F1097093C4
:109CE000F2098093F309DF91CF911F910F91FF90BB
:109CF000EF90DF90CF90BF90AF909F908F907F902C
:109D00006F905F904F903F902F900895E091CC0915
:109D1000F091CD09019100000093B30009E0EC3C03
:109D2000F00700EC17E008F0F801E093CC09F0939D
:109D3000CD0908950C949C4E0C949E4E0F931F9346
:109D40002F93E091CC09F091CD0901910093B300DC
:109D500009E0EC3CF00708F400C010F0E0ECF7E09C
:109D6000E093CC09F093CD0926E02A95F1F700C0E5
:109D70002F911F910F9108950000E091A907E0FF36
:109D8000DDCFE1E1EA95F1F700C00895220024005B
:109D9000260028002B002D0030003300360039004B
:109DA0003D004000440048004C00510056005B005C
:109DB000600066006C0073007900810088009000EC
:109DC0009900A200AC00B600C100CC00D800E500AC
:109DD000F3000101100121013201440157016C011E
:109DE00081019801B001CA01E5010202210241028C
:109DF00064028802AE02D7020303300361039403B6
:109E0000CB03050442048304C70410055D05AF05B8
:109E100005066106C2062907960709088308050991
:109E20008E09200ABA0A5D0B0A0CC10C840D510E72
:109E30002B0F121007110A121D1340147415BA16B5
:109E400014188319071BA31C571E24200E22142448
:109E500039267F28E82A752D293006330F364539F3
:109E6000AD3C49401B442848734CFE50CF55EA5A3C
:109E700051600C661D6C8B725A79928037885090B5
:109E8000E598FDA19FABD3B5A3C000000000000082
:109E900000000000000000000000000000000000C2
:109EA00000000000000000000000000000000000B2
:109EB00000000000000000000000000000000000A2
:109EC0000000000000000000000000000000000092
:109ED0000000000000000000000000000000000082
:109EE0000000000000000000000000000000000072
:109EF0000000000000000000000000000000000062
:109F0000000306090C101316191C1F2225282B2EDE
:109F1000313336393C3F414447494C4E51535558F3
:109F20005A5C5E60626466686A6B6D6F70717374B0
:109F3000757678797A7A7B7C7D7D7E7E7E7F7F7F69
:109F40007F7F7F7F7E7E7E7D7D7C7B7A7A7978764F
:109F500075747371706F6D6B6A68666462605E5C65
:109F60005A585553514E4C494744413F3C3936337A
:109F7000312E2B2825221F1C191613100C0906033D
:109F800000FDFAF7F4F0EDEAE7E4E1DEDBD8D5D244
:109F9000CFCDCAC7C4C1BFBCB9B7B4B2AFADABA80F
:109FA000A6A4A2A09E9C9A9896959391908F8D8C32
:109FB0008B8A888786868584838382828281818159
:109FC0008181818182828283838485868687888A53
:109FD0008B8C8D8F9091939596989A9C9EA0A2A41D
:109FE000A6A8ABADAFB2B4B7B9BCBFC1C4C7CACDE8
:109FF000CFD2D5D8DBDEE1E4E7EAEDF0F4F7FAFD05
:10A00000808182838485868788898A8B8C8D8E8FD8
:10A01000909192939495969798999A9B9C9D9E9FC8
:10A02000A0A1A2A3A4A5A6A7A8A9AAABACADAEAFB8
:10A03000B0B1B2B3B4B5B6B7B8B9BABBBCBDBEBFA8
:10A04000C0C1C2C3C4C5C6C7C8C9CACBCCCDCECF98
:10A05000D0D1D2D3D4D5D6D7D8D9DADBDCDDDEDF88
:10A06000E0E1E2E3E4E5E6E7E8E9EAEBECEDEEEF78
:10A07000F0F1F2F3F4F5F6F7F8F9FAFBFCFDFEFF68
:10A08000000102030405060708090A0B0C0D0E0F58
:10A09000101112131415161718191A1B1C1D1E1F48
:10A0A000202122232425262728292A2B2C2D2E2F38
:10A0B000303132333435363738393A3B3C3D3E3F28
:10A0C000404142434445464748494A4B4C4D4E4F18
:10A0D000505152535455565758595A5B5C5D5E5F08
:10A0E000606162636465666768696A6B6C6D6E6FF8
:10A0F000707172737475767778797A7B7C7D7E7FE8
:10A1000000020406080A0C0E10121416181A1C1E5F
:10A1100020222426282A2C2E30323436383A3C3E4F
:10A1200040424446484A4C4E50525456585A5C5E3F
:10A1300060626466686A6C6E70727476787A7C7E2F
:10A140007F7D7B79777573716F6D6B69676563610F
:10A150005F5D5B59575553514F4D4B4947454341FF
:10A160003F3D3B39373533312F2D2B2927252321EF
:10A170001F1D1B19171513110F0D0B0907050301DF
:10A18000FFFDFBF9F7F5F3F1EFEDEBE9E7E5E3E1CF
:10A19000DFDDDBD9D7D5D3D1CFCDCBC9C7C5C3C1BF
:10A1A000BFBDBBB9B7B5B3B1AFADABA9A7A5A3A1AF
:10A1B0009F9D9B99979593918F8D8B89878583819F
:10A1C00080828486888A8C8E90929496989A9C9E9F
:10A1D000A0A2A4A6A8AAACAEB0B2B4B6B8BABCBE8F
:10A1E000C0C2C4C6C8CACCCED0D2D4D6D8DADCDE7F
:10A1F000E0E2E4E6E8EAECEEF0F2F4F6F8FAFCFE6F
:10A200007F7F7F7F7F7F7F7F7F7F7F7F7F7F7F7F5E
:10A210007F7F7F7F7F7F7F7F7F7F7F7F7F7F7F7F4E
:10A220007F7F7F7F7F7F7F7F7F7F7F7F7F7F7F7F3E
:10A230007F7F7F7F7F7F7F7F7F7F7F7F7F7F7F7F2E
:10A500000309131E28313A40464C5054585B5E6193
:10A51000636567696B6C6E6F707172737475767753
:10A52000777879797A7A7B7B7C7C7C7D7D7D7E7E79
:10A530007E7E7F7F7F7F7F7F7F7F7F7F7F7F7F7F2D
:10A540007F7F7F7F7F7F7F7F7F7F7F7F7F7E7E7E1E
:10A550007E7D7D7D7C7C7C7B7B7A7A797978777750
:10A56000767574737271706F6E6C6B696765636119
:10A570005E5B5854504C46403A31281E1309030084
:10A58000C6CCD5DBDFE3E5E7E9EAEBECEDEEEFEF98
:10A59000F0F0F0F1F1F1F1F2F2F2F2F2F2F2F2F3A4
:10A5A000F3F3F3F3F3F3F3F3F3F3F3F3F3F3F3F37B
:10A5B000F3F3F3F3F3F3F3F3F3F3F3F3F3F3F3F36B
:10A5C000F3F3F3F3F3F3F3F3F3F3F3F3F3F3F3F35B
:10A5D000F3F3F3F3F3F3F3F3F3F3F3F3F3F3F3F34B
:10A5E000F2F2F2F2F2F2F2F2F1F1F1F1F0F0F0EF58
:10A5F000EFEEEDECEBEAE9E7E5E3DFDBD5CCC60017
:10A6000000283D42302D2C2B2C2D2E2F303233356F
:10A6100037393B3D3F414345484A4C4E50535557CF
:10A62000595B5D5F61636567696B6C6E70717374B4
:10A63000757778797A7B7C7D7D7E7E7F7F7F7F7F5B
:10A640007F7F7F7F7F7F7E7E7D7D7C7B7A79787741
:10A6500075747371706E6C6B69676563615F5D5B68
:10A6600059575553504E4C4A484543413F3D3B395D
:10A6700037353332302F2E2D2C2B2C2D30423D28C8
:10A6800000E9E5FED4D7D7D7D6D4D2D0CECCCAC82D
:10A69000C6C3C1BFBDBAB8B6B4B1AFADABA9A7A56B
:10A6A000A3A19F9E9C9A999795949391908F8D8C3E
:10A6B0008B8A89888887868585848484838383833D
:10A6C0008383838383848484858586878888898A35
:10A6D0008B8C8D8F909193949597999A9C9E9FA126
:10A6E000A3A5A7A9ABADAFB1B4B6B8BABDBFC1C33E
:10A6F000C6C8CACCCED0D2D4D6D7D7D7D4FEE5E9F7
:10A70000F9F8F9F5EBE1DDDEE0E2E4E5E6E5E4E2C7
:10A71000DED9D2CAC1B7ACA299918A8683818080E2
:10A720008182838586888A8C8D8F90929395969767
:10A7300098999A9B9B9C9D9D9D9E9E9E9F9F9F9F4F
:10A740009F9F9F9E9E9E9D9D9D9C9B9B9A99989747
:10A7500096959392908F8D8C8A888685838281804E
:10A76000808183868A9199A2ACB7C1CAD2D9DEE230
:10A77000E4E5E6E5E4E2E0DEDDE1EBF5F9F8F90039
:10A780000708070B151F2322201E1C1B1A1B1C1E4B
:10A7900022272E363F49545E676F767A7E7F7F7F11
:10A7A0007F7E7D7B7A7876747371706E6D6B6A696B
:10A7B0006867666565646463636262626161616162
:10A7C000616161626262636363646565666768694B
:10A7D0006A6B6D6E7071737476787A7B7D7E7F7F25
:10A7E0007F7F7E7A766F675E54493F362E27221E22
:10A7F0001C1B1A1B1C1E2022231F150B07080700F9
:10A800001F313D444E5354565A5F64696E747679D5
:10A810007C7F7F7F7F7F7F7F7F7F7F7F7F7F7F7F4B
:10A820007F7F7F7F7F7F7F7F7F7F7F7F7F7F7F7F38
:10A830007F7F7F7F7F7F7F7F7F7F7F7F7F7F7F7F28
:10A840007F7F7F7F7F7F7F7F7F7F7F7F7F7F7F7F18
:10A850007F7F7F7F7F7F7F7F7F7F7F7F7F7F7F7F08
:10A860007F7F7F7F7F7F7F7F7F7F7F7F7F7F7F7FF8
:10A870007F7F7F7F7F7F7F7F7F7F7F7C7871684C4A
:10A880002C1C120C0A0B0A05FDF3E9DFD4CAC0B771
:10A89000AEA69E97918B8685828080808080808006
:10A8A00080808080808080808080808080808080A8
:10A8B0008080808080808080808080808080808098
:10A8C0008080808080808080808080808080808088
:10A8D0008080808080808080808080808080808078
:10A8E0008080808080808080808080808080808068
:10A8F000808080808087919DACC4CBD4DDF2FAFA51
:10A90000E0E9F6E0A8E1B1E060E06D933197E9F7A6
:10A9100011240895992777272CE3629F080E191EAA
:10A92000A8E1B1E0A00DB11D4C9311240895992721
:10A930002CE3629F080E191EA8E1B1E0A00DB11D25
:10A940005091B407450F4C93112408958093B40798
:10A9500008958093B2079093B30708958091AA0752
:10A96000089511241092AA0708958093BD070895B1
:10A97000882329F48091B5079091B60708958091B6
:10A98000B9079091BA070895F999FECF92BD81BD9C
:10A9900060BDF894FA9AF99A78940895F999FECFDF
:10A9A00092BD81BDF894F89A80B578940895129A72
:10A9B000C895C895129840E080E090E020E030E033
:10A9C00036952795969587951398C895C895009BB9
:10A9D0003068019B9068139AC895C8954F5F4031C5
:10A9E00079F73093B6072093B5079093BA07809311
:10A9F000B9078091B5079091B6078F30910539F06E
:10AA00008091B9079091BA078F30910561F428E0E1
:10AA100088E190E00FB6F894A895809360000FBE8F
:10AA200020936000FFCF08951092060A009903C09A
:10AA300081E08093060A019905C08091060A826030
:10AA40008093060A0E94D75408951F9380E090E0F7
:10AA50000E94CE54182F81E090E00E94CE5490E0E6
:10AA6000382F20E0210F311D85E52A35380709F4FC
:10AA700091E0892F1F910895CF93DF93C0E0D0E03C
:10AA8000FE01E059FF4F6491CE010E94C45421960B
:10AA9000C032D105A9F7C0E2D0E0CE016FEF0E942D
:10AAA000C454CE0101966FEF0E94C454A09688E072
:10AAB000C030D80791F7DF91CF91089590E026E15B
:10AAC00030E0829FF001839FF00D929FF00D1124E2
:10AAD000E75FF54F628708956093F009089590E06D
:10AAE00026E130E0829FF001839FF00D929FF00DF0
:10AAF0001124E75FF54F13861182089590E026E157
:10AB000030E0829FF001839FF00D929FF00D1124A1
:10AB1000E75FF54F81E0838B089590E026E130E018
:10AB2000829FF001839FF00D929FF00D1124E75F4B
:10AB3000F54F6187089590E026E130E0829FF001B3
:10AB4000839FF00D929FF00D1124E75FF54F648312
:10AB5000089590E026E130E0829FF001839FF00DA0
:10AB6000929FF00D1124E75FF54F65830895909350
:10AB7000640A8093630A8FE68093690A1092BF0784
:10AB8000E9E0FAE021E08FEF98E1208310868683E8
:10AB9000878314861182958376963AE0E136F3072F
:10ABA000A1F7089510920A0A1092200A1092360A0C
:10ABB00010924C0A019690936D0A80936C0A9093C0
:10ABC000080A8093070A9093700A80936F0A109284
:10ABD0006B0A10926A0A1092620A1092610A10922D
:10ABE000650A81E08093BF071092680A1092670A95
:10ABF0000895E3E1FAE09091000186E1989FC00199
:10AC000011248E0F9F1F2AEF04C0308137FF20834D
:10AC10007696E817F907C9F71092BF070895DC0187
:10AC20002D913C911197A9014F5F5F4F11965C9355
:10AC30004E93F901249130E027FF15C02F77307033
:10AC40003695322F222737952795CA014F5F5F4FE0
:10AC5000FC018491982F9F77290F311D87FDF0CF3C
:10AC600011965C934E93C9010895FC01108A1286D7
:10AC70008FEF81876087138A118A91E09387128A08
:10AC800014828683428308958093690A08950E94FE
:10AC90009F4D0895EF92FF920F931F93DF93CF93F1
:10ACA00000D0CDB7DEB7182F062FE82EFF2486E19F
:10ACB00090E0E89EF001E99EF00DF89EF00D112461
:10ACC000E75FF54F8385882321F08181882309F090
:10ACD00085C0222391F486E190E0E89EF001E99E90
:10ACE000F00DF89EF00D1124E75FF54F138A828571
:10ACF000882309F073C0108671C0133059F481E0C5
:10AD000091E09093F2098093F10981E08093F0093A
:10AD1000042F0DC0812F60E02A8349830E949F4D3C
:10AD2000812F4981642F0E94804D49812A810F37EC
:10AD300089F486E190E0E89EF001E99EF00DF89E2E
:10AD4000F00D1124E75FF54F8091660A878787E64B
:10AD50009AE02CC089E0089FC0011124E091630AA9
:10AD6000F091640AE80FF91F33968591949100974A
:10AD700071F486E190E0E89EF001E99EF00DF89E06
:10AD8000F00D1124E75FF54F158A148A11C0FC01FC
:10AD9000349166E170E0E69EF001E79EF00DF69ECC
:10ADA000F00D1124E75FF54F37870196958B848B63
:10ADB00086E190E0E89EF001E99EF00DF89EF00D2E
:10ADC0001124E75FF54F0487118286E1189FC001C7
:10ADD0001124875F954F622F0E9435560F900F9078
:10ADE000CF91DF911F910F91FF90EF900895CF9237
:10ADF000DF92EF92FF921F93CF93DF93E2E1FAE0AD
:10AE00008181992787FD90952081820F911D8F3F29
:10AE1000910519F014F08FEF90E097FF02C080E0E9
:10AE200090E0808376968AE0EA36F80749F78091C9
:10AE3000BF07882309F05FC17AC140916C0A509125
:10AE40006D0ADA011196B0936D0AA0936C0AFA01AB
:10AE500044914F3F71F5BD016F5F7F4F70936D0A55
:10AE600060936C0AFD01A491AF3219F41092BF07F0
:10AE700050C1A63009F032C1FB0131969F012F5F0E
:10AE80003F4F30936D0A20936C0A8491833529F4E7
:10AE90003093700A20936F0A21C1853409F01EC1D6
:10AEA00080916F0A9091700A90936D0A80936C0A5A
:10AEB00015C147FF02C04093650A842F8F70242F6D
:10AEC00030E0207F30702039310541F0203B3105E2
:10AED000A1F0203C310509F076C05EC09D012F5FD6
:10AEE0003F4FFD014491B9016F5F7F4F70936D0A31
:10AEF00060936C0AF901249181C09D012F5F3F4F3F
:10AF0000FD01A491A9014F5F5F4F50936D0A4093DB
:10AF10006C0AF9019491A73071F4282F30E02C9F2E
:10AF2000F0012D9FF00D3C9FF00D1124E75FF54FD0
:10AF3000990F9783D3C0AB3071F4282F30E02C9F4A
:10AF4000F0012D9FF00D3C9FF00D1124E75FF54FB0
:10AF5000990F9683C3C0AC3571F4282F30E02C9F35
:10AF6000F0012D9FF00D3C9FF00D1124E75FF54F90
:10AF7000990F9483B3C0A43609F0B0C0282F30E0F5
:10AF80002C9FF0012D9FF00D3C9FF00D1124E75FE9
:10AF9000F54F990F9583A2C09D012F5F3F4F3093CE
:10AFA0006D0A20936C0AFD01249190E08C9FD001E2
:10AFB0008D9FB00D9C9FB00D1124A75FB54F1C96BF
:10AFC0002C931C978BC02091650A822F8F7030E0E4
:10AFD000207F30702039310541F0203B310511F1DF
:10AFE000203C310509F07AC06EC09D012F5F3F4FB4
:10AFF00030936D0A20936C0AFD012491682F70E054
:10B000006C9FF0016D9FF00D7C9FF00D1124E75FA8
:10B01000F54F9081992309F461C0220F64850E9445
:10B020004A565CC09D012F5F3F4F30936D0A2093BD
:10B030006C0AFD012491473081F490E08C9FD0018F
:10B040008D9FB00D9C9FB00D1124A75FB54FE22FCF
:10B05000EE0F1796EC93179741C04B3081F490E0B8
:10B060008C9FD0018D9FB00D9C9FB00D1124A75FC8
:10B07000B54FE22FEE0F1696EC9316972FC04C3576
:10B0800081F490E08C9FD0018D9FB00D9C9FB00DFE
:10B090001124A75FB54FE22FEE0F1496EC9314978F
:10B0A0001DC04436D9F490E08C9FD0018D9FB00D27
:10B0B0009C9FB00D1124A75FB54FE22FEE0F1596A0
:10B0C000EC9315970BC090E08C9FF0018D9FF00DD5
:10B0D0009C9FF00D1124E75FF54F44878CE69AE0C2
:10B0E0000E940F5690936B0A80936A0A1092620A2C
:10B0F0001092610A02C0C6E1D0E08091610A90918D
:10B10000620A20916A0A30916B0A8217930709F448
:10B1100094CE01969093620A8093610A8091670AA7
:10B120009091680A01969093680A8093670A11EDDE
:10B13000E12E19E0F12ECAE0DAE010E0BFEFCB2EED
:10B14000D12C8A89882309F05BC08B899C89009760
:10B1500009F453C09F858E85981708F049C04DC0EB
:10B160008B85EB89FC898F37E1F4DF018D91BC8BF6
:10B17000AB8B8F3FF1F061811196BC8BAB8BE82FCD
:10B18000F0E0EE0FFF1FE057FF4F0190F081E02D40
:10B19000812F0995EB89FC8981918E87FC8BEB8B44
:10B1A00026C0BF016F5F7F4F7C8B6B8B84918F3F7D
:10B1B00021F418821C8A1B8A20C09B012F5F3F4FFD
:10B1C0003C8B2B8BFB01649190E0880F991F80577B
:10B1D0009F4FFC0125913491812FF9010995EB894D
:10B1E000FC89CF0101969C8B8B8BE491EE871F86A7
:10B1F0009F858E85981709F4B3CF8F858F5F8F87D2
:10B200008A85882319F480E090E068C088898F3FA0
:10B2100011F08F5F888B8F81882309F459C038859E
:10B22000332309F455C09E81992309F451C020911C
:10B23000690A222309F44CC0989FC0011124805050
:10B240009F4F692F7727432F50E0649FC001659F70
:10B25000900D749F900D112480509F4F692F772778
:10B260004D8150E0649FC001659F900D749F900DCB
:10B27000112480509F4F492F552730E0429FC00135
:10B28000439F900D529F900D112480509F4F892F06
:10B2900099273B813323F1F0EA81F0E0E050F14659
:10B2A00024912058239F9001112420503F4F232F99
:10B2B0003327A601421B530B489F9001499F300D35
:10B2C000589F300D112420503F4F832F992702C0E3
:10B2D00080E090E02A813C81230F2A83F70180835C
:10B2E0001F5F8AE090E0E80EF91E6696143009F0C0
:10B2F00028CFDF91CF911F91FF90EF90DF90CF90FB
:10B300000895EF92FF920F931F93CF93DF9329E05D
:10B31000829F90011124C091630AD091640AC20FE8
:10B32000D31F9E012D5F3F4FF901A591B491FE01FE
:10B3300094919150923010F413E01DC09091200A26
:10B340009923B1F090912C0A981711F4442381F4B9
:10B350009091360A992371F09091420A981711F44E
:10B36000442341F42091300A9091460A921710F438
:10B3700011E001C012E0E12EFF24FD01949126E1CD
:10B3800030E0E29EE001E39ED00DF29ED00D11244C
:10B39000C75FD54F9F871196BD8BAC8B8D8701E022
:10B3A000098386E1189FC0011124875F954F40E50E
:10B3B0000E943556133049F481E091E09093F209F0
:10B3C0008093F1090093F00915C08BE090E0E89EAE
:10B3D000F001E99EF00DF89EF00D1124EE0FFF1F15
:10B3E000E55FF54F812F60810E94804D812F6A8932
:10B3F0000E949F4DDF91CF911F910F91FF90EF9091
:10B4000008950F931F93082F162F0E94804D202F11
:10B4100030E08BE090E0289FF001299FF00D389FED
:10B42000F00D1124EE0FFF1FE55FF54F10831F9104
:10B430000F910895482F50E02BE030E0429FF0013B
:10B44000439FF00D529FF00D1124EE0FFF1FE55F9B
:10B45000F54F9081961B9083692F0E94804D08952F
:10B46000482F50E02BE030E0429FF001439FF00D69
:10B47000529FF00D1124EE0FFF1FE55FF54F9081F5
:10B48000690F60830E94804D08950895089508957E
:10B49000EF92FF920F931F93CF93DF93FA01949152
:10B4A00031967491E92EFF244E5F5F4F2CE3629F2B
:10B4B00090011124082F10E0200F311FC62FD0E07B
:10B4C000C70FD11D6CE370E0C69FD001C79FB00DC0
:10B4D000D69FB00D1124A00FB11F0CC0FB01049129
:10B4E00009938F5F6F5F7F4F8917C0F34E0D5F1D0C
:10B4F000245C3F4F2A173B0731F0E901C85EDE4F5D
:10B50000BA0180E0F1CFDF91CF911F910F91FF90B1
:10B51000EF9008950F931F93CF93DF938C01C0E0BA
:10B52000D0E007C00E94AE548823E1F30E94B154DA
:10B530002196C017D107B4F3DF91CF911F910F91DE
:10B5400008957F928F929F92AF92BF92CF92DF9297
:10B55000EF92FF920F931F93CF93DF93E82EF62E77
:10B56000EA016901480100E010E00EC08E2D8A0D4D
:10B57000672DA4010E948A540894A11CB11CAC162A
:10B58000BD06A4F30F5F1F4F0C151D052CF4AA2454
:10B59000BB24702E7F0CF3CFDF91CF911F910F91C1
:10B5A000FF90EF90DF90CF90BF90AF909F908F90E3
:10B5B0007F90089570E0982F969580FF12C0292FF4
:10B5C00030E086E190E0289FF001299FF00D389F40
:10B5D000F00D1124E60FF71FED56F54F80818F70A7
:10B5E0000895292F30E086E190E0289FF001299FFF
:10B5F000F00D389FF00D1124E60FF71FED56F54FB3
:10B60000808182958F700895982F969570E080FFC5
:10B6100012C0292F30E086E190E0289FF001299F99
:10B62000F00D389FF00D1124E60FF71FED56F54F82
:10B630008081807F13C0292F30E086E190E0289F31
:10B64000F001299FF00D389FF00D1124E60FF71F30
:10B65000ED56F54F80818F704295407F840F808337
:10B660000895FF920F931F93CF93DF93EC0124E093
:10B67000CC0FDD1F2A95E1F7C80FD91FCF58D54F42
:10B680000B851C85FF2443C0802F612F0E94DA5A4E
:10B69000882339F0813081F08230C9F08330B1F5F0
:10B6A00026C0802F612F44E00E94045B812F9927E0
:10B6B00087FD9095459615C0802F612F44E00E942C
:10B6C000045B802F992787FD909501961AC0802FE3
:10B6D000612F44E00E94045B812F992787FD90959C
:10B6E000019666E170E00E949866182F0FC0802FC7
:10B6F000612F44E00E94045B802F992787FD90957D
:10B70000C79668E370E00E949866082FF3942F2D87
:10B7100030E0888199812817390708F4B5CFDF9187
:10B72000CF911F910F91FF9008957F928F929F92DA
:10B73000AF92BF92CF92DF92EF92FF920F931F933F
:10B74000CF93DF9390E0EC0134E0CC0FDD1F3A950E
:10B75000E1F7C80FD91FCF58D54F1B850C8578014D
:10B76000BB24CC24DD2464C09F2CAE2C8F2D6E2DE9
:10B770000E94DA5A482F882341F08130A1F08230AC
:10B78000F9F0833051F1702E0CC08E2D992787FD72
:10B790009095459666E170E00E949866E82E702EBE
:10B7A0007A94812E27C08F2D992787FD9095019639
:10B7B00068E370E00E949866F82E812E839419C089
:10B7C0008E2D992787FD9095019666E170E00E9485
:10B7D0009866E82E702E7394E4CF8F2D992787FDFD
:10B7E0009095C79668E370E00E949866F82E812EC7
:10B7F0008A94702EDD2031F450E04E5F5F4F43702D
:10B8000050700DC01C1514F441E009C00B1514F460
:10B8100042E005C0C11614F443E001C040E0892DA8
:10B820006A2D0E94045BD394C12EB02E072D182DD3
:10B830002D2D30E0888199812817390708F494CF9D
:10B8400009858B8580270827098780278B871A859C
:10B850008C85812718271A8781278C87802F612F55
:10B860000E94DA5A8F83882339F0813041F0823088
:10B8700041F0833061F408C00D87115007C00F5F9D
:10B8800004C00D871F5F02C001500D871E87DF9126
:10B89000CF911F910F91FF90EF90DF90CF90BF90CD
:10B8A000AF909F908F907F9008958F929F92AF92CC
:10B8B000BF92CF92DF92EF92FF920F931F93CF939D
:10B8C000DF93E82EF62EC62FD0E0FE0164E0EE0FE7
:10B8D000FF1F6A95E1F7EC0FFD1FEF58F54F83E06E
:10B8E00090E091838083458314821682108A1786A4
:10B8F0001382128210869E01220F331FC90143E07A
:10B90000880F991F4A95E1F7821B930B0196880FC8
:10B91000991F63E070E045E050E021E030E000E096
:10B9200010E00E94A15A81E0E81611F58FE08093A3
:10B930007A0A1BE010937B0A8DE080937C0A1093B7
:10B940007D0A8FE06BE041E00E94045B8EE06BE0DB
:10B9500041E00E94045B8DE06BE041E00E94045BEB
:10B9600080E180937E0A10937F0AE092780A91C06A
:10B97000FF2089F41BE0912EBEE0BB2EABE0AA2E87
:10B98000F0E1CF2E88248394EBE0DE2E0DE07BE007
:10B99000E72E1FE046C08091050A833081F46AE0FB
:10B9A000962E5AE2B52E4AE0A42E38E2C32E23E0AA
:10B9B000822E9AE0D92E0BE28AE0E82E0FC00CE02E
:10B9C000902E1AE2B12EBCE0AB2EA8E2CA2EF3E014
:10B9D0008F2EECE0DE2E0BE27CE0E72E19E221C098
:10B9E0001F5F163320F40F5FB394C3941AC0FF2077
:10B9F00031F062E0B62ECC2403E011E006C0BB2497
:10BA0000B39453E0C52E00E012E0E39485E18E1577
:10BA100028F49924AA24DD24EE2403C0D39493941B
:10BA2000A394812F6E2D0E94DA5A8430C9F6802F9C
:10BA30006D2D0E94DA5A843099F68B2D692D0E9463
:10BA4000DA5A843069F68C2D6A2D0E94DA5A8430D5
:10BA500039F6812F6E2D482D0E94045B8B2D692DA8
:10BA6000482D0E94045B802F6D2D482D0E94045BA1
:10BA7000FE0144E0EE0FFF1F4A95E1F7EC0FFD1FBA
:10BA8000EF58F54FC586A6861187E2860387D486D0
:10BA90008782DF91CF911F910F91FF90EF90DF9000
:10BAA000CF90BF90AF909F908F9008958F929F926C
:10BAB000BF92CF92DF92EF92FF920F931F93CF939B
:10BAC000DF93B82E10E01EC0802F612F0E94DA5A3B
:10BAD000843058F0E82FF0E0EF5FFE4F4081802F78
:10BAE0008E5F6E2D50E00E948A540F5F083361F71D
:10BAF0001F5F163139F4C1E7DAE0E8E0EE2EF12CF1
:10BB0000DD2465C000E074E0E72EE10EDDCF19858D
:10BB10000A85812F602F0E94DA5A602F6C5FA7017F
:10BB200045505040480F511D812F8E5F0E948A540E
:10BB30000B851C85CC2447010894810891082AC0F4
:10BB4000802F612F0E94DA5A882339F0813039F032
:10BB5000823039F0833041F406C0115005C00F5FC8
:10BB600003C01F5F01C0015007FF02C007E30AC006
:10BB7000083314F000E006C0163114F010E002C0E3
:10BB800017FD15E1612F6C5F802F8E5FA4010E946D
:10BB90008A54C3942C2D30E088819981029728170C
:10BBA000390770F21B850C85812F602F0E94DA5AAD
:10BBB000602F6C5FA701480F511D812F8E5F0E947F
:10BBC0008A54D394619689E090E0E80EF91EDB1464
:10BBD00008F49DCFDF91CF911F910F91FF90EF90CF
:10BBE000DF90CF90BF909F908F900895FF920F931A
:10BBF0001F93F82E262F82E190E06FE070E041E085
:10BC000050E030E000E010E00E94A15A6F2D615F2B
:10BC100082E145E150E00E948A541F910F91FF900C
:10BC20000895FF920F931F93DF93CF930F92CDB799
:10BC3000DEB7F82E0E943B6728E330E040E050E09A
:10BC40000E94CD66162F0E943B6726E130E040E05F
:10BC500050E00E94CD66062F0E943B6726E030E050
:10BC600040E050E00E94CD66962F995F08C01F5FAC
:10BC7000183310F00F5F10E0063108F000E0812F5C
:10BC8000602F99830E94DA5A9981843081F7FF20CE
:10BC900019F4993009F49AE0812F602F492F998384
:10BCA0000E94045B602F6C5F9981E92FF0E0EF5FE9
:10BCB000FE4F4081812F8E5F50E00E948A540F908A
:10BCC000CF91DF911F910F91FF9008950F931F93D4
:10BCD0000E943B6728E330E040E050E00E94CD66E0
:10BCE000162F0E943B6726E130E040E050E00E94C2
:10BCF000CD66062F08C01F5F183310F00F5F10E0ED
:10BD0000063108F000E0812F602F0E94DA5A84305B
:10BD100091F7812F602F46E00E94045B602F6C5FDB
:10BD2000812F8E5F45E150E00E948A541F910F9150
:10BD30000895CF92DF92FF920F931F93CF93DF93DB
:10BD4000082FF62EEA01182F1B5F212F1150CE016C
:10BD50006AE070E00E948466482F822F6F2D0E9457
:10BD60009754CE016AE070E00E948466C62EE60118
:10BD70006E01D72EE601C114D10439F708C0812F16
:10BD80006F2D40E050E00E948A54115004C0C02F33
:10BD9000DD27C7FDD095812F90E08C179D077CF79C
:10BDA000DF91CF911F910F91FF90DF90CF90089579
:10BDB000EF92FF920F931F93CF93DF93EC017B01E0
:10BDC0008A0183E26FE0AE010E94995E80E00E94EA
:10BDD000B8540097D9F781E090E00E948A5A80E039
:10BDE0000E94B8549C019093FA098093F9098091BC
:10BDF000010A9091020A8095909582239323909353
:10BE0000FE098093FD0987FD04C086FD05C024FF5F
:10BE100002C0219602C025FD2197EC16FD0610F404
:10BE2000E80104C0C017D10708F4E70183E26FE01E
:10BE3000AE010E94995E8091F9099091FA09909360
:10BE4000020A8093010A8091FD099091FE098130D8
:10BE5000910509F0C0CFCE01DF91CF911F910F91D5
:10BE6000FF90EF900895FF920F931F93CF93DF936E
:10BE7000182FF62EEA01FA01449101E0403239F41C
:10BE8000812F6F2D40E050E00E948A5409C04B334F
:10BE900014F4405301C04453812F6F2D0E949754D6
:10BEA000FE01E00FF11D44911F5F442311F00F5F6D
:10BEB000E5CFDF91CF911F910F91FF900895FF92F1
:10BEC0000F931F93F82E81E190E06CE070E04AE060
:10BED00050E026E030E000E010E00E94A15A82E14C
:10BEE0006DE04BE755E90E94335F84E16FE042E883
:10BEF00055E90E94335F84E160E149E855E90E9419
:10BF0000335F07C08F2D0E94B85484FF08C01123EF
:10BF100031F080E062E00E94F65D10E00CC08F2DF1
:10BF20000E94B85485FF07C0112329F481E062E024
:10BF30000E94F65D11E08F2D0E94B854813091056A
:10BF400009F78F2D0E94B8540097D9F7812F1F91C0
:10BF50000F91FF9008952F923F924F925F926F92B0
:10BF60007F928F929F92AF92BF92CF92DF92EF9289
:10BF7000FF920F931F93DF93CF93CDB7DEB72B972D
:10BF80000FB6F894DEBF0FBECDBFD82EA62E0E94EE
:10BF9000F9558091120180FF04C08CEC95E80E9455
:10BFA000D2550E94805410E00BC0802F612F44E0D6
:10BFB0000E94045B0F5F0833C1F71F5F163111F059
:10BFC00000E0F3CF8091050A813031F0823009F131
:10BFD000833009F062C030C010E0812F60E045E09E
:10BFE0000E94045B812F65E145E00E94045B1F5FB6
:10BFF000183399F710E080E0612F45E00E94045B60
:10C0000087E3612F45E00E94045B1F5F163199F7BB
:10C0100044C010E0812F6AE045E00E94045B1F5F8E
:10C020001833C1F710E08CE1612F45E00E94045BFA
:10C030001F5F1631C1F731C010E0812F69E045E084
:10C040000E94045B8AE0612F45E00E94045B812F1F
:10C05000855F69E045E00E94045B85E1612F45E072
:10C060000E94045B812F825D6CE045E00E94045BCE
:10C07000012F045F8DE2602F45E00E94045B812F59
:10C080008D5D6CE045E00E94045B82E2602F45E03C
:10C090000E94045B1F5F1A3081F6C0900E0181E0A0
:10C0A000A81649F484E163E04AE050E00E94995EFA
:10C0B0000AE0F02E0CC092E0A91641F440910F0165
:10C0C0005091100184E163E00E94995EFF24109179
:10C0D00011018D2D60E04C2D0E94555C84E062E0E2
:10C0E00041E355E90E94335FE2E0DE1659F480E255
:10C0F00062E04BE355E90E94335F82E061E04C2D42
:10C100000E94555C19830E94665E8D2D0E94565DCB
:10C110009924EE24BD2C81E090E00E948A5AF2E03E
:10C12000AF1629F04091730A5091740A04C04091EF
:10C13000710A5091720A8DE062E00E94995E82E07D
:10C14000B81679F4A81629F04091840A5091850A0E
:10C1500004C04091820A5091830A89E262E00E9401
:10C16000995E93E0E91629F48C2D0E94115E14E08B
:10C17000E12E9394ECE39E1631F4F3E0AF16D9F57B
:10C18000FA94992403C083E0A816B1F5F7FE05C020
:10C19000998191509983BBE3FB2E8EE063E04EE6DC
:10C1A00055E90E94335FE9814E2F552747FD509591
:10C1B00083E163E00E94995E4F2D552747FD50951E
:10C1C0008AE163E00E94995EF981FF2369F5FF200F
:10C1D00059F5DB2C2091730A3091740A8091840AFE
:10C1E0009091850A8217930708F47CC328173907B2
:10C1F00008F47AC374C3992482E0A816A9F4809144
:10C200000F01909110012091710A3091720A281744
:10C21000390709F466C32091820A3091830A2817EE
:10C22000390761F5DB2C60C391E0A91639F5992037
:10C2300059F4CC2049F0FA944F2D552747FD5095DD
:10C2400084E163E00E94995EFF20C1F480911201B5
:10C2500081FF05C084E06FEF41E00E948159CA94DC
:10C260008091790A882311F4C092760A80918A0A13
:10C27000882311F4C092870AAAE0FA2E21E73AE057
:10C28000E9EFF9E0FF83EE8381E09AE09D838C8300
:10C29000FDEF6F2EF9E07F2EE2E0F0E0FB83EA8312
:10C2A0008824839444245524DD24332433943B8709
:10C2B0002A87DFC28D2D0E94B8549C01EE81FF8138
:10C2C00091838083EC81FD8180819181809590951F
:10C2D00082239323F30191838083992009F5EA85D2
:10C2E000FB8580858823E1F0815080874091790A21
:10C2F000882D63E050E00E94995EEA85FB85808589
:10C30000882371F4C58214828A819B8163E070E086
:10C3100045E050E021E030E000E010E00E94A15A4A
:10C32000F301108114FF20C0EA85FB850285818519
:10C33000602F0E94DA5A823039F0EA85FB859481B9
:10C34000992339F0882381F0EA85FB85848188234D
:10C3500059F0EA85FB858481882311F00F5F27C09F
:10C360000150EA85FB851DC015FF29C0EA85FB85C4
:10C3700002858185602F0E94DA5A882339F0EA8588
:10C38000FB859481992339F08230C9F0EA85FB85D9
:10C3900084818823A1F0EA85FB858481882321F0AC
:10C3A00001500687178206C00F5FEA85FB85068766
:10C3B00082E08783EA85FB858185858758C016FFE3
:10C3C00020C0EA85FB850185802F62850E94DA5AAC
:10C3D000813039F0EA85FB859481992339F08330E7
:10C3E00081F0EA85FB858481882359F0EA85FB8505
:10C3F0008481882311F00F5F28C00150EA85FB85F6
:10C400001DC017FF29C0EA85FB850185802F628545
:10C410000E94DA5A833039F0EA85FB8594819923AA
:10C4200039F08130C9F0EA85FB8584818823A1F049
:10C43000EA85FB858481882329F00150058783E004
:10C44000878305C00F5FEA85FB8505873782EA850C
:10C45000FB85828586870BC013FF09C08D2D0E9446
:10C460005F5F882309F042C28B2D0E94565DEA85EA
:10C47000FB8596818581981708F4D5C181856285F1
:10C4800047810E94045BEA85FB858585883314F02B
:10C49000158606C087FF04C087E3EA85FB8585878C
:10C4A000EA85FB858685863114F0168606C087FFEF
:10C4B00004C085E1EA85FB858687EA85FB8585855D
:10C4C00066850E94DA5A182F843010F08530F1F416
:10C4D000F1E0FA1528F012E01D1909F41CCECDC1C7
:10C4E0008091120181FF05C082E06FEF41E00E9460
:10C4F00081598D2D90E00E94315B8B2D6D2D4C2D3F
:10C500000E94555C8B2D0E94565D05CE8630F9F455
:10C510008091120181FF05C083E06FEF41E00E942E
:10C520008159EA85FB85878590890196908B87875D
:10C530000E94665EEA85FB858281938101969383E2
:10C540008283F2E0FE1508F485C0E39483C088304E
:10C5500089F48091120181FF05C083E06FEF41E013
:10C560000E948159EA85FB85878590890396908B87
:10C5700087871FC08C3019F58091120181FF05C09B
:10C5800083E06FEF41E00E948159EA85FB852081BD
:10C590003181878590892630310510F0039705C0D9
:10C5A000821B930B0396EA85FB85908B8787EA8530
:10C5B000FB85828193810596938382834AC08B3069
:10C5C00079F48091120181FF05C083E06FEF41E0B3
:10C5D0000E9481598AE0EA85FB85808734822DC0DC
:10C5E000893089F48091120181FF05C083E06FEFEB
:10C5F00041E00E9481598AE0EA85FB858087858138
:10C60000869585831AC08A3029F58091120181FFB1
:10C6100005C083E06FEF41E00E9481598AE0EA851E
:10C62000FB8580878581882311F4358204C0880FBB
:10C63000EA85FB858583EA85FB8582819381059662
:10C64000938382834091790A882D63E050E00E94B1
:10C65000995EEE24EA85FB8516828585668547818D
:10C660000E94045BEA85FB85818562856C5FA2017F
:10C67000495F5F4F8E5F0E948A54EA85FB858585FE
:10C680008187668562876C5F478150E04D5F5F4FB1
:10C69000440D551D8E5F0E948A54EA85FB85878173
:10C6A000882339F0813051F0823069F08330B1F461
:10C6B00010C0EA85FB858685815009C0EA85FB8527
:10C6C00085858F5F0AC0EA85FB8586858F5F8687B3
:10C6D00005C0EA85FB85858581508587EA85FB85D0
:10C6E000278530891216130624F4808191810196E2
:10C6F00009C02115310541F0EA85FB8580819181D2
:10C70000820F931F91838083EA85FB8587859089BB
:10C710000197908B8787C20108969987888764C0A4
:10C72000EA85FB85838564856C5F8E5F41E050E020
:10C730000E948A54EA85FB8523840485822D602F1C
:10C740000E94DA5A882339F0813041F0823049F072
:10C750008330B9F40CC0802F815005C0822D8F5FCB
:10C7600008C0802F8F5FEA85FB85848705C0822DF6
:10C770008150EA85FB858387822D602F44E00E94EB
:10C78000045BEA85FB858385883314F0138606C035
:10C7900087FF04C087E3EA85FB858387EA85FB85FD
:10C7A0008485863114F0148606C087FF04C085E1B5
:10C7B000EA85FB858487EA85FB8503852484802FB1
:10C7C000622D0E94DA5A622D6C5F48855985480FA8
:10C7D000511D802F8E5F0E948A54EA85FB858785D4
:10C7E00090890196908B8787EA85FB85878590895C
:10C7F00097FD96CF1730B9F48091120181FF05C0E3
:10C8000083E06FEF41E00E9481598D2D0E94955B7E
:10C810008B2D0E94565DEA85FB858281938105966A
:10C8200093838283EE24EA85FB8586818F5F8683EE
:10C83000EE81FF8181919191FF83EE83EC81FD81F7
:10C8400081939193FD83EC83D3948A859B85419654
:10C850009B878A87E9E0F0E04E0E5F1EFCE18F0EB9
:10C8600082E090E0680E791EEA81FB817C96FB8372
:10C87000EA83DB1408F41ECD4ECCDB2C1430B0F56B
:10C880008091120181FF05C085E06FEF41E00E94B9
:10C8900081598D2D0E94565DF1E0DF1629F48AE161
:10C8A0006BE045E455E912C0113029F488E16BE0F2
:10C8B0004FE455E90BC0123029F488E16BE04CE5F8
:10C8C00055E904C08AE16BE049E655E90E94335F0F
:10C8D00080E00E94B85488309105D1F707C013E07A
:10C8E000CFCFDB2C11E0CCCF12E0CACF2B960FB606
:10C8F000F894DEBF0FBECDBFCF91DF911F910F9196
:10C90000FF90EF90DF90CF90BF90AF909F908F906F
:10C910007F906F905F904F903F902F9008959F92DF
:10C92000AF92BF92CF92DF92EF92FF920F931F933D
:10C93000CF93DF930E94F9558091120180FF04C0CC
:10C9400081E890E90E94D2550E94805487E064E01B
:10C950004EEC50E00E94485A88E164E04EE551E018
:10C960000E94485A87E264E046EA51E00E94485A31
:10C9700085E16BE046EA50E00E94485A86E165E1B5
:10C980004EEE53E90E94335F82E166E142E054E9F2
:10C990000E94335F80E167E14CE154E90E94335F1C
:10C9A0008FE068E14AE354E90E94335F83E169E183
:10C9B0004AE554E90E94335FC3E7D4E91FE084E10C
:10C9C000612FAE010E94335F1F5F2B961431B9F7C0
:10C9D00080E065E00E94F65D83E260E14AEC54E9A4
:10C9E0000E94335F40910E0183E261E150E00E94BA
:10C9F000995E4091050A50E033E0440F551F3A9587
:10CA0000E1F746555B4683E262E10E94335F409165
:10CA100012018EE0489FA001112446515B4683E23B
:10CA200063E10E94335FEE24FF24AA24BB24650146
:10CA30002EE0922E81E090E00E948A5A0894A11C78
:10CA4000B11CC11CD11C80E00E94B8549C01909381
:10CA5000FA098093F9098091010A9091020A809560
:10CA60009095822393239093FE098093FD0984FF80
:10CA700003C024E0F20EA9C085FF02C0F394A5C054
:10CA800080FF12C0FF2031F4C601B5010E9440674B
:10CA900080E0ACC021E0F21639F4C601B5010E9475
:10CAA00040678E2D8F5FA2C087FF2BC06F2D70E077
:10CAB000615F7F4F83E290E04FE050E021E030E0A3
:10CAC00000E010E00E94A15A81E0F81621F4E394FE
:10CAD00023E0E2222CC082E0F81621F440910E01FE
:10CAE0004F5F39C023E0F21621F44091050A4F5FF1
:10CAF00041C084E0F81609F068C0409112014F5F10
:10CB00004DC086FF62C06F2D70E0615F7F4F83E292
:10CB100090E04FE050E021E030E000E010E00E94C3
:10CB2000A15A21E0F21689F4EA9483E0E8224E2D1E
:10CB300050E093E0440F551F9A95E1F746535B464A
:10CB400083E260E10E94335F40C022E0F21661F4AC
:10CB500040910E0141504F7140930E0183E261E11B
:10CB600050E00E94995E31C083E0F81689F440914C
:10CB7000050A415043704093050A50E083E0440F9A
:10CB8000551F8A95E1F746555B4683E262E1DACFAD
:10CB900024E0F216D1F440911201415043704093C9
:10CBA0001201499DA001112446515B4683E263E1D5
:10CBB0000E94335F8091120180FF05C081E890E9F7
:10CBC0000E94D25502C00E94F9558F2D65E00E9447
:10CBD0007866F92E892F0E94F65D8091F90990916F
:10CBE000FA099093020A8093010A24CFDF91CF9132
:10CBF0001F910F91FF90EF90DF90CF90BF90AF907B
:10CC00009F9008958DE895E80E94B75580EB0E94AB
:10CC100044568EEE91E00E94A9548DE30E94A654E2
:10CC20000E94805480E16BE04EEC50E00E94485A34
:10CC30008FE16BE046E151E00E94485A8EE190E0BE
:10CC40000E948A5A86E06FEF41E00E9481598AE58E
:10CC500090E00E948A5A0E948F64882349F08130B4
:10CC600049F0823051F0833059F08430A1F721C06F
:10CC700081E001C082E060E038C082E061E035C060
:10CC80000E94805484E16FE04BE255E90E94335FDB
:10CC900080910F019091100164EF71E044E050E049
:10CCA0000E94D85E9093100180930F0182E062E0B1
:10CCB0001CC00E94805484E16FE042E255E90E946A
:10CCC000335F4091110183E26FE050E00E94995E72
:10CCD0008091110190E06AE070E041E050E00E9434
:10CCE000D85E8093110182E063E00E94AB5FB3CF16
:10CCF000991B79E004C0991F961708F0961B881FAE
:10CD00007A95C9F780950895AA1BBB1B51E107C00E
:10CD1000AA1FBB1FA617B70710F0A61BB70B881FCB
:10CD2000991F5A95A9F780959095BC01CD0108955A
:10CD300097FB092E07260AD077FD04D0E5DF06D041
:10CD400000201AF4709561957F4F0895F6F790953D
:10CD500081959F4F0895A1E21A2EAA1BBB1BFD01CE
:10CD60000DC0AA1FBB1FEE1FFF1FA217B307E407CA
:10CD7000F50720F0A21BB30BE40BF50B661F771F22
:10CD8000881F991F1A9469F7609570958095909502
:10CD90009B01AC01BD01CF01089597FB092E05262B
:10CDA0000ED057FD04D0D7DF0AD0001C38F45095C0
:10CDB0004095309521953F4F4F4F5F4F0895F6F7BF
:10CDC00090958095709561957F4F8F4F9F4F0895F7
:10CDD000A0E0B0E0EEEEF6E60C947067EC01E880BF
:10CDE000F9800A811B81E114F1040105110541F468
:10CDF00084E2E82E89EDF82E8BE5082F87E0182FC6
:10CE0000C801B7012DE133EF41E050E00E94CD664B
:10CE100027EA31E440E050E00E9449675B016C0181
:10CE2000C801B7012DE133EF41E050E00E94CD662B
:10CE3000CA01B9012CEE34EF4FEF5FEF0E94496752
:10CE40009B01AC012A0D3B1D4C1D5D1D57FF04C00D
:10CE50002150304040405048288339834A835B83C7
:10CE60005F77B901CA01CDB7DEB7EAE00C948C67F1
:10CE70000E94E866089583E191E00E94E8660895C3
:10CE80006093130170931401809315019093160120
:10CE90000895629FD001739FF001829FE00DF11D04
:10CEA000649FE00DF11D929FF00D839FF00D749F24
:10CEB000F00D659FF00D9927729FB00DE11DF91FD0
:10CEC000639FB00DE11DF91FBD01CF01112408952D
:10CED0002F923F924F925F926F927F928F929F928A
:10CEE000AF92BF92CF92DF92EF92FF920F931F9378
:10CEF000CF93DF93CDB7DEB7CA1BDB0B0FB6F89429
:10CF0000DEBF0FBECDBF09942A88398848885F8468
:10CF10006E847D848C849B84AA84B984C884DF80D9
:10CF2000EE80FD800C811B81AA81B981CE0FD11DBD
:10CF30000FB6F894DEBF0FBECDBFED010895F89493
:02CF4000FFCF21
:10CF42000400000000010215161718191A1B031E0F
:08CF52000002030100000000D1
:00000001FF
